:100000005446495300010000042E020055BD223E13
:1000100009140104160530094E36593009140151EE
:10002000160530094E3659300914010516053009F8
:100030004E36594C03000000000000000000000094
:1000400054464353002000007C0E020000000000D4
:1000500000000210012100002521000027210000DE
:10006000292100002B2100002D2100003D2100004E
:100070003D2100003D2100003D2100002F21000016
:10008000312100003D21000033210000935F00007A
:1000900093600000372100003D2100004DF9001061
:1000A000372100007F3E0000853E00003D2100001A
:1000B0003D210000C35A0000615000008B3E00004B
:1000C000C9570000372100003D2100003D210000FC
:1000D0000000000000000000000000000000000020
:1000E0000000000000000000000000000000000010
:1000F0000000000000000000000000000000000000
:1001000000000000000000000000000000000000EF
:1001100000000000000000000000000000000000DF
:1001200000000000000000000000000000000000CF
:1001300000000000000000000000000000000000BF
:1001400000000000000000000000000000000000AF
:1001500000F003F800F020F8FEE70D480168890878
:100160008900002001C101C101C101C17047000027
:100170006CFE0010FEE7FEE7FEE7FEE7FEE7FEE7A7
:10018000FEE7FEE7FEE703480047FEE7FEE7000064
:10019000202100003D21000000F002F800F068F886
:1001A0000AA090E8000C82448344AAF10107DA45D2
:1001B00001D100F05DF8AFF2090EBAE80F0013F0BC
:1001C000010F18BFFB1A43F001031847BC0D0100D3
:1001D000EC0D01000A444FF0000C10F8013B13F045
:1001E000070408BF10F8014B1D1108BF10F8015B90
:1001F000641E05D010F8016B641E01F8016BF9D183
:1002000013F0080F1EBF10F8014BAD1C0C1B09D1D9
:100210006D1E58BF01F801CBFAD505E014F8016B4B
:1002200001F8016B6D1EF9D59142D6D370470000DD
:10023000103A24BF78C878C1FAD8520724BF30C812
:1002400030C144BF04680C607047000000230024E4
:1002500000250026103A28BF78C1FBD8520728BFD6
:1002600030C148BF0B6070471FB51FBD10B510BD32
:10027000DFF80CD0FFF7F8FF05F0F4F810F04CF8B9
:100280000000021003B4FFF7F1FF03BC10F04CF8BC
:1002900008B5002103200B460A4600910FF050FBE1
:1002A00008BD38B5EC4D0024AC80EC802C810FF0FB
:1002B00024FB2861FF206870E8482346224604603A
:1002C000446004720120A8700320214600940FF0BE
:1002D00037FB012038BD38B5DF4D02286C78224647
:1002E0000DD0052810D0A24208BF38BD002003461B
:1002F0000246214600900FF023FB6C7038BD0229A6
:1003000014BF01240224EEE7022914BF64246524EB
:10031000E9E738B5D24BD34C0A461B7824784FF026
:10032000010C6343002401465B00604600940FF01B
:1003300007FB38BD38B54FF0010C062400250B46ED
:1003400002462146604600950FF0FAFA38BD2DE9C5
:10035000F04104460127002503F00700BE4E884601
:10036000012804BF0020308146D0022844D13089C2
:1003700004280BD2002818BFF06802D10FF001FB4F
:10038000F06010F8011B2170F0602EE0062808D202
:100390000FF0F9FA3189C1F10501C900C840207098
:1003A00023E0082808D20FF0F2FA3189C1F10701E1
:1003B000C900C840207018E00C2808D20FF09DFA40
:1003C0003189C1F10B01C900C84020700DE00E2831
:1003D00008D20FF094FA3189C1F10D01C900C8406B
:1003E000207002E0FF20207000273089401C80B27E
:1003F00030810E2828BF012588F800503846BDE816
:10040000F08130B403F007000024DFF84CC201286B
:100410000BD06046BCF808308088022B0CD2120248
:1004200042EA1020ACF804000CE0ACF80440ACF850
:100430000640ACF8084008E0DCF8105018442844A6
:1004400000F8022C581CACF808000C7030BC0020DE
:100450007047F0B40746002003F007047E4D0646BF
:10046000012C08BF2E8117D0DFF8ECC1022CBCF89C
:1004700006C003D013F0070F0AD00DE028892B69BE
:100480000CEB0002401C9A5C3A702881012003E0CA
:10049000120242EA1C22EA800E70F0BC704738B5A6
:1004A00003F0070000240D4601280AD16A482146BE
:1004B0000B4604818480C48002200A4600940FF019
:1004C0003FFA2C70002038BD30B583B0DDE9064519
:1004D00000EB051C002C18BF022C16D00021012CAB
:1004E0006CD0032C1CBF03B030BD0F22027003225E
:1004F000427041808180C180018141818181817B05
:1005000021F00101817303B030BD0CF8105C0CF8D0
:100510000F4CB1F8AC302CF80E3CB1F8AE302CF8E2
:100520000C3C91F88A302CF80A3C91F88B302CF86E
:10053000083C91F88C302CF8063C8B8A2CF8043C53
:1005400092F848301CF8022C63F300020CF8022CDD
:1005500091F8E820012A1CBF03B030BD62228DF85B
:10056000002091F891208DF8012091F8912000EB66
:10057000021232F80E2C120A8DF8022091F8912006
:1005800000EB021212F80E2C8DF8032091F8912046
:1005900000EB021232F80C2C120A8DF8042091F8AC
:1005A0009110062200EB0110694610F80C0C8DF832
:1005B000050001200BF07EFA03B030BD0CF8105C92
:1005C00001200CF80F0C2CF80E1C2CF80C1C2CF82D
:1005D0000A1C2CF8081C2CF8061C2CF8041C1CF80F
:1005E000020C062220F001000CF8020C63208DF8AA
:1005F00000008DF8015058886946000A8DF8020005
:1006000098788DF803009888000A8DF8040018790E
:100610008DF8050001200BF04DFA03B030BD0E49F6
:100620000020087070470C48007870470A49012084
:1006300008707047094A1154704700225A2101205E
:100640000BF011BA70470449002818BF01208870C8
:100650007047014880787047000001105003011076
:10066000CA000110CB0001107047FE480068D0F8A6
:10067000C00000F00100704710B5044601F0ADFB6A
:1006800000280CBF012100212142F64909D0086849
:10069000D0F8C00010F0010F03D00A68002090606D
:1006A00002E00A6801209060002C14BF01200020A5
:1006B0000968086210BDEB480068006A002818BF8E
:1006C00001207047E74A126802EBC000416370479F
:1006D000E449096801EBC000006B00F480707047CA
:1006E000E04A1021126802EBC00041637047DD4907
:1006F0000A68D2F8402160F30D220868C0F8402152
:100700007047D8480068D0F84001C0F30520704712
:10071000D44A00F00F03C0F303101268002902EB63
:10072000C31202EB4010D0F8401114BF41F0010198
:1007300021F00101C0F840117047CA4A00F00F01D2
:10074000C0F30310126802EBC11101EB4010D0F8A6
:10075000400100F001007047C2494FF0000C0A68E8
:10076000C2F820C003680A68136042680B685A60C8
:1007700082680B689A60C2680B68DA60426A0B682C
:100780001A64826A0B685A6403690A689361426951
:100790000B68DA61426B0B681A66836B0A68136731
:1007A000C26B0B685A67026C0B689A67426C0B68E5
:1007B000C3F88020826C0B68C3F88420C26C0B687D
:1007C000C3F88820026D0B68C3F88C20026E0B689A
:1007D000C3F89C20426E0B68C3F8A020826E0B68A1
:1007E000C3F8A420C26E0B68C3F8A820C26F0B68C0
:1007F000C3F8C020D0F880300A68C2F8C430D0F8FE
:1008000084200B68C3F8C820D0F888200B68C3F890
:10081000CC20D0F88C200B68C3F8D020D0F89C20D6
:100820000B68C3F8E020D0F8A4200B68C3F8F020D0
:10083000D0F8A8200B68C3F8F420D0F8AC200B68DF
:10084000C3F8F820D0F8B0300A68C2F8FC300B6862
:1008500021225A630B68DA63C2690B685A62C26A62
:100860000B689A64026B0B68DA64026F0B68C3F85A
:10087000AC20D0F890300A68C2F8D430D0F8942078
:100880000B68C3F8D820D0F8A0200B68C3F8E42088
:10089000426F0B68C3F8B020826F0B68C3F8B420B6
:1008A000D0F8F8210B68C3F88022D0F8FC210B683F
:1008B000C3F88422D0F800220B68C3F88822D0F84D
:1008C00004220B68C3F88C22D0F808320A68C2F8F8
:1008D0009032D0F80C220B68C3F89422D0F8102282
:1008E0000B68C3F89822D0F814220B68C3F89C2236
:1008F000D0F818220B6822F48032C3F8B022D0F866
:10090000B4200B68C3F80021D0F8B8200B68C3F8F6
:100910000421D0F8BC200B68C3F80821D0F8C0200F
:100920000B68C3F80C21D0F8C4200B68C3F8102161
:10093000D0F8C8200B68C3F81421D0F8CC200B687D
:10094000C3F81821D0F8D0200B68C3F81C21D0F8C8
:10095000D4200B68C3F82021D0F8D8200B68C3F846
:100960002421D0F8DC200B68C3F83021D0F8E02037
:100970000B68C3F84021D0F8E4200B68C3F8442189
:10098000D0F8E8200B68C3F84821D0F8EC200B68B9
:10099000C3F84C21D0F8F0200B68C3F85021D0F8F0
:1009A000F4200B68C3F85421D0F8F8200B68C3F882
:1009B0005821D0F8FC200B68C3F85C21D0F8202126
:1009C0000B68C3F88021D0F824210B68C3F8842178
:1009D000D0F828210B68C3F88821D0F82C210B68A7
:1009E000C3F88C21D0F830210B68C3F89021D0F8DF
:1009F00034210B68C3F89421D0F838210B68C3F870
:100A00009821D0F83C210B68C3F89C21D0F84031E4
:100A10000A68C2F8A031D0F844210B68C3F8A421B9
:100A2000D0F848210B68C3F8B021D0F84C210B68EE
:100A3000C3F8C021D0F850210B68C3F8C421D0F806
:100A400054210B68C3F8C821D0F858210B68C3F8AB
:100A5000CC21D0F85C210B68C3F8D021D0F86021FC
:100A60000B6801E0E02B0100C3F8D421D0F8642129
:100A70000B68C3F8D821D0F868210B68C3F8DC21D3
:100A8000D0F86C210B68C3F8E021D0F870210B6816
:100A9000C3F8E421D0F874210B68C3F8E821D0F83A
:100AA00078210B68C3F8EC21D0F87C210B68C3F8DF
:100AB000F021D0F880210B68C3F8F421D0F88431FC
:100AC0000A68C2F8F831D0F888210B68C3F8FC2115
:100AD000D0F88C210B68C3F80022D0F890210B6865
:100AE000C3F80422D0F894210B68C3F80822D0F888
:100AF00098210B68C3F80C22D0F89C210B68C3F82E
:100B00001022D0F8A0210B68C3F81422D0F8A42139
:100B10000B68C3F81822D0F8A8210B68C3F81C2270
:100B2000D0F8AC210B68C3F82022D0F8B0210B68B4
:100B3000C3F82422D0F8B4210B68C3F83022D0F8CF
:100B4000B8210B68C3F84022D0F8BC210B68C3F869
:100B50004422D0F8C0210B68C3F84822D0F8C42141
:100B60000B68C3F84C22D0F8C8210B68C3F8502298
:100B7000D0F8CC210B68C3F85422D0F8D0210B68F0
:100B8000C3F85822D0F8D4210B68C3F85C22D0F8FF
:100B9000D8210B68C3F86022D0F8DC210B68C3F8B9
:100BA0006422D0F8E0210B68C3F86822D0F8E42171
:100BB0000B68C3F86C22D0F8E8210B68C3F87022E8
:100BC000D0F8EC210B68C3F87422D0F8F0210B6840
:100BD000C3F87822D0F8F4210B68C3F87C22FE4ACF
:100BE000126832F0FF0307D10B68D3F8903062F33C
:100BF00003030A68C2F89030F84A82F801C0C36F54
:100C000013F0010F1CBF01235370D0F88C3013F088
:100C1000010F03D0537843F0020353700B68D3F8ED
:100C2000C030D1F800C023F00103CCF8C0300B680D
:100C3000D3F8D030D1F800C023F00103CCF8D03085
:100C4000D0F8900010F0010F03D0507840F004006D
:100C500050700868D0F8D400096820F00100C1F88D
:100C6000D4007047DD4800787047DC4880787047D2
:100C7000DA49C8707047D948C0787047D74988604A
:100C80007047D7480068C06870472DE9F047DFF823
:100C90004C93D34C064610F0010F18BF16F4801F7A
:100CA0007ED001F089F800287AD099F8010040F050
:100CB000020089F801002068D0F8AC00216820F01B
:100CC0000800C1F8AC002068D0F800022168C1F823
:100CD00080012068D0F804022168C1F884012068EE
:100CE000D0F808022168C1F888012068D0F80C0209
:100CF0002168C1F88C012068D0F810022168C1F881
:100D000090012068D0F814022168C1F8940120688D
:100D1000D0F818022168C1F898012068D0F81C02A8
:100D20002168C1F89C012068D0F820022168C1F830
:100D3000A0012068D0F824022168C1F8A40120682D
:100D4000D0F830022168C1F8B0012068D0F8400224
:100D50002168C1F8C0012068D0F844022168C1F8B8
:100D6000C4012068D0F848022168C1F8C801206891
:100D7000D0F84C022168C1F8CC012068D0F85002AC
:100D80002168C1F8D0012068D0F854022168C1F868
:100D9000D4012068D0F858022168C1F8D80100E0D9
:100DA00035E02068D0F85C022168C1F8DC012068D9
:100DB000D0F860022168C1F8E0012068D0F8640230
:100DC0002168C1F8E4012068D0F868022168C1F800
:100DD000E8012068D0F86C022168C1F8EC012068B5
:100DE000D0F870022168C1F8F0012068D0F87402D0
:100DF0002168C1F8F4012068D0F878022168C1F8B0
:100E0000F8012068D0F87C022168C1F8FC0199F84B
:100E1000010099F8031016F4003F00EA010518BF1D
:100E200025F0010516F4802F18BF25F0020516F4F1
:100E3000002F18BF25F004052068D0F8B002216803
:100E400020F48030C1F8B00215F0070F72D020688E
:100E5000D9F808704FF00008D0F8B802216840F0C7
:100E60000100C1F8B8022068D0F8B802216820F06B
:100E70000100C1F8B8022068D0F8B002216840F43F
:100E80008030C1F8B00240F2E73A0FE003F023F9F6
:100E900050462168D1F8B81211F0010F02D04FF07E
:100EA000010803E0011EA0F10100F2DC381EA7F1E9
:100EB000010702DDB8F1000FE8D0B8F1000F39D01A
:100EC000206815F0010FD0F8C0000CBF20F0010021
:100ED00040F001002168C1F8C000206815F0020F41
:100EE000D0F8D00014BF40F0010020F001002168CC
:100EF000C1F8D000206815F0040FD0F8D40014BF5A
:100F000040F0010020F001002168C1F8D40089F808
:100F10000250012089F80000D9F80400C9F808003F
:100F20002068D0F8B002216840F48030C1F8B002E7
:100F300045E0FFE72068D0F8C000216820F00100FC
:100F4000C1F8C0002068D0F8D000216820F001006E
:100F5000C1F8D0002068D0F8D400216820F001004A
:100F6000C1F8D400002089F80200F5B1022089F808
:100F700000000120C9F808002068D0F8B0022168FC
:100F800040F48030C1F8B0022068D0F8B80221687F
:100F900040F00100C1F8B8022068D0F8B80221681A
:100FA00020F00100C1F8B80209E02168D1F8B012C0
:100FB000226821F48031C2F8B01289F8000020685C
:100FC000D0F8400116F0020F20F00D0018BF40F0DD
:100FD000010016F0080F05E0E0FE03001400011008
:100FE000E02B010018BF40F0040016F0040F18BFFA
:100FF00040F008002168C1F8400116F0010F44D00C
:1010000001F0C9F8054601F0C9F801462068C0683A
:1010100000280EBF28460846294600282068D0F838
:10102000C00114BF40F0010020F001002268C2F8A6
:10103000C00141B12068D0F8E001216840F0010012
:10104000C1F8E00107E02068D0F8E001216820F055
:101050000100C1F8E00116F0200F18BF00251DD0D7
:10106000284601F0A2F80028206800EB4510D0F8CF
:10107000401214BF41F0010121F00101C0F84012FB
:101080006D1C022DECD3BDE8F0872068D0F8C001BC
:10109000216820F00100C1F8C001D4E72068D0F831
:1010A0004002216820F00100C1F840022068D0F819
:1010B0006002216820F00100C1F86002BDE8F087FD
:1010C0002DE9F003FA49024602F00F03D1F800C0FF
:1010D00000200CEBC315C2F3031305EB4313D3F845
:1010E000403113F0010F0DD142F01003C3F303138D
:1010F00005EB4313D3F8403113F0010F04BFBDE8F3
:10110000F00370470CEBC214D4F81C31DCF81C104F
:10111000C3F3080901F00807D4F800111FFA81F899
:10112000002142EA0113C3F3031305EB4313D3F881
:10113000403113F0010F14D004EB4113D3F844C134
:10114000CCF3080617F1000C1CBFD3F844C1CCF354
:10115000023CD3F8403106FA0CFCC3F3054360446B
:101160001844491C0229DCD300FB08F0C9EB091123
:10117000BDE8F00300EB4100704770B5CC4E30681D
:10118000006800F01F040120FFF79AFF05460220C7
:10119000FFF796FF054400F0E8FB31682844D1F8DA
:1011A000C01011F0010F09D03168D1F8C410C1F39B
:1011B00009016143C1EB011100EB41004FF47A7169
:1011C000484347F23051B0FBF1F070BD2DE9F041DA
:1011D000B74E05463068006810F01F0408BF0124B0
:1011E0000120FFF76DFF07460220FFF769FF074464
:1011F00000F0BBFB3918AF4F002D18BF002953D0AA
:1012000030680022D0F8C00010F0010F37D07820ED
:10121000B0EB151F306809D9D0F8CC00336820F046
:101220000F0040F00100C3F8CC002DE0D0F8C4005E
:10123000A14BC0F309006043A0EB001003EB400C8E
:101240009E48A0FB0530430ABCFBF1F0102828BFE4
:101250000F20834298BF1846002808BF012005D000
:10126000012884BF00FB11C2B2FBF0F23368D3F84F
:10127000CC3060F303033068C0F8CC3004E0B7FB37
:10128000F5F0884288BF421AC4EB04104000B2FB5C
:10129000F0F0B0F5005F28BF41F6FF703268526889
:1012A00060F30C023068426030684068C0F30C00A4
:1012B0006043C0EB001001EB4000B7FBF0F0BDE86D
:1012C000F08170B57A4801680968006801F01F056F
:1012D0004068C0F30C060120FFF7F2FE044602202E
:1012E000FFF7EEFE044400F040FB06FB05F1C1EB06
:1012F000011104EB410108446E49B1FBF0F070BDEF
:101300006B480068D0F8CC0000F00F0070476849C7
:101310000A6852680B68C2F30C025B6860F30C0346
:101320000868436010467047614800684068C0F331
:101330000C0070475E49096801EBC010D0F800014D
:101340004EF6602180B2B1FBF0F0401C40087047BF
:1013500030B44EF6602331B1B3FBF1F1491C4A08B9
:10136000B2F5804F01D343F6FF72B3FBF2F1491C93
:101370004D084F4953080028096801EBC01107BF09
:10138000981FA3F10C0CD1F8040180B218BFA2F190
:10139000060C2CF0010CD1F8004162F30F04C1F8E7
:1013A0000041D1F8002163F31F42C1F80021D1F8B8
:1013B000042160F30F02C1F80421D1F810016CF38D
:1013C0000F00C1F81001284630BC70473849096841
:1013D00001EBC010D0F80001000C7047344B1A68C4
:1013E00002EBC012D2F800C161F31F4CC2F800C179
:1013F000002818BF7047881F1A680C3921F00101B6
:10140000D2F8042160F30F021868C0F804211868AC
:10141000D0F8100161F30F001968C1F8100170478E
:10142000234A00F00F01C0F30310126802EBC11150
:1014300001EB4010D0F84401C0F3080070471C4A8B
:1014400000F00F03126802EBC312D2F81431C0F39C
:10145000031002EB4010CB1AD0F8442161F30802CC
:10146000C0F84421D0F844119B1E63F31841C0F822
:10147000441170470E490A68D269096812F0100FCA
:1014800000F00F0201EBC211D1F82021C0F30310CC
:1014900001EB4010D2B2D0F84401C0F3080008BFFD
:1014A0000022801A0004000C08BF012070470000D1
:1014B000E02B010000389C1C1B810700898888886C
:1014C0004FEA101C0007C00EFC4B02FA00F01B682C
:1014D00003EBCC1303EB810101F5C0410B6818430A
:1014E00008607047F54B020900071B68C00E03EB4C
:1014F000C21202EB810101F5C041096821FA00F036
:1015000000F003007047EE4B00F00F02C0F3031031
:101510001B6803EBC21202EB4010C0F84C1170477D
:10152000E74A00F00F01C0F30310126802EBC1118B
:1015300001EB4010D0F84C017047E14B00211A68D4
:10154000D26912F0080F0CD000F00F011A68C0F336
:10155000031002EBC11101EB4010D0F84401C0F3BD
:10156000023108467047D64A1368DB69D2F800C0DA
:1015700043F00803CCF81C3000F00F031268C0F3EE
:10158000031002EBC31202EB4010D0F8442161F3C8
:101590000E32C0F844217047C94B00211A68D26945
:1015A00012F0080F0CD000F00F011A68C0F30310FE
:1015B00002EBC11101EB4010D0F84801C0F3024129
:1015C00008467047BE4A00F00F03C0F303101268CC
:1015D00002EBC31202EB4010D0F8482161F3124233
:1015E000C0F848217047042988BF704730B40023F1
:1015F000B34C2268D269254612F0080F00F00F02A2
:101600002D68C0F3031005EBC21202EB40121CBFA1
:10161000D2F84401C0F302330020D4F800C0DCF853
:101620001CC01CF0080F1CBFD2F84801C0F30240D8
:10163000C91A0844042803DD081A011D042003E028
:101640000028BCBF0144002019442368DB69D4F89A
:1016500000C043F00803CCF81C30D2F8443161F3E9
:101660000E33C2F84431D2F8481160F31241C2F887
:10167000481130BC7047924900280868806904D03E
:10168000096840F0080088617047096820F0080088
:10169000886170478A4800688069C0F3C00070475D
:1016A000874A00F00F01C0F30310126802EBC1116A
:1016B00001EB4010D0F8480180B27047804B002108
:1016C0001A68D26912F0080F0CD000F00F011A68E6
:1016D000C0F3031002EBC11101EB4010D0F8480138
:1016E000C0F30051084670470120704730B4022A09
:1016F000DDF808C026BF921E52080022022B26BF2A
:101700009B1E5B0800236F4C00F00F05A4FB0C4CE4
:101710004FEA1C14DFF8A8C1C0F30310DCF800C0C6
:101720000CEBC51C0CEB4010D0F854C161F31B6CE2
:1017300062F3134C63F30B2C64F3070CC0F854C131
:1017400030BC704770B45E4D00F00F04C0F303105E
:101750002D68DDF80CC005EBC41404EB4010D0F884
:1017600054010029C0F30366C0F30345C0F303240A
:10177000C0B218BF0E6012B16900891C116013B1AC
:101780006100891C1960BCF1000F04BF70BC704778
:1017900000EB80008000CCF8000070BC704770B493
:1017A00091B000224FF480456C10EC4601E0082A0D
:1017B00005D2531C03EB8303B5FBF3F304E0D31F03
:1017C00003EB8303B4FBF3F35B1A48BF5B424CF8B3
:1017D0002230521C102AEAD30026009B01215CF81B
:1017E00021209A42BCBF13460E46491C1029F6D34D
:1017F000334900F00F02C0F30310096801EBC21176
:1018000001EB4011D1F85801D1F8582100F00F0038
:1018100066F30302C1F85821082807D2401C00EBE8
:101820008000B5FBF0F011B070BC7047C01F00EB3A
:101830008000B4FBF0F011B070BC7047204A00F09B
:101840000F01C0F30310126802EBC11101EB40104D
:10185000D0F8580100F00F00082834BF401CC01F0A
:1018600000EB800034BF4FF480414FF40051B1FBD6
:10187000F0F0704710F00F0F08BF7047104A00F0EB
:101880000F000029126802EBC010D0F824110CBF21
:1018900021F4803141F48031C0F8241170470021D7
:1018A00010F00F0F12D0064A00F00F00126802EB82
:1018B000C010D0F8240110F4803F05E0F82B01009F
:1018C000E02B0100CDCCCCCC18BF012108467047DD
:1018D000444902460868D0F8AC0012F0010F0A68CB
:1018E000C0F3C000D2F8AC2005D0096842F008026D
:1018F000C1F8AC207047096822F00802C1F8AC209A
:101900007047384A136858671068816770473549CF
:1019100000280868D0F8AC0005D0096840F0020043
:10192000C1F8AC007047096820F00200C1F8AC00B3
:1019300070472C4900280868D0F8AC0005D0096829
:1019400040F00100C1F8AC007047096820F00100C8
:10195000C1F8AC00704723480068D0F8DC0070473D
:1019600020490968C1F8E000704770B41D4E00209E
:101970003168D1F8401111F0010F04BF70BC7047FD
:1019800011F0040F336801F00805D3F81C31D6F8C4
:1019900000C0C3F30803DCF800C11FFA8CF4D6F8CA
:1019A00000C0DCF844C1CCF3080C18BFC1F30740F9
:1019B0003268D269C1F3052112F0080204D03268FE
:1019C000D2F84421C2F30232002D18BF491C0CFA90
:1019D00002F201FB0200604370BCC3EB031100EB99
:1019E00041007047E02B0100FEF765BE10B5FEF721
:1019F00062FE012818BF10BD0020FEF73DFE212128
:101A00000020FEF75FFE2121BDE810400120FEF717
:101A100059BE10B5FEF728FEFEF74DFE01280AD18B
:101A20000020FEF729FE21210020FEF74BFE212198
:101A30000120FEF747FE0121052001F0BAFD01213A
:101A4000052001F0B6FDFF490020487110BD10B51A
:101A50004FF4066001F003FEBDE810404FF406604D
:101A600001F0F0BDF74A0146507B002818BF012065
:101A7000002918BF012151737047F24A516A506220
:101A800008467047EF4900200873C8708870704797
:101A9000EC4900200873C870887070472DE9F34F37
:101AA00000F00F056800861EA1B0002445EA04106E
:101AB000FEF743FE00283BD02298002100EBC4171C
:101AC000EC46002007EB81120CEB811352F82080CA
:101AD00043F82080401C1028F8D3491C0229F0D379
:101AE000D94900224FF0020809683019434601EB3A
:101AF000C01723FA02F101F0010107EB82100CEB91
:101B00008111A0F55F50B1E8004E00F50040521C75
:101B1000A0E8004EB1E8004EA0E8004EB1E8004E4B
:101B2000A0E8004E91E8020E80E8020E4245E0D3A4
:101B3000641C022CBAD323B0BDE8F08F70B5064602
:101B4000FEF7DFFDC04D0446EEB12868A201314624
:101B500000F580400EF0EEFB2868002100EB8410B9
:101B600000F58040016041608160C16001614161B8
:101B70008161C161016241628162C162016341634D
:101B80008163C16370BD81012868BDE8704000F5C4
:101B900080400EF0D4BB10B5AA4CE061FFF775F899
:101BA000FFF760F8A1696FF30F01A161A269C1B2EB
:101BB00042EA0121A161022818BF10BDA06940F0CE
:101BC0000100A06110BDA14801688968A04A1143C5
:101BD00002689160016809689E4A006811430160CB
:101BE00000F001BF70B5994A05460C46106883683D
:101BF0009748116818438860106800689549084341
:101C00001168086000F0EFFE002C4FD00020FEF7B6
:101C100033FD206820B1FEF79FFD0020FEF72CFD6C
:101C20002846FFF7B8FF0020FEF787FDC8B16068BF
:101C3000FFF784FF844DE16839B128684FF4807262
:101C400000F5C0400EF076FB02E0834800F089FD0D
:101C5000616959B128684FF4807200F500400EF0B8
:101C600069FB0120FEF769FD60B907E028684FF4C1
:101C7000807100F500400EF062FBF2E71120FEF7E4
:101C80005CFD28B1A16800291CBF0120FFF706FFF9
:101C90000220FEF752FD18B91220FEF74EFD28B1C2
:101CA000216900291CBF0220FFF7F8FE00206549CA
:101CB0000873C87088704862487B002048734FF4EE
:101CC000066001F0CCFCBDE870404FF4066001F006
:101CD000B9BC10B50020FEF7CFFC00F069FE5948F2
:101CE0000079002808BF10BD5848016809680268DB
:101CF00021F0030141F00D7141F080511160016844
:101D00008968006821F0020141F00D7141F08051B5
:101D1000816010BD4FF4066001F098BC10B54FF41F
:101D2000066001F093FCFEF7C6FC01280AD10020F2
:101D3000FEF7A2FC21210020FEF7C4FC2121012096
:101D4000FEF7C0FC45480168D1F8B012006821F4E4
:101D50008031C0F8B0120020FEF78EFC00F028FEA3
:101D600038480079002808BF10BD38480168096864
:101D7000026821F0030141F00D7141F080511160C2
:101D800001688968006821F0020141F00D7141F09D
:101D90008051816010BD10B501F05DFC10F0600055
:101DA00018BF012010BD2748C06970472549002889
:101DB00018BF01200870704722480078002818BF1B
:101DC000012070471F488069704772B61D498A69B3
:101DD00022EA0000886162B670471A4840780028FD
:101DE00018BF0120704770B5FEF765FC002818BFCA
:101DF00070BD0024134D2C73EC70AC702121204673
:101E0000FEF760FC21210120FEF75CFC6C70BDE850
:101E100070400120FEF730BC70B50446FEF74BFC65
:101E2000002818BF70BD0021064D2973E970A97004
:101E300021210020FEF746FC21210120FEF742FC73
:101E4000022C0DE020000110F82B0100E82B01000E
:101E500002003412030034125C030110E02B010075
:101E60003CBF0120FEF73CFC012068702C62BDE8FD
:101E70007040FEF701BC10B5FEF71DFC002818BF2E
:101E800010BD0020FB4C2073E070A0702121FEF7F4
:101E900019FC21210120FEF715FC0120FEF720FC92
:101EA000012060702062BDE81040FEF7E5BB002015
:101EB000FEF7E2BBEF490020C87088700120FEF7F2
:101EC000DBBBEC4988627047EA48806A70470020B3
:101ED00000F070BC012000F06DBC10B5FFF73BFDB9
:101EE0000446FFF73DFDE448044208BF10BDE14849
:101EF000816941F0040181610E2101EAD43104F0CD
:101F000001020A43816962F31F418161DB48016874
:101F100041F02001016010BD002818BF0120D54903
:101F200008717047D6487047D6487047D148C06A94
:101F30007047D048006B7047CE48406B70472DE922
:101F4000F00FCF4E4FF0000C88B006F14007E1468D
:101F50004FF0FF3806F80C8007F80C900CF1010CDC
:101F6000BCF1200FF6DB4FF0000C002807D912F867
:101F70000C4006F80C400CF1010C6045F7D800222B
:101F800094464FF0010A00280BD9B456002C05DB0B
:101F9000202C3CBF0AFA04F444EA0C0C521C824286
:101FA000F3D3002214466D460AFA02FB1BEA0C0F1B
:101FB0001ABFAC54641C05F80280521C202AF3DBC3
:101FC0000022002810D916F902C0BCF1000F08DB6E
:101FD000BCF1200F3ABF15F80CC007F802C007F893
:101FE0000280521C8242EED3A24C00220028C4F888
:101FF0002C9008D917F902C0944501D0E76202E09D
:10200000521C8242F6D3A04F0020A7F1600CA7F12A
:1020100020060CF8008006F8009007F80090401C9D
:102020002028F6DB0020002905D91A5C0CF80020D6
:10203000401C8142F9D80020024600290BD91CF926
:102040000230002B04DB202B3CBF0AFA03F31843B9
:10205000521C8A42F3D3002213460AFA02FB1BEAFF
:10206000000F1ABFAB545B1C05F80280521C202ADB
:10207000F3DB002200290AD91CF90230002B03DB14
:10208000202B3CBFEB5CBB54521C8A42F4D3002291
:10209000C4F83490002907D9BB56934201D0676336
:1020A00002E0521C8A42F7D311F0010F18BF1F2221
:1020B00009D00AFA02F3034203D10AFA02F21043EA
:1020C00001E0521EF5D5002213460AFA02F7074234
:1020D0001ABFAB545B1C05F80280521C202AF4DBAB
:1020E000002000290AD91CF90020002A03DB202A3D
:1020F0003CBFAA5C3254401C8842F4D30020C4F890
:10210000309000299EBF08B0BDE8F00F70473256EE
:10211000824204D0266308B0BDE8F00F7047401C2F
:102120008842F4D308B0BDE8F00F7047574900EB80
:10213000401001EB8010704700EBC000544900EBE9
:10214000400001EB80007047DFF828C1012B8CF8BC
:1021500006008CF8071003D9401C20F0010011463E
:102160008CF808008CF8091000FB01F24FF6FF71A3
:1021700001EA4202ACF8122001EA4000ACF8140077
:1021800070473C48407A70473A48007A7047394A6D
:102190009072D17270473748C07A70473548807A5C
:1021A00070473C4A1070517070473A49085C70475C
:1021B0002DE9F047DFF8BCA004469AF80D0000288E
:1021C00004BF9AF802000EF0BFF89AF80C0000283D
:1021D00008BFBDE8F0874FF00009DAF81C00C846D8
:1021E0004F464E464D4610F0020F1CBFDFF89C9044
:1021F00010F0040F06D0BAF81210244A21F00101A1
:1022000001EB020810F0010F04D010F0100F0CBF0A
:102210001F4F1F4E10F0200F18BF1F4DDAF8280077
:102220002060FEF722FD10F0010F06D0FFF768F8DE
:10223000022828BF9AF8030000D20020C4E901094F
:10224000C4E90565C4E903870120BDE8F0870949B1
:1022500000200873704710B50446FEF752FA820159
:102260000E48006800F580412046BDE810400EF0A1
:1022700061B8000020000110010007005C0001109F
:102280005C0301107C030110DC030110FC0301104E
:102290003C0C01102E000110140D0110F82B010050
:1022A0002DE9F041FEF72DFA04460020FFF738F93A
:1022B0000022002C24D9F94F012541F6F0763B6825
:1022C000002103EB821C05FA01F3034212D04B08F4
:1022D0000CEB830303F580434FEAC1781B684FEA98
:1022E000D86823FA08F3C3F30C03B34202D90020E1
:1022F000BDE8F081491C2029E5D3521CA242DED35F
:102300000120BDE8F0812DE9F05F00F00F06002408
:10231000E24F8846750046EA0410FEF70EFA60B3F5
:1023200002218A46002308EBC41B0020002908D99B
:102330002AFA00F202F001029A421CBF401C8842B5
:10234000F6D3884216D2A5F10209D7F800E0A144DD
:102350000EEBC9190BEB831C002209EB801909EB6A
:10236000820000F58040D0F840084CF82200521C52
:10237000102AF4D35B1C022BD7D3641C022CCAD3C3
:10238000BDE8F09F2DE9F05F00F00F06700000251A
:10239000A0F1020B012741F6F07846EA05194846FC
:1023A000FEF7CBF9002834D04846FFF7C6F807FA05
:1023B00000F4022C88BF02244846FFF7B1F800223F
:1023C000002C26D9B54B0BEB05011B6803EBC11A9A
:1023D00000210AEB821907FA01F3034213D04B08DC
:1023E00009EB830303F580434FEAC17CD3F84038FF
:1023F0004FEADC6C23FA0CF3C3F30C03434502D918
:102400000020BDE8F09F491C2029E4D3521CA242C1
:10241000DED36D1C022DC0D30120BDE8F09F9F4B81
:102420004FF6FF7C1B6803EB8111430801EB83012E
:1024300001F58041C007C00E0CFA00FC0B6802FADF
:1024400000F023EA0C03184308607047934A1268AF
:1024500002EB8111420801EB820101F58041C007C6
:102460000968C00E21FA00F080B270472DE9FF4FD5
:102470008A4883B01D460068109C00F580401746CE
:102480000E460190FEF717F95FEA00081CBF002016
:10249000FEF7F2F80020FFF743F88246701900902B
:1024A000B04284BF4FF0010B4FF6FF7E26D9019852
:1024B0004FF0000C00EB8611039B17E00BFA03F0C2
:1024C00010EA0A0F11D05808DD0751F82020ED0E50
:1024D0000EFA05F922EA090234F8029B0CF1010C0C
:1024E00009FA05F52A4341F820205B1CBC4538BF9A
:1024F000202BE3D30098761C8642D8D3B8F1000F86
:1025000004BF07B0BDE8F08F00206549C87088702F
:1025100007B00120BDE8F04FFEF7AEB82DE9F04757
:1025200007465E489A46144600680E46089D00F528
:102530008049FEF7C0F85FEA00081CBF0020FEF7E4
:102540009BF806EB0A03B34284BF564907EB040C21
:102550001AD93C4609EB86100FE00A57202A0BD205
:1025600002EBD27A4FEA6A0AD20750F82AA0D20EBA
:102570002AFA02F225F8022B641C644538BF202C8D
:10258000EBD3761C9E42E4D3B8F1000F08BFBDE840
:10259000F08700204249C8708870BDE8F0470120EC
:1025A000FEF76AB82DE9F05F3D4E3C4A4FF0000857
:1025B0004FF6FF7700280C4645D0116801F5804999
:1025C00000F00F01C0F3031001290EBF0021022902
:1025D000BDE8F09F022828BFBDE8F09F01EB000A8C
:1025E000FEF769F805001CBF0020FEF745F8002043
:1025F00009EBCA19002209EB801153084FEAC27C8B
:102600004FEADC6C01EB830307FA0CFBD3F840A81C
:1026100004FA0CFC2AEA0B0A4AEA0C0C521CC3F816
:1026200040C8202AE9D3401C0228E3D3002D08BF6C
:10263000BDE8F09F86F8038086F80280BDE8F05F71
:102640000120FEF719B8106800F58049FEF733F84D
:1026500005001CBF0020FEF70FF84FF0000C002211
:1026600009EB8C115308D007C00E07FA00FB51F894
:1026700023A004FA00F02AEA0B0A4AEA0000521CDE
:1026800041F82300202AEDD30CF1010CBCF1210FFD
:10269000E5D3002DCED1BDE8F09F0000F82B01005E
:1026A000200001107C03011010B5FEF7E3FE624923
:1026B000088210BD604AC1B200F4F853128A9142F8
:1026C00088BF11464FF0640C01FB0CF1B1FBF2F135
:1026D0001A0A02FB0C1189B210F4005F12BF08B293
:1026E000484200B270470028B8BF404280B2B4BF31
:1026F00000214FF4005100F4F85211434E4AC0B289
:10270000128A504341EA102070474C4800F029B823
:1027100010B54A4800F025F849484FF42461006894
:10272000BDE8104000F580400DF009BE424810B5EC
:10273000808B00F48170FFF72EFA414C4FF48071CA
:10274000206800F5C0400DF0FAFD20684FF40461E8
:1027500000F580400DF0F3FDBDE810400020FEF7CD
:10276000D6BD70B5364D04464FF48071286800F52B
:10277000C0400DF0E4FD002101206256002A15DB67
:10278000D31702EB137C4FEA2C132E682CF00F0C9E
:1027900006EBC31303EB810303F5C043A2EB0C026A
:1027A00052001E6800FA02F232431A60491C2029C6
:1027B000E3D370BD70B5204C0546A06A401CA062F2
:1027C000607850B1206A10B1206A401E2062206AF1
:1027D000002804BF0020FDF74FFF20212846FDF709
:1027E00071FF616A00291CBF28468847FEF73AFA44
:1027F00002281AD113480168D1F8B81211F0010F5C
:1028000013D00168D1F8B812026841F00101C2F892
:10281000B8120168D1F8B812006821F00101C0F8BF
:10282000B812A06940F00200A0610748016841F0B9
:102830002001016070BD0000200001105C03011048
:10284000F82B0100E02B01005C000110F0B4002423
:102850007D4E012382B0002808BF337019D00128B3
:10286000347018BF747014D0784D286800687849A7
:102870000143286801603178764A61B110684BF6EF
:10288000083CC0F80CC01068DFF8CCC1C0F808C024
:102890000CE07370E8E7D2F800C07048CCF80C0088
:1028A000D2F800C04FF0BB70CCF808006C4800684C
:1028B00030F0FF0C08D1D2F800C0DCF80CC060F397
:1028C000030C1068C0F80CC040F2E24CC9B11068AB
:1028D000806840F01807106887600120009004E0CD
:1028E0000198471E0197FBD20098471E009728BF0A
:1028F000CDF804C0F4D210688068176840F48050A6
:10290000B8600120009004E00198471E0197FBD2B7
:102910000098471E009728BFCDF804C0F4D2707805
:1029200028B11068C068166840F03000F060106888
:10293000D0F8B000166840F00100C6F8B0000120E1
:10294000009004E00198461E0196FBD20098461EB6
:10295000009628BFCDF804C0F4D21068C367D2F83F
:1029600000C04FF4E060CCF810001068C0F8884058
:1029700000291CBF1068C0F894301068C068116846
:1029800020F03000C86010688068116820F01800DE
:1029900020F48050886028680068296820F00400CE
:1029A00040F00D7040F08050086002B0F0BC7047FD
:1029B00028480168C968026821F03001D1600168C7
:1029C0008968006821F0180121F4805181601F4856
:1029D00001680968006821F0040141F00D7141F0BF
:1029E000805101607047194801680A6818490068F9
:1029F00011430160144917480A7832B1026892689D
:102A000041F218031A4303689A60497829B10168B2
:102A1000C968026841F03001D1600168D1F8B01096
:102A2000006841F00101C0F8B01070470D49C0B214
:102A300041EA0020074909680864704705490A48C7
:102A4000096808647047000058000110E82B010075
:102A500004003412E42B01002000BB0005F4010047
:102A6000D0FE030013005FA000005FA05948584942
:102A7000026891610268891CD1610268491E516334
:102A800002681268036822F0030242F00D7242F0FD
:102A900080521A6002685269036822F0010242F013
:102AA0000D7242F080525A61026812691143026845
:102AB000116102684849916000684849C16048490D
:102AC00000200860704770B501F0FBFA444D2C6897
:102AD0002CB10020286001F0F9FA204670BD30BF0B
:102AE00000F064FE0028F2D000F073FE6860EEE7AC
:102AF0002DE9F04101F0E5FA354E364CDFF8E08083
:102B0000771CD8F800503DB10020C8F8000001F053
:102B1000DDFA2846BDE8F08172B620684663206879
:102B2000876120BF206886612068476362B6BFF373
:102B30006F8FBFF34F8F00F039FE0028E1D000F017
:102B400048FEC8F80400DCE722480168096802680A
:102B500021F0030141F00D7141F0805111600268D4
:102B600020499160016809691F4A006811430161A9
:102B700030BF704772B61649164802685163026842
:102B8000C91CD1610068891E816162B67047114815
:102B900001680968154A00681143016070470D48D3
:102BA00001680968006821F0030141F00D7141F0EE
:102BB00080510160704772B605490648026891610C
:102BC0000268891CD1610068491E416362B6704782
:102BD00000003412E82B01003C00341228003412AB
:102BE0005C0001100800341201003412030034129A
:102BF0007047002818BF0120F549096848607047F0
:102C00000022B2EBD10F26D20368B3F1FF3F04BF1D
:102C10004368B3F1FF3F17D18368B3F1FF3F04BFAF
:102C2000C368B3F1FF3F0FD10369B3F1FF3F04BFA6
:102C30004369B3F1FF3F07D18369B3F1FF3F04BF9D
:102C4000C369B3F1FF3F01D0002070472030521C10
:102C5000B2EBD10FD8D30120704710B40023B3EBEF
:102C6000D20F30D2D0F800C00C68A44522D1D0F8E1
:102C700004C04C68A4451DD1D0F808C08C68A44598
:102C800018D1D0F80CC0CC68A44513D1D0F810C02E
:102C90000C69A4450ED1D0F814C04C69A44509D1E3
:102CA000D0F818C08C69A44504D1D0F81CC0CC69F8
:102CB000A44502D010BC00207047203020315B1C9E
:102CC000B3EBD20FCED310BC012070472DE9F041F9
:102CD000054601F000FA0020BD4A21264FF4825734
:102CE000844611680E60C5F800C011680968136851
:102CF00041F0040119601168096811F0040FFAD15C
:102D000011680F6040232C460021D4F80080B8F1F0
:102D1000FF3F04BFD4F80480B8F1FF3F1DD1D4F8C1
:102D20000880B8F1FF3F04BFD4F80C80B8F1FF3F32
:102D300013D1D4F81080B8F1FF3F04BFD4F8148049
:102D4000B8F1FF3F09D1D4F81880B8F1FF3F04BFB4
:102D5000D4F81C80B8F1FF3F09D01168C1F800C059
:102D6000401CC0B20828BCD30220BDE8F081491C39
:102D70002034B1EBD30FC8D31068C0F800C00120D5
:102D8000BDE8F0812DE9F041054601F0A4F90020ED
:102D90008F4B0926844619680E60C5F800C0196873
:102DA00009681A6841F0040111601968096811F096
:102DB000040FFAD12C464FF4806200212768B7F146
:102DC000FF3F04BF6768B7F1FF3F17D1A768B7F1AE
:102DD000FF3F04BFE768B7F1FF3F0FD12769B7F1A5
:102DE000FF3F04BF6769B7F1FF3F07D1A769B7F19C
:102DF000FF3F04BFE769B7F1FF3F09D01968C1F889
:102E000000C0401CC0B20328C5D30220BDE8F08139
:102E1000491C2034B1EBD20FD0D31868C0F800C0E1
:102E20000120BDE8F0812DE9F05F0F4680460426C1
:102E30004FF0020A4FF0000BDFF8949101F04BF9CC
:102E4000D9F8001044463846C1F800A00F21B0E878
:102E50002C10A4E82C10491EF9D2D9F80000006803
:102E6000D9F8001040F004000860D9F800000068AC
:102E700010F0040F07D000BF00BFD9F800000068B1
:102E800010F0040FF7D1D9F80000C0F800B04546A3
:102E900038460F21D5E90023D5E902C4D0F800E077
:102EA000964504BF42689A4205D18268624504BFD4
:102EB000C268A24208D0761E03D34046FFF706FF41
:102EC000BCE70220BDE8F09F10301035491EE1D26A
:102ED0000120BDE8F09F70B50D46044601F0FBF8F7
:102EE0004FF48072214628460DF024FA012070BD6F
:102EF0002DE9F041C0B014460E46054610F0FF0F14
:102F000023D025F0FF086F4601F0E5F84FF48072FA
:102F1000414638460DF00EFAE8B2C0F58077A74278
:102F200088BF274668443A4631460DF012FA4046BB
:102F3000FFF7CCFE022843D069464046FFF773FFF7
:102F4000022841D03D443E44E41BB4F5807F19D3B0
:102F50004FF48072314668460DF0FBF92846FFF7C2
:102F6000B5FE02282CD069462846FFF75CFF0228F0
:102F70002AD0A4F5807405F5807506F58076B4F541
:102F8000807FE5D2C4B16F4601F0A5F84FF480729E
:102F9000294638460DF0CEF92246314668460DF0F6
:102FA000D8F92846FFF792FE022809D0694628463C
:102FB000FFF739FF022807D040B00120BDE8F081BB
:102FC00040B00A20BDE8F08140B00B20BDE8F081A0
:102FD000CC2B010034490A6810600968086100F0D0
:102FE00016B831490A6810600968486100F00FB8E6
:102FF0002D490968486770472B49096888677047F9
:103000002948012102681166006801657047274A56
:103010001168096B10F0010F18BF21F4404110F046
:10302000020F1CBF21F4405141F4805110F0040FF5
:1030300018BF21F4406110F0080F18BF41F440712F
:1030400010F0100F18BF41F0C00110F0200F18BF92
:1030500041F0300110F0400F18BF41F00C0110F0AA
:10306000800F18BF41F0030141F4BE01136841F025
:10307000204119631168D1F8901010F4807F1CBFB3
:1030800021F0030141F0020110F4007F1CBF21F088
:103090000C0040F0080141F4BE00116840F02040EF
:1030A000C1F8900070470000D42B0100DC2B010018
:1030B0007047F74801688A68F64903680A439A60CE
:1030C0000268D26811430268D16001684969F24A16
:1030D0000068114341617047ED4801684969026821
:1030E00021F0010141F00D7141F080515161016801
:1030F000C968026821F0400141F00D7141F0805132
:10310000D16001688968006821F0400141F00D71CB
:1031100041F080518160704710B5DD4C20688168B6
:10312000DC482268014391602168C968084321682E
:10313000C86020684069D849084321684861D74879
:1031400043F63F710268D160026800219163026812
:1031500091640068C0F8B01003210A2000F029FA39
:103160000A2000F04AFA20684069216820F0010036
:1031700040F00D7040F0805048612068C0682168C0
:1031800020F0400040F00D7040F08050C860206892
:103190008068216820F0400040F00D7040F08050C1
:1031A000886010BDBD4A13681860136859604843B1
:1031B000116888607047B94A1368186013685960CD
:1031C000484310F0010F18BF401C11688860704719
:1031D000B2490968C1F8B0007047B04918B1096830
:1031E0000120886470470968002088647047AB49F3
:1031F0000A6890630868C068096840F00200C86007
:103200007047DFF898C210B4DCF800402062DCF8A8
:1032100000004162DCF800008262DCF80000C3625A
:10322000DCF8001001200863DCF80000406B10F0AF
:10323000010F06D020BFDCF80000406B10F0010F3A
:10324000F8D110F0020018BF4FF0FF3010BC7047EB
:1032500092480168C968006821F00201C1607047A6
:103260008E480168C968006841F00101C16070477B
:103270008A4BD3F800C0CCF8200018684162186867
:1032800082621968012008641868406C10F0010F10
:1032900005D020BF1868406C10F0010FF9D110F074
:1032A000060018BF4FF0FF3070477C480168C968BE
:1032B000006821F00101C160704778480168C96861
:1032C000006841F00401C1607047027C017B02F09C
:1032D0003F0241EA0241714A136899651368016827
:1032E000596213684168996213688168D9621368EA
:1032F000012119651168496D11F0010F05D020BF3A
:103300001168496D11F0010FF9D11368DB6D8382EB
:103310001368DB6D1B0CC38213681B6E0383136879
:103320001B6E1B0C438313685B6E83831268526EA3
:10333000C2F30E42C28311F0020018BF4FF0FF30FB
:10334000704756480168C968006821F00401C160EF
:10335000704752480168C968006841F00801C160BF
:103360007047DFF838C110B4DCF80040A267DCF821
:1033700000201062DCF800004362DCF8000081628B
:10338000DCF8001001200867DCF80000406F10F046
:10339000010F06D020BFDCF80000406F10F0010FD5
:1033A000F8D110F0060018BF4FF0FF3010BC704786
:1033B0003A480168C968006821F00801C160704797
:1033C00001684FEA314235490B68C3F89C200A680E
:1033D0004068C2F8A0000868C068096840F0200092
:1033E000C860704701684FEA31422C490B68C3F846
:1033F0009C200A688088C2F8A0000868C068096834
:1034000040F02000C8607047244BD3F800C0CCF8CF
:103410002000186842621868816219680120C1F8AA
:1034200094001868D0F8980010F0010F06D020BF63
:103430001868D0F8980010F0010FF8D110F00600CD
:1034400018BF4FF0FF307047144A136818621068B5
:10345000416211680120C1F890001068D0F898000E
:1034600010F0010F06D020BF1068D0F8980010F0BF
:10347000010FF8D110F0060018BF4FF0FF30704771
:1034800006480168C968006821F02001C1607047E2
:10349000E82B01004000341201003412EC2B010033
:1034A0001B480168C968006841F01001C16070479D
:1034B000A3F1050C164B10B41C68C4F888C0D3F8EF
:1034C00000C0CCF820001868426218688162196850
:1034D0000120C1F880001868D0F8840010F0010FB6
:1034E00006D020BF1868D0F8840010F0010FF8D182
:1034F00010F0060018BF4FF0FF3010BC70470448B2
:103500000168C968006821F01001C16070470000BF
:10351000EC2B0100244810B50268022111650268F5
:1035200001211166026810215167026841F206010B
:10353000516602680021916602680421C2F8881071
:1035400002689021C2F884100168D1F884100268E2
:1035500041F00101C2F8841002684FF481711166D4
:1035600000680166032000F048F80021032000F005
:1035700020F8002010BD10B5032000F049F80A48DB
:103580004FF48071026811660268002111660268BA
:1035900010219167006802214165002010BD034998
:1035A0000020087070470000D82B01006400011053
:1035B000704700F00303DA004FF0FF0C0CFA02F240
:1035C0004FF0050C0CEBC303994000F00C030028EE
:1035D00008DA30480068184443691140934319439E
:1035E000416170472C4800681844D0F800331140FE
:1035F00093431943C0F80013704700F01F010122E4
:1036000002FA01F1244A4009126842F8201070477A
:1036100000F01F01012202FA01F11F4A400912685D
:1036200002EB8000C0F88010704700F01F010122FB
:1036300002FA01F1184A4009126802EB8000C0F852
:103640008011704714490968086070471249096879
:10365000C1F88000704710480068006870470E4944
:103660000968C1F8800170470A480068806870479F
:1036700008490A6892680968886010467047054AD8
:103680001268926800F1100352F8230042F82310E8
:1036900070470000C82B0100C42B010002210C2040
:1036A000FFF787BFCB4801688A68CB4903680A43A4
:1036B0009A600268D26800681143C1607047C548CB
:1036C00001688968026821F4805141F00D7141F070
:1036D000805191600168C968006821F4805141F00F
:1036E0000D7141F08051C1607047BC4881B00168E4
:1036F000096F11F4007FFAD10168896E11F0010F92
:1037000009D00168D1F8841000910168D1F88410C3
:10371000009A9142F9D00168096F11F4007F03D13A
:1037200002684CF271011166006842F24131816613
:1037300001B07047A9494FF40D520B689A660A68A8
:10374000126F0B68DA66012898BF012005D9401E68
:10375000B0F5803F28BF4FF6FF7080B24FF05C524B
:1037600042EA00200A68506609684FF01140C1F82B
:103770008000BAE7994881B00168096F11F4007FB1
:10378000FAD10168896E11F0010F09D00168D1F8F2
:10379000841000910168D1F88410009A9142F9D008
:1037A00000684FF40D51816601B070478948006888
:1037B000806810F4805008BF704788480068806EA9
:1037C00000F00100704785480068406EC0F30F208C
:1037D000704782480068D0F88400704710B50C200C
:1037E000FFF723FF0C20FFF708FF7C490220096840
:1037F000486710BD794910B50968032088670C2017
:10380000FFF706FFBDE810400C20FFF70EBF744A1B
:103810001168106008467047704810B50168096F5C
:103820000068C1666E480068002818BF80476D4870
:10383000016841F48051016010BD694840687047DB
:10384000644810B501688A68634903680A439A604E
:103850000268D26800681143C160604C032021688F
:1038600088670C20FFF7D4FE0C20FFF7DEFE00F087
:10387000A9F95D4B04201968C1F8880019684FF652
:10388000FF70C1F88C0072B621684FF40D50886645
:103890002068006F2168C86621685448486621681E
:1038A0004FF01140C1F88000FFF71FFF19684FF477
:1038B0000070086662B610BDF8B572B64748016878
:1038C000096F11F4007FFAD10168896E11F0010FC0
:1038D00009D00168D1F8841000910168D1F88410F2
:1038E000009A9142F9D002684FF40D5191663E4919
:1038F0004FF400330A68136662B60968D1F80412FF
:10390000344D00294AD0364C4FF6FF73591AA16046
:103910002A689269D5F800C002F00F02DCF81CC0DA
:103920000CF00F0C6244121D01FA02F2A2F5EA41FA
:10393000DFF8BCC03139614530D20068D0F884006E
:10394000191AE160B1F5803F28D22A4B4FF0000CE4
:10395000A1FB03070CFB037301FB0C3163460CF066
:10396000FDFC401C40082061B0F57A7F38BF4FF461
:103970007A70214B9968002908BF98605A681A60CC
:103980009968C3E901108A421FD9824205D9814250
:1039900001D9616002E0606000E0626000F023F93C
:1039A00028688068296820F4805040F00D7040F04D
:1039B000805088602868C068296820F4805040F0F2
:1039C0000D7040F08050C860F8BD8242E5D8814259
:1039D000E1D8DEE7E82B010000103412F42B0100DF
:1039E000680001105C000110F02B010000FEFF37A1
:1039F0002F6E160000879303580D011013480168BD
:103A00008968134A00681143816012480168496956
:103A1000026841F40071516101680969026841F06E
:103A20000401116101680969006841F01001016138
:103A300070470849096888607047BFF34F8F054990
:103A400005480968C860BFF34F8FFEE7E82B010007
:103A500004003412C82B01000400FA051E48016856
:103A600089681E4A0068114381601D4801684969E0
:103A7000026841F0010151610168096A036821F09F
:103A80000F0218490A431A62174B8A1E1B68C3F8B3
:103A9000C42000680165704711480068006900F0A3
:103AA000700070470E48114902681163026810499E
:103AB000516302680F49C2F890100068491FC0F8AE
:103AC0009410704706480168496C00291ABF0068C5
:103AD0004068094870470000E82B010004003412D8
:103AE000DC2B010003005FA0E42B0100C0845FA079
:103AF00095995FA00A005FA061B66505022824BF02
:103B000000207047FE4B53F8202043F82010104649
:103B1000704770B5FB4C2068006FF94D10F0010F35
:103B200006D021680120C8662868002818BF804791
:103B30002068006F10F0020F08BF70BD02202168DE
:103B4000C8666868002808BF70BDBDE870400047BF
:103B5000ED4810B501688A68EC4903680A439A6029
:103B60000268D26811430268D160E64902220B68FC
:103B70001A65D1F800C00123CCF86030D1F800C03C
:103B80000323CCF86C3009684A65016889680268CB
:103B900021F0800141F00D7141F080519160016888
:103BA000C968006821F0800141F00D7141F0805139
:103BB000C1600920FFF721FD0221BDE81040092066
:103BC000FFF7F7BCD04801688A68D04903680A4308
:103BD0009A600268D26800681143C160C949022036
:103BE000096808657047C749022009684865C648E2
:103BF00001688968026821F0800141F00D7141F08F
:103C0000805191600168C968006821F0800141F02D
:103C10000D7141F08051C1607047BB4800688068F9
:103C2000C0F3C0107047B7480168096F11F4007FF6
:103C300004D000684FF440710166704700684FF48B
:103C400080710166704710B5AE4C2068C06F10F0EF
:103C5000020F4FF0010018BF03202168486700F0F1
:103C6000C5F9A9490A689269096802F00F02D040B3
:103C7000C969226801F00F01C8400521B0FBF1F0CD
:103C80004FF405710009C2F880100CF06CFBA04ADB
:103C9000A04B0CF06DFB0CF070FB2168C1F88400A8
:103CA0002068006F10F4007F04D021684FF440704A
:103CB000086610BD21684FF48070086610BD9148F9
:103CC0000168096F11F4807F04D000684FF44071DF
:103CD0000166704700684FF4007101667047894BB8
:103CE00030B41A68D26F12F0010F1DBF4FF0030CF1
:103CF0001A68C2F874C0022204BFD3F800C0CCF81E
:103D000074204FF0020C00EB4005C5EBC0104FF4DF
:103D10009674C1EBC0004C4300EB80007E4904EB7D
:103D20004010A1FB001078490022C0080C68A4696B
:103D3000096804F00F04C96901F00F012144C8406B
:103D40000521B0FBF1F0B0F5803F05D3511C4008D0
:103D5000CAB2B0F5803FF9D242EA0C211A6841F0AC
:103D60001001C2F888101968C1F88C001868006F3B
:103D700010F4807F05D019684FF44070086630BC9D
:103D8000704719684FF40070086630BC70475D4892
:103D90000168096F11F4003F04D000684FF440310E
:103DA0000166704700684FF48031016670475548DE
:103DB0000168096F11F4803F04D000684FF440316E
:103DC0000166704700684FF40031016670474D4846
:103DD0000068006FC0F3002070474A480068006F19
:103DE000C0F340207047484909688968C1F3C01191
:103DF000002904BF002070474249002808680CBF12
:103E0000D0F80002D0F8040270473F4B1A6892685D
:103E1000C2F3C012002A04BF00207047394A0028AC
:103E200010680CBFD0F88000D0F88800C0F30A20DA
:103E300012680CBFD2F88020D2F8882002F00F025E
:103E4000D3F800C0DCF818C01B680CF00F0CDB695D
:103E500003F00F0363441A449140012202EB400037
:103E600048432E49A1FB0010000970472C4901204E
:103E70000870704770B4244BC1EB011149001A68F7
:103E80009269D3F800C002F00F02DCF81CC00CF0FD
:103E90000F0C6244121DD14008BF012104D0B1F5BE
:103EA000803F28BF4FF6FF711A689268C2F3C012B4
:103EB000002A1CBF70BC70471A68D2F808C0134AA9
:103EC0001C684CEA020CC4F808C0D3F800C0DCF847
:103ED0000CC04CEA0202D3F800C0CCF80C20094A0E
:103EE0000224D2F800C0CCF8504015684FF4003CD2
:103EF000C5F860C016680425C6F88850156811E03A
:103F000080000110F02B0100E82B0100800034122A
:103F10007B14AE47E17A843FCDCCCCCC89888888AD
:103F20007C000110C5F88C1011681B4DCD6611681E
:103F30004C671A4902283CBF194E46F82010002150
:103F40001848017016684FF400713166017819B98C
:103F500020BF01780029FBD01068C0F860C010684D
:103F600085671068C56610684465186880681968B8
:103F700020F0800040F00D7040F08050886018689C
:103F8000C068196820F0800040F00D7040F080504B
:103F9000C86070BC70470000020002021D5E000095
:103FA000800001107C000110244900200A68906004
:103FB0000968086022494860704710B51F4C2168A5
:103FC00048602168002088600221401EFFF7F1FA56
:103FD00021680720086010BD1849002009680860A2
:103FE000704717480188491C018070471448806851
:103FF00070472DE9F041124C002705462780A06844
:104000004FF47A71B0FBF1F00C4E401E31684860FD
:10401000306887600221C81EFFF7CBFA316807209D
:1040200008602188A942FCD330680760BDE8F081B0
:10403000044948430249886070470000C02B0100D2
:104040008800011040420F00704770B52C4C0546A7
:104050004FF40D502168886621680320C8662168E6
:104060002848486621684CF2710008662168264895
:10407000C1F88000216842F24630886602210020A3
:10408000FFF797FA0020FFF7B8FA002D08BF70BDC0
:104090002068806E42F2413108432168886670BD15
:1040A000174810B502680121916700684FF40D515F
:1040B00081660020FFF7ACFABDE810400020FFF752
:1040C000B4BA0F4901200968486770470C490120BC
:1040D0000968886770470A494CF2710009680866E8
:1040E0007047074881B04CF271010268116601689F
:1040F000096F0268D1660068006F009001B07047D8
:10410000D02B010007383937009C1C9170B5FF4D4A
:1041100000244FF400612C706C70AC70FC480CF003
:104120000EF94FF40061FB480CF009F9FA48AC6055
:10413000EC70046044608460C46004614461846124
:10414000C461046244628462C4620463446384633D
:10415000C463046444648464C4640465446584651D
:10416000C465046644668466C466046744678467FD
:10417000C4672C71682180300CF0E1F86821E748B1
:104180000CF0DDF8EC6070BDE0490020487070472D
:10419000DE4840787047DD48C078002818BF01200D
:1041A0007047DA480079002818BF01207047D748C7
:1041B0008078002818BF01207047D448407800EB71
:1041C000800101EBC000D64901EBC00070472DE92A
:1041D000F041CE4D0446D2496A78D24F02EB8200BC
:1041E00000EBC200D04E01EBC0033A783078214694
:1041F0001044420018460CF0ACF86A78C74902EB4C
:10420000820000EBC20001EBC0033A78307821460F
:104210001044420018460CF09CF801202871BDE8BB
:10422000F081BA48C0687047B849B948497800EB8E
:10423000C12070472DE9F041B44E07463078002880
:1042400014BFBA48BA48047814BFBA48BA480578C7
:1042500004FB05F8FEF72DFF29462046FEF7A2FFD6
:10426000AC4C7078A4F5006104EBC02201EBC020D7
:104270003B460146FEF7C5FFFEF72EFF70784FEA7A
:10428000480204EBC02039460CF063F80120B070FE
:10429000BDE8F0812DE9F0479C4D04469C486978C3
:1042A000DFF8888200EBC12C2878DFF88492A14ED9
:1042B000A14F2146002815BF98F8002099F800204A
:1042C00033783B7802FB03F04FEA400260460CF083
:1042D00040F89048697800EBC12C287821460028E6
:1042E00015BF98F8002099F8002033783B7802FB3E
:1042F00003F04FEA400260460CF02BF80120A87052
:10430000BDE8F08781488068704770B58B4C0546E2
:1043100001462278804852000CF01BF8227829468A
:10432000520087480CF015F878490120C87070BD1C
:104330002DE9F04FDFF8D481ADF63C0D98F802007E
:10434000CDF8200898F803B098F804A0FDF74CFBCE
:10435000CDF83808FDF741FDCDF83408FCF7E4FF4F
:10436000CDF83008FCF781FCCDF82408FDF73EFBC2
:10437000DDF8240810F0010F02D0FDF734FD04E051
:104380000020FCF7C4FFFDF776FD002425464FF022
:104390000109CDF81C4804F053FC012814D00DF598
:1043A0000060FDF705FF002800F0E9810DF50060D1
:1043B00005F08FF9002088F80100DDF80C0828B31B
:1043C000BBF1000F05D021E00120CDF81C0800F062
:1043D000BCB9002C18BF002D074621D0FEF769FE9E
:1043E000564E01213078FEF7DDFE554A3B46A2F1DC
:1043F00040010846FEF705FFFEF76EFE30783946AD
:1044000042004F480BF0A5FF88F80390DDF808083C
:10441000002800F0EF80DDF8200888B100F0EAB84D
:10442000464E3946307842003B480BF092FF3078D8
:104430003946420042480BF08CFF88F80390E5E7CC
:1044400098F80000DDF8086800283DD1D8F8087019
:1044500027B336480078CDF82C0836480078CDF8D8
:104460002808FEF726FEDDF82818DDF82C08FEF7F0
:10447000A2FE31463A460846FEF7FAFEFEF72CFE4B
:1044800030480078022804BF384604F0F9FE2D4871
:104490000078092804BF304604F0F2FE2A4800786C
:1044A000012811D9274F3878042804BF304604F07A
:1044B000E7FE314668460BF065FF0646387805286A
:1044C00004BF304604F0DCFE002C18BF002D56D08F
:1044D000CDF8286898F80000002814BF1348144845
:1044E000077814BF13481448067807FB06F0CDF888
:1044F0002C08FEF7DEFD31463846FEF753FE054E2A
:1045000098F8010006EBC02220E0000094000110A2
:10451000640D011064150110642501104C26011072
:10452000E4250110CF000110D0000110CD000110D2
:10453000CA000110CE000110CB000110D100011003
:10454000A425011051010110CC000110A6F5006155
:1045500001EBC0200146DDF82838FEF752FEFEF7D9
:10456000BBFDDDF82C08DDF82818420098F80100A2
:1045700006EBC0200BF0EDFE88F802902FE0FD481E
:1045800098F8011098F8002000EBC1203146002A6D
:1045900014BFF94AF94A137814BFF94AF94A127854
:1045A00003FB02F24FEA42020BF0D3FEF64898F802
:1045B000011098F8002000EBC1203146002A14BFFA
:1045C000ED4AEE4A127814BFED4BEE4B1B7802FB1E
:1045D00003F24FEA42020BF0BCFE88F80290EB486F
:1045E0000078032806D1E34898F8011000EBC120B9
:1045F00004F046FEDDF8140800287CD0BAF1000F64
:1046000079D1064698F8000038BBD8F80C7027B36B
:10461000DF480178DF4800780844401C40080190DA
:1046200002200090FEF745FDDDE90010FEF7C3FD16
:1046300031463A460846FEF71BFEFEF74DFDD648CA
:104640000078022804BF384604F01EFFD2480078E4
:10465000092804BF304604F017FF002C18BF002DB6
:1046600032D0CB4800960178CA4800780E18FEF781
:1046700020FD701C40080221FEF794FD98F801000F
:10468000C64F00EB800101EBC000A7F1680107EB0A
:10469000C00201EBC0010846009BFEF7B2FDFEF729
:1046A0001BFD98F80100720000EB800101EBC000D7
:1046B00007EBC00000990BF04CFE88F80490B64858
:1046C0000078032834D128E098F80100B04FB14AAF
:1046D00000EB800101EBC001B1483B78127800EBA0
:1046E000C1001A44314652000BF033FE98F8010025
:1046F00000EB800100E01BE001EBC001A7483A7825
:1047000000EBC103A348314600781044420018462C
:104710000BF01FFE88F80490D1E798F8010000EB39
:10472000800101EBC0019E4800EBC10004F0ACFE2B
:10473000FDF78DFDD8F81400641C6D1C844228BF61
:10474000854214D3D8F8100088B10420C8F81400AA
:10475000FDF74CF9DDF83008FCF7D9FDDDF8380835
:1047600090B1DDF8340868B1FDF785FB0CE0DDF8A9
:10477000240810F0010F08BFFDF77DFB0BE600F0E9
:10478000C0FE08E6FDF72FFBDDF81C0838B1DDF8A8
:10479000200888F8020088F803B088F804A0DDF843
:1047A0001C080DF63C0DBDE8F08F10B50024FDF798
:1047B000FAFA7C4910F0020F0AD08A78002A08BF62
:1047C000012410F0040F03D0CA78002A08BF012486
:1047D00010F0010F18BF10F0100F03D00879002857
:1047E00008BF01240020002C08BF10BD0020087065
:1047F000BDE810409CE508B50F2100F02EFF012810
:1048000004D1FFF7D2FF009001F093F8654881785A
:1048100000291CBF0179002904D0C07800281CBFE2
:10482000012008BD002008BD08B50F2100F015FFCC
:10483000012804D1FFF7B9FF009001F07AF8594838
:10484000817800291CBF0179002904D0C078002894
:104850001CBF012008BD002008BD70475149002041
:104860008870C870087100F0A9BC10B54FF40061E1
:1048700040480BF064FDBDE810404FF40061424831
:104880000BF05DBD2DE9F047464F8046089839781A
:10489000002914BF384939490D78A0EB030905FBFD
:1048A00009F603FB05F4FEF704FC49462846FEF72B
:1048B00079FC354D787808EB440805EBC02101EB15
:1048C0004402A5F5006101EBC02000EB4400434623
:1048D0000146FEF796FCFEF7FFFB7878720005EBC9
:1048E000C02000EB440041460BF033FD0120B870BE
:1048F000BDE8F087002818BF01202A49887070475A
:1049000070B5284D040004BFA86070BD02F02DF9F9
:1049100050B91948244B2146027819480078504371
:10492000420018460BF015FD1F48A86070BD1F49D6
:104930000020086048608860C8600861486188613C
:10494000C861086248628862C86208634863886315
:10495000C863086448648864C864086548658865F5
:10496000C865086648668866C866086748678867D5
:10497000C8677047640D0110CD000110CA00011016
:10498000CE000110CB00011064150110510101107F
:10499000CF000110D0000110560101104C2601106B
:1049A000E425011094000110641D0110642501101C
:1049B00086487047002818BF01208549C870704795
:1049C00010B5682183480BF0BAFCBDE8104068219F
:1049D00081480BF0B4BC002818BF01207C49087145
:1049E000704710B57A4C002804BFE06010BD682203
:1049F00001467A480BF0ADFC7848E06010BD744980
:104A00004861704770B5724C00210546A170E17095
:104A1000217100F0D3FB002D14BF01200020207075
:104A2000BDE8704084E42DE9F04F8BB04FF4006195
:104A30006B480BF084FC682168480BF080FCFDF7A4
:104A4000B2F90446FCF7D0FF0990FDF7C6F90890CB
:104A5000FCF76AFC0790FCF7C9FF0020FCF757FC45
:104A6000FDF709FA00252E4604F0EAF8012856D091
:104A70006846FDF79DFB00285ED0684604F029FEDD
:104A800014F0020F1CD05748DFF854B1DDF808903D
:104A900090F800805448DA460778FEF70AFB0120B8
:104AA000FEF79BFB39464046FEF785FB52464946DA
:104AB0005846FEF7DDFB0020FEF78FFBFEF70CFBF0
:104AC00014F0010F18BF14F0100F20D04748DFF882
:104AD0000CB14FF0020801784548DA46DDF8149031
:104AE00000780844401C4708FEF7E3FA0120FEF76F
:104AF00074FB41463846FEF75EFB5246494658462F
:104B0000FEF7B6FB0020FEF768FBFEF7E5FAFDF7BF
:104B10009EFB6D1C102D03D2FDF7ADF9A4E7012615
:104B2000FCF764FF0798FCF7F2FB099848B1089876
:104B300028B1FDF7A0F904E000F0E3FC94E7FDF7ED
:104B400052F9E6BB224F14F0020F19D02548DFF8C6
:104B500090C0017824486346007801FB00F21020E1
:104B60000021002A0AD933F9118008EB5008B8FB5C
:104B7000F0F52CF81150491C8A42F4D81848B86056
:104B800014F0010F18BF14F0100F18D01748134B72
:104B9000017817489C4600780A184FF010014FF032
:104BA00000000AD03CF9105005EB5105B5FBF1F4BB
:104BB00023F81040401C8242F4D80848F8600BB03B
:104BC0003046BDE8F08F01207047000064250110D9
:104BD00094000110E42501104C260110B4260110A8
:104BE000641D0110CD000110CE000110CF00011096
:104BF000D00001102DE9FF4F81B0984691468B46B9
:104C00000026FE4804240E9F90F800A0FC4805787A
:104C10000BF0BDFB01465FEA0800DFF8E88328D10E
:104C20002A1F2046042AC8BF2A1B09DD31F910308B
:104C3000142B01DB012603E0401C00B29042F5DB9F
:104C4000B7F1FF3F18BF002E13D1B9F1000F10D0FC
:104C50000198FFF7BCFA98F80000052898BF401C9F
:104C600008D9281B00902346524600215846FFF7DA
:104C700009FE002088F8000005B0BDE8F08FE1488B
:104C80004078012818BF002070470021DD48C1701E
:104C9000817070472DE9F05F00248A46B0F900204A
:104CA000B0F9021005462746A046A3462646A1466F
:104CB000501A48BF881A03B205EB4A0030F9021CAB
:104CC00030F9042C881A48BF501A00B2082BA8BF2C
:104CD000082807DB07F046FB002804BF0123AAF1E0
:104CE000020002D00023AAF1010001B218468B4253
:104CF0002ADC35F910204245C4BF904600F0FF0978
:104D000098421DDD05EB400C3CF902CCACEB0202F5
:104D1000D21D0E2A05D804F1010C0CF0FF048842C4
:104D20000ED1A7420BD22746884203D10E2A98BF44
:104D300046B201D9421E56B2F21B4FFA82FB002442
:104D4000401C80B28142D4DAAAF10400874205DD1A
:104D5000CB45DEBFB1450020BDE8F09F0120BDE896
:104D6000F09F70B5A94AA84906461478097800EB67
:104D700044021046FFF78EFF054621463046FFF7F6
:104D800089FF00229F49002D1CBF0028CA7008D14E
:104D9000C878401CC0B2C8700A2882BFCA70002000
:104DA00070BD012070BD2DE9F34F91B00CA8119991
:104DB000079003A80590944800270DF1080E00788D
:104DC0000090019091480DF1100B3E46027806923A
:104DD000B1F9005031F912C0ADF8302001202C4655
:104DE0006346ADF80870ADF80C20ADF81070012ADC
:104DF00024DD31F91080A845C8BF4546A045BCBF99
:104E00004446ABF8000001EB400831F9109038F946
:104E100002ACBAEB090848BFA9EB0A080FFA88F8F8
:104E2000B84507DD4746CA45D4BF8046A0F1010812
:104E3000AEF80080401C00B28242DADCDDF804806B
:104E4000501C08EB020A824524DD31F9102062452E
:104E5000C8BF94469A4202DA1346059A108001EBC5
:104E6000400231F9108032F9029CB9EB080248BFC8
:104E7000A8EB090212B2B24208DD1646C145D4BF02
:104E80000246421EDDF81C80A8F80020401C00B23B
:104E90008245DADC5E48ACEB03030268012092F83D
:104EA0001F118B42C4BF2B1B8B4205DD92F81E11D4
:104EB0008E42C8BF8F4200DC00200890002800F01E
:104EC0000D81DDE91145BDF930000590BDF90800FF
:104ED000079000980F90069E0020CDE90A060F98D3
:104EE000771E3044A0F101080690059834F91000AF
:104EF0000E90079834F910000D900020009001905A
:104F00008346824681460990FFF757F90146002003
:104F100002461090079800280BDB34F910C00D9B57
:104F2000BCEBA30F01DA0A9003E0401E00B28242FC
:104F3000F3DD0798B31A83420CDD34F910E0DDF895
:104F400034C0BEEBAC0F01DA074603E0401C00B2F0
:104F50009842F2DB0598B31883420CDC34F910E078
:104F6000DDF838C0BEEBAC0F01DA0B9003E0401E59
:104F700000B28342F2DDDDE905039B1A83420BDDBB
:104F800034F910C00E9ABCEBA20F01DA804603E0A0
:104F9000401C00B29842F3DB0B9840453DDA05EB2C
:104FA000400235F91030B2F902C0B3EB0C0248BF31
:104FB000ACEB0302019B1A4412B2019201EB4002D6
:104FC00031F91030B2F902C0B3EB0C0248BFACEBC0
:104FD0000302009B1A4412B2009204EB400234F91F
:104FE0001030B2F902C0B3EB0C0248BFACEB0302C5
:104FF000099B401C1A4412B200B20BE0CA00011017
:10500000CB000110AC000110CF000110D000011046
:10501000DC01011009924045C1DB0A98B8422DDA43
:1050200005EB400235F910C0B2F90230BCEB0302C7
:1050300048BFA3EB0C0252440FFA82FA01EB400284
:1050400031F910C0B2F90230BCEB030248BFA3EB48
:105050000C025A440FFA82FB04EB400234F9103080
:10506000B2F902C0B3EB0C0248BFACEB03024A44F6
:10507000401C00B20FFA82F9B842D1DBDDE9000131
:10508000411A0998B1EB600FDFBFABEB0A00B0EB40
:10509000690F109800280AD0EB498878401CC0B2EC
:1050A0008870032884BF002088701BD912E0E6496D
:1050B000002088700B98A8EB00010F98B1EB600FEF
:1050C00004DC0A98381AB0EB660F0BDD2046FFF7B8
:1050D00048FE38B94FF0FF30089003E0DA4900206D
:1050E000C8708870089813B0BDE8F08F0120704731
:1050F000D548008B80B270470120704770B51546C7
:105100000E46044606F0F7FF002C18BF70BD0428B9
:1051100018BF052806D0CD48006890F82400A842A2
:1051200088BF70BD3046BDE870400BF035B9C64849
:10513000407B7047DDF800C001434FF0000008BF1E
:105140008CF8000052EA030108BF8CF80000704799
:105150002DE9F047994614460D468246089E06F012
:105160007BFFB94F4FF0060828B9B4EB450FC8BF15
:10517000A6F800800BDC06F06FFF012807D1B9F11B
:10518000000F0CBFBAF1FF3F002004D03872BD827F
:10519000FC82BDE8F087B7F91400B7F9161008448F
:1051A0002919884202DA387A401C3872387A06287F
:1051B00024BFA6F800800520E9D3E7E7A248002134
:1051C0008182C18206F04BBF9F490020C87248838C
:1051D000087370472DE9F04790468946044606F06B
:1051E0003BFF994E002750B3B6F91A008442C8BF5E
:1051F000748320460BF0D5F804460D46B6F91A0024
:105200000BF0CFF8924A934B0BF0B2F822462B46A4
:105210000BF0E0FA18D2B9F1010F15D0F07A401C6A
:10522000C0B2F0720A2898BFBDE8F087F7727783A2
:1052300001203073FF2088F80000BDE8F087F77286
:1052400077833773BDE8F087F772BDE8F08782494E
:105250000180418081800021C180018142F20F7272
:1052600042818181C1810182418270472DE9F047ED
:1052700005467A4892460F4690F8009078480A26EC
:10528000002490F8008006F0E7FE01466E480129F0
:1052900016D0B0F91810012930DD1E23428A0021F2
:1052A000A2421CBF44828173002219EB080C12D069
:1052B00035F912409C420ADD81730020BDE8F08779
:1052C0003C2301240526BAF1000FE7DDE5E7521C77
:1052D00092B29445ECD8827B0123521CD2B28273E5
:1052E000B24288BFC37302D8C27B012A06D14FF0F5
:1052F000FF323A60C371C173817301720020BDE84F
:10530000F08770B515460C4606F0A6FE01281ED1A2
:105310004D4B4FF0000C002DC2BF83F810C0002091
:1053200070BD187C0121401CC0B218740A2888BFC7
:10533000597402D8587C012809D14FF0FF30206001
:10534000D97183F811C083F810C083F808C0002019
:1053500070BD10B5044606F09BFF002808BF10BDC5
:105360000BF024F8092804D00BF020F80A2818BF05
:1053700010BD06F0FCFF012818BF10BD4FF0FF3034
:10538000314920600120C87110BD2DE9F84F1D463C
:10539000DDE90A499246064606F0ADFE00962A4E21
:1053A0000027777306F074FF4FF0010858B106F03C
:1053B0006FFFD8B10AF0FAFF09280FD00AF0F6FF04
:1053C0000A280BD012E04A4669465046FFF74EFFC6
:1053D0004A4669465046FFF794FF07E006F0C7FFCC
:1053E000012803D1801E009086F807800098B0F154
:1053F000FF3F15D00098002806BF70790128BDE84E
:10540000F88F777186F80D80002D1CBF2846FEF7B7
:1054100011FF002C1CBF20460AF0CDFFBDE8F88F1D
:10542000F079012818BFBDE8F88FF77186F80D8074
:10543000002D1CBF2846FEF72DFF002C1CBF204668
:10544000FEF7C5FED6E70000AC000110DC0101103C
:10545000CDCCCCCCCCCCE43FF1D8FFFFCF000110B9
:10546000D000011010B504F0CBFF05F053F8002078
:1054700010BD0000FE4800787047FD480078022803
:1054800005D005281CBF0020704704F09ABA06F02A
:1054900032BEF7490870704770B5F54D04460E46A8
:1054A0002878A04211D0022817D0052814BF002068
:1054B00004F087FA44EA06212A7841EA024141EAE7
:1054C00000621521012006F0CEFA062C28BF70BD1F
:1054D000DFE804F015060A12150E06F00CFEE9E7E7
:1054E000304600F033FA0AE0304606F0F9FD06E0F7
:1054F000304604F05BFA02E0304606F05DFB2C70AB
:1055000070BDDC4900200968B1F8641011F4807F97
:1055100008BF7047FDF7D7BAD64900200968B1F82F
:10552000641011F4807F08BF7047FDF7E1BAD149DC
:1055300000200968B1F8641011F4007F08BF7047BB
:105540000AF03EBFCB4900200968B1F8641011F49D
:10555000806F08BF70470AF038BFC54948780028F7
:105560001CBF401E4870704770B5C3490868D0F82A
:10557000CC00BF4C10F0030F0BD0096840F4BE0004
:1055800040F02040C1F8C8006078002804BF012026
:105590006070BA4800688068B64D10F0020F296844
:1055A00007D1B7480068406910F0010F01D060785A
:1055B00040B1B1F86410002011F4807F18BFFDF7EE
:1055C00097FA07E0B1F86410002011F4806F18BF5B
:1055D0000AF0FBFEAB49084208BF70BD2968496E5E
:1055E000090C617070BD10B572B6FEF759FDBDE8CB
:1055F0001040FEF722BA10B5012802D0022805D0CB
:1056000008E04FF42F30FDF761FB03E09C499E4812
:105610000968086772B6FEF743FDBDE81040FEF763
:105620000CBA9348006970479148C0687047904928
:10563000486170478E48406970478D49886170475E
:105640008B48806970478B48026802F5B073118AF5
:10565000508A02F5A072FCF772BC2DE9F04FDFF81A
:10566000109297B00E46C9F8100004F02DFEC9F84C
:105670000C0000287DD090F800C089F802C0417865
:1056800089F80310837804460CF1010089F804308E
:1056900000F0FE0089F80500E27889F806202079FC
:1056A00089F80700607989F8080009F10A004FF0CD
:1056B000000B80F800B080F801B0207889F809006C
:1056C0006046FCF741FD99F8081099F80700FCF7CF
:1056D0005EFD6946204604F014FE606A10F4801FE7
:1056E00008D0FCF769FB28B10C9808900D98099038
:1056F0000E980A90608AD9F8145000281CBF68439D
:10570000050B678BD9F81880002F08BF4FF480571E
:105710004FF4805A002016F0020F18BF40F21120FB
:1057200016F0040F18BF40F4857016F0080F18BF6C
:1057300040F0040016F0010F18BF40F48460616A65
:1057400008406FF30F0141EA00060098109004989A
:105750001190089812900198139007981590CDF821
:1057600050B010A93046FCF73DFA16F0020F72D087
:1057700000E02BE004F0A5FA5FEA000B33D004F060
:10578000B7FA6843050B59460020FBF7E1FD218A73
:1057900000291CBF0020FBF752FE04F0C9FA08FBE9
:1057A00000F0000B00F50060010A0820012202FA57
:1057B00000F30B4201D1401EF9D5A0F10408A07BF3
:1057C000002818BFA0F1010B17D112E0294800688A
:1057D000B0F8640010F4807F18BFFDF789F900204D
:1057E00017B0BDE8F08FB4F80CB0BBF1000FCAD110
:1057F000CDE70020FBF7A1FE8346E07B002814BF25
:10580000401EFBF7C9FE0BEB0801042905DDA8EBE0
:10581000010101F10408042104E00029BCBFA8EB48
:10582000010800218044B8F1040F05DDA8F104004F
:10583000C5404FF0040807E0B8F1000F04DAC8F1E2
:10584000000085404FF000080020FBF78CFE414629
:105850000020FBF7B7FE16F0010F40D0A18A002907
:105860001CBF0120FBF774FDB4F818800EE00000A7
:10587000C8000110DC010110E42B0100E82B01003D
:10588000DC2B010008000300AD2007B0B8F1000FC9
:1058900007D041460120FBF7D2FD41461120FBF71E
:1058A000CEFD94F81680B8F1000F09D0A8F10101DF
:1058B0000120FBF758FEA8F101011120FBF753FE70
:1058C00094F81780B8F1000F09D0A8F10101012068
:1058D000FBF778FEA8F101011120FBF773FEE07AD7
:1058E00000281CBF0001FBF771FC029804F0C5F909
:1058F000039830B12B4699F8032099F802100AF06A
:1059000069FD5246394628460AF069FD0598FEF7BA
:10591000F7FF069800F0F7FF16F0100F05D0099872
:10592000FFF75FF80A9801F07CF817B00120BDE896
:10593000F08F10B5FCF7F2F904F0A7F90249002046
:10594000C860012010BD0000C8000110FE49487069
:105950007047FD4840787047FC4810B4FC4A016825
:10596000914218D14168B1F5887F14D80022D0F84F
:1059700008C003461146B2EB9C0F24BF10BC704711
:1059800053F82140491C2244B1EB9C0FF8D3002A64
:1059900004BF10BC7047002010BC7047EB48FDF7F7
:1059A00095B9E949012048707047E749002008701F
:1059B00070472DE9F34FDFB000200F4647904E901F
:1059C0004D9072B6FCF7EFF90646FEF726F948B19E
:1059D000FEF7FDF94E90FEF7DAF9FEF7FEF94D906D
:1059E000FEF7E5F9FCF7EFF8FBF7FEFF5790FCF741
:1059F000F4F95690FBF7FAFFFDF7D8FE5590FDF746
:105A0000B9FE4FF49350FDF72AFE62B60022154608
:105A100030AC44F82250521C062AFAD3DFF83493F3
:105A200016F0020F4FF0010809D0CDF8C080D9F868
:105A300000004FF4046100F580400AF080FCC54A84
:105A400016F0010F44F64000126802EB000612D077
:105A50004FF4007130460AF072FC0120FAF76DFE37
:105A6000002818BFCDF8C8801120FAF766FE00287C
:105A700018BFCDF8CC80DFF8E0B2DFF8CCA23098C8
:105A800080B30020FBF74CFD00909BF800008DF8E0
:105A90000400B2480078012894BFB148B1480078AA
:105AA0008DF805000020FBF709FE002818BF4FF015
:105AB000FF3003908DF80670BAF80400ADF80800C6
:105AC0000020FBF7D7FCADF80A00D9F8000000F57C
:105AD00080400590D9F800000690D9F8000000F544
:105AE000005007903198FF2748B30020FBF718FDBE
:105AF00008909BF800008DF824008DF825800B9508
:105B00008DF82670BAF80400ADF828000020FBF7E5
:105B1000B1FCADF82A009DF80500D9F8001001EBA2
:105B2000801101F580410D919DF804104843D9F88A
:105B3000001001EB40000E9000F500500F908A4DD0
:105B4000DFF828B2329870B30120FBF7E9FC10901F
:105B5000FBF797F800280CBF9BF8000028788DF819
:105B600044000120FBF7E9FC08FA00F08DF845003D
:105B70000120FBF795FDC04313908DF84670BAF8ED
:105B80000600ADF848000120FBF774FCADF84A00B0
:105B90001596D9F8000000F504601690D9F80000B9
:105BA00000F521501790339898B31120FBF7B8FCFB
:105BB0001890FBF766F800280CBF28789BF80000C7
:105BC0008DF864001120FBF7B8FC08FA00F08DF89E
:105BD00065001120FBF764FDC0431B908DF86670D3
:105BE000BAF80600ADF868001120FBF743FCADF8E9
:105BF0006A00D9F8000044F6C00108441D90D9F8A5
:105C0000000000F52C601E90D9F8000000F52B5024
:105C10001F909DF845100220022988BF8DF845008D
:105C20009DF86510022988BF8DF865004FF055304A
:105C30001B901390BDF8480000F58060ADF8480057
:105C4000BDF8680000F58060ADF86800FBF722FD44
:105C500058900120FBF70FFD0120FBF745FD5B90FD
:105C60000020FBF70AFF5A900020FBF7FBFE59903B
:105C70000020FBF74CFB5C90FCF7FDF800204A90FD
:105C80004990379045904798002840F0C28302F031
:105C9000D7FF012800F0BD834A98802800F2B9831D
:105CA0003EA8FCF785FA002800F0AD833EA803F07B
:105CB00010FD4998401C499000F09C8300204990B9
:105CC0004A98401C4A90002038AA012142F820102E
:105CD000401C0628F8D33798002808BF369013D008
:105CE000012804BF0020369000F0FC80022804BF89
:105CF0000020369000F02982032804BF012047903D
:105D000000F0578300F085BB369930A850F8210089
:105D100000287CD0369A684600EB42100022489258
:105D200007794279D0F800804692B0F9086042695C
:105D30004C9245998269C068C1F105054B9099B3B1
:105D4000002D65DB14E00000E400011000AF02004C
:105D500054435246F82B0100CD000110CC00011035
:105D6000CB000110CE000110CF000110D0000110B7
:105D700046984FF00009002864D905F10800012178
:105D800001FA00FBE81D01FA00F0519001234B9845
:105D900003FA09F1084018BF0120002152904C98E5
:105DA0008C4600EB891A84E0FFE746984FF0000A22
:105DB000002847D901214B9801FA0AF3034214BF86
:105DC0004FF0010E4FF0000E00204C99844601EB7D
:105DD0008A1B30E00121814011EA080F28D04108D8
:105DE0004F915BF82190C1074FEA19434FEA0343F3
:105DF000CC0E29FA04F132F9023B89B29B1B0CF15B
:105E0000010CBEF1000F18BF5B42002B01E061E006
:105E10005BE0C8BF41F4005141F480514FF6FF737D
:105E2000A34029EA0303A1400B434F994BF82130CB
:105E3000401C202801D2BC45CCD346980AF1010A67
:105E40008245B7D33DE00120884010EA080F2DD0ED
:105E5000480850905AF82000CB07DC0E4F90E040E5
:105E600032F9023BDDF848E19B1B80B20CF1010CDA
:105E7000BEF1000F18BF5B4210F4005F02D0002B90
:105E800004DA01E0002B01DD20EA0B00002DC4BF85
:105E9000519B18434FF6FF7E0EFA04FE4F9BA04025
:105EA00023EA0E03034350984AF82030491C202966
:105EB00001D2BC45C7D3469809F101098145FFF4D9
:105EC00065AF002D04BF0120489038A9369A489844
:105ED00041F822003698401C36900628FFF414AF93
:105EE00000F067BA369930A850F82100002800F079
:105EF0002481369A684600EB4210002245994F9261
:105F000004794679837905684893B0F90880426935
:105F10004B92C368826951934089489BC1F108073D
:105F200018405090D9B1002F73DB4FF0000A002EBB
:105F30006ED90120B8404C90781E012101FA00F082
:105F400054900123519803FA0AF1084018BF012028
:105F5000002146904B988C4600EB8A1B93E04FF053
:105F6000000A002E54D90123519803FA0AF108407F
:105F700018BF0120002146904B988C4600EB8A1BED
:105F800040E001208840284239D0480852905BF810
:105F90002000CB074FEAD3694C9020FA09F032F980
:105FA000023BDDF818E180B2A3EB08030CF1010C11
:105FB000BEF1000F18BF5B4210F4005F09D0002B48
:105FC0000EDA10F4F85018BFA0F5807040F40050BD
:105FD00006E0002B04DD10F4F85018BFA0F5807027
:105FE00040F080004FF6FF7E4C9B0EFA09FE23EA3C
:105FF0000E0300FA09F0034352984BF82030491C75
:10600000202901D2A445BCD30AF1010AB245AAD382
:1060100040E043E001208840284231D048085390B6
:106020005BF82000CB074FEAD369529020FA09F0C1
:1060300032F9023BDDF818E180B2A3EB08030CF162
:10604000010CBEF1000F18BF5B4210F4005F02D0DC
:10605000002B04DA01E0002B01DD4C9B9843002F5C
:10606000C4BF549B18434FF6FF7E529B0EFA09FEA5
:1060700023EA0E0300FA09F0034353984BF820304B
:10608000491C202901D2A445C4D30AF1010AB24512
:10609000FFF457AF002FC8BF4F984ADC4FF0000AFB
:1060A000002E44D94898C0F580704690489840F436
:1060B000807B4B990020024601EB8A1931E00121D7
:1060C0004FEA174C81404FEA0C4C294226D04FEA48
:1060D0005008C10759F82870CB0E27FA03F11FFAB0
:1060E00081FCDDF818E10CF0FF0101EB5E01DDF849
:1060F00040E101EA0B01521C714588BF71462CF04A
:10610000FF0C4CEA01014FF6FF7C0CFA03FC27EA76
:106110000C0C99404CEA010149F82810401C202839
:1061200001D2A242CBD30AF1010AB245C1D3012068
:106130004F90369A38A941F822003698401C369084
:106140000628FFF4CFAE00F034B9369930A850F8E5
:106150002100002800F0278145985390684600EB05
:10616000411000214F910168519101794891417985
:1061700046918179B0F9089042695292D0E906843B
:106180004289C06850905398C1F5807602EA0107B1
:1061900010F0010F13D046984FF0000B00287DD966
:1061A0000121509801FA0BF2104018BF01204B90CA
:1061B0005299002001EB8B1182464C91E0E00020C7
:1061C000FBF792FA0546469948984143032000EBB5
:1061D000410020F00302414620460AF0BAF8284662
:1061E000FBF782FA46984FF0000B002856D901229F
:1061F000509802FA0BF1084018BF012000214B9083
:1062000052980D4600EB8B1E4FE0012000FA01F280
:106210005198024246D038F9020B6D1CA0EB0903DD
:106220004B98002818BF5B42480854905EF8200045
:10623000CA074FEAD26A4C9020FA0AF082B2C2F33F
:10624000042002F0FF0C12F4005F02D0002B02DBEE
:1062500004E0002B02DDACEB060401E00CEB0604CD
:10626000BC4205DD1F283ABF0024401C3C4606E026
:10627000002C04DA0028C6BF3C46401E002402F46D
:10628000005242EA00204FF6FF734C9A204303FA73
:106290000AF39A4300FA0AF0024300E079E05498C6
:1062A0004EF82020491C202902D248988542ACD3C0
:1062B00046980BF1010B834599D36AE0012101FA5D
:1062C00000F251990A4258D034F9021B4B9AA1EBC3
:1062D00009010AF1010A002A18BF494238F9022BC4
:1062E000A2EB090218BF52420029B4BF4B420B4631
:1062F000002AB8BF52429A423FD94C9B420854925E
:1063000053F82220C3074FEAD36E5D9222FA0EF2B1
:1063100093B2C3F3042203F0FF0C13F4005F02D026
:10632000002902DB04E0002902DD0CEB060501E098
:10633000ACEB0605BD4205DD1F2A3ABF0025521C05
:106340003D4606E0002D04DA002AC6BF3D46521E37
:10635000002503F4005141EA02214FF6FF725D9BD4
:10636000294302FA0EF223EA020201FA0EF142EA8E
:106370000103549A4C9941F82230401C202802D243
:1063800048998A459AD346980BF1010B8345FFF44F
:1063900007AF5398032826BF01204F904F9838A984
:1063A000369A41F822003698401C36900628FFF4B1
:1063B000CCAE0123002038A951F82020EAB1401CBE
:1063C0000628F9D3CBB137981F2811D2401C0121E0
:1063D00001FA00F237905F98024209D13798401CC9
:1063E0003790032804D801FA00F25F980242F5D0F2
:1063F00000204590479818B10BE04598401CF8E7FD
:10640000FBF739FD43E4FFF787F8479800283FF48E
:106410003EACFBF7EBFA5898FBF72DF95B98FBF7CE
:1064200063F95A98FBF729FB5998FBF71BFB5C981B
:10643000FAF76DFF579830B1569810B1FBF71BFD76
:1064400001E0FBF7D0FCFDF7E8FB48B14E980028CF
:1064500018BFFDF7E8FB4D98002818BFFDF72FFC8B
:106460005598002818BFFDF740F9479800280CBF41
:106470000120002061B0BDE8F08F2DE9F14FADF6AD
:10648000080D00200090FBF797FC4FF000080190EA
:1064900000F0FCB8404603F017FF002800F0F4803D
:1064A0000189DDF8080801EA000424F0CC0030F48A
:1064B0007C4000F0E9800020FBF778FC0F2140468B
:1064C000FFF7CBF8002800F0DF80FBF76CFC81467B
:1064D00020F480150098002840F0D4802846FBF76F
:1064E0005AFBFF210F20FFF764FA0090FBF77EFABA
:1064F000009800287DD114F0010F0ED0FFF794F81A
:10650000074602AE4FF0040A3046FBF7A4FE97F9A7
:106510002C103246504603F016FF14F0100F2BD00B
:1065200005F4801040F00106FFF77EF8824616F071
:10653000020F0BD00DF1080B04275846FBF78BFE1A
:106540009AF92C105A46384603F0FDFE16F0010F5A
:1065500012D00DF1080B082759460120FBF7D3FE96
:1065600016F4801F18BF0C270AEB07005A4690F953
:106570002810384603F0E7FE0098002839D114F0BF
:10658000660F07D0FEF74FFA0090FBF72FFA00983E
:10659000002877D114F0020F0CD0FDF7B3FE0646A9
:1065A000FFF742F80523320004D090F92D10184669
:1065B00003F0C9FE14F0040F0CD0FDF7A3FE06464D
:1065C000FFF732F80623320004D090F92E10184657
:1065D00003F0B9FE14F0200F25D005F4801040F030
:1065E000010715F0100018BFFDF71BFE82461026AC
:1065F00000E047E0FFF718F817F0020F18BF052674
:1066000007D117F0010F04D017F4801F0CBF092623
:106610000D265246102E06D22AB1304490F9281089
:10662000304603F090FE14F0400F23D005F48010A4
:1066300040F0010715F0100018BFFDF7F2FD82468B
:106640001026FEF7F1FF17F0020F18BF062607D13C
:1066500017F0010F04D017F4801F0CBF0A260E2676
:106660005246102E06D22AB1304490F928103046F6
:1066700003F069FE009828B919F4801F02D015F4C0
:10668000801F1AD0FFF755F908F1010803F018FE32
:10669000404503D9009800283FF4FCAE0198FBF771
:1066A00085FBFF4900200870009800280CBF0120DE
:1066B00000200DF60C0DBDE8F08F0120FBF776FBF6
:1066C00045F4801504F0700408E72DE9F04FF44814
:1066D000CDB04478FEF7CEFE012870D1F1480068B5
:1066E000B0F93610B0F9340009F07EFE14F0020F54
:1066F0007ED00DF5807BFFF72FF90025EA4F30267D
:106700004FF488784FF050094FF0FF3A78B1B0E875
:106710000E108BE80E10B0E80E100DF5887B8BE89C
:106720000E100FC80DF5907B8BE80F0013E0FF22D1
:106730003021584609F05DFECDE94495CDE942652A
:10674000CDF82CA1CDF828A1CDF824A14695CDE90E
:10675000475ACDE94078DFF854B35846FCF7B6FA0B
:106760004598401C459040F27770FFF786FE01285F
:1067700003D1FEF728FA012817D047980022401CC1
:1067800047901F21CDF81091022005F06CF90DF50E
:10679000807903F079FD98B181694891C169499187
:1067A00041694A91C0684B9012E014F0080F14BF81
:1067B000A220A12044904698401C4690E7E74EE076
:1067C000CDF82CA1CDF828A1CDF824A1CDF820A199
:1067D000CDE94265CDE940780021D9F808304A4634
:1067E000084652F820C0401C6144B0EB930F00E013
:1067F0001DE0F6D34D42FF22511C6846C9F80C50EB
:1068000009F0F7FDD9F80820F9E804018DE8270020
:10681000B9E80F0004AD85E80F0099E80F0008AD56
:1068200085E80F0058466946FCF7FDFA10E014F0C1
:10683000010F0DD040F22220FFF71FFE012808BFF4
:10684000FEF7C1F920B901221F21022005F00BF942
:10685000FEF704F801212246084605F004F94DB080
:10686000BDE8F04F02F0B6B98D49888070478C4979
:10687000C880704770B50126FFF76EF820B1006937
:10688000A12818BFA22801D0002070BD002403F069
:1068900017FD002831D9204603F016FD00281EBF41
:1068A000058925F0CC0030F47C4021D00F21204612
:1068B000FEF7D3FEE0B115F0010F09D0FBF7F0FCB5
:1068C00030B944F480721E21022005F0CCF8002675
:1068D00015F0100F0AD00120FBF754FD30B944F435
:1068E00080521E21022005F0BEF80026FFF721F895
:1068F000641C03F0E5FCA042CDD8304670BD0020FA
:106900007047002070472DE9F04F654EADF60C0D35
:106910000028B06004BF0DF60C0DBDE8F08F317893
:1069200011F0020F6BD16249DFF88C810C7861495C
:106930000D78C6F80C800090FDF7E4FCCDF8040853
:106940005E4890F800905E4807785E4890F800A096
:10695000BAF1010F8CBF0DF1040BC346DDF804083A
:106960000099002809FB07F04FEA40024BD001A82C
:1069700009F0EFFC4B4601AA00975846DDF80418D1
:1069800009F02CFEBAF1010F0FD95946404609F023
:10699000F9FC404509D0464A014640461378454A2D
:1069A00012785A43520009F0D4FC0027F068B84628
:1069B000002D18D930F9021B0122012C0FD930F912
:1069C00002CBACEB010109B20029B8BF49420BB2BE
:1069D000BB42C8BF1F466146521CA242EFD308F11A
:1069E0000108A845E6D32F480068B0F82C01B8424A
:1069F000C4BF0020F060307840F0020030700DF627
:106A00000C0DBDE8F08F584609F0A3FCBAE7244806
:106A1000816800291BBF017811F0020F0020C068B7
:106A200070472DE9F84F1E4E0028306108BFBDE8C1
:106A3000F88F317811F0100F18BFBDE8F88F224D94
:106A4000824622484FF00009047821480778FBF776
:106A5000AAF910F0100F02D0FDF7E3FB814604EB1A
:106A600007084FEA48025146284609F072FCB9F17E
:106A7000000F09D00220009008F1010043082A46C7
:106A80004946104609F0AAFD0020B5F90030A91CBE
:106A90000122012F2AD931F902CBACEB030319E013
:106AA000E4000110DC0101105443524600AF020023
:106AB000CA000110CB0001101C270110CD000110ED
:106AC000CE000110CC0001101C2F0110CF000110CE
:106AD000D00001101BB2002BB8BF5B421BB2834237
:106AE000C8BF18466346521CBA42D4D331F9023BA0
:106AF0000122012C0FD931F902CBACEB03031BB2FD
:106B0000002BB8BF5B421BB28342C8BF1846634626
:106B1000521CA242EFD31F490968B1F82E118142DD
:106B2000C8BF00257561307840F010003070BDE8B6
:106B3000F88F1948016900291BBF017811F0100F67
:106B400000204069704713481349006890F82521D8
:106B50008878401CC0B28870824228BF70470020ED
:106B6000887001210846FEF797BC0B48C078704733
:106B700009490020C870704710B50446FDF7C2FBF4
:106B80004FF40062214609F0E4FB03490120C8707C
:106B900010BD0000DC010110E4000110704700206E
:106BA000704710B503F00700042808BFFEF71BFD6F
:106BB000002010BD70B503F00702FA4CFA4B4FF0FD
:106BC000000C012A02D0022A23D020E005201870F0
:106BD000C3F80CC0FCF776FF2168AC260E70226863
:106BE000010A51702168887003F004FB78B1EF4D01
:106BF000286803F0E5FB50B1286890F8200010F0F9
:106C0000020F04D02068467021684320887000205D
:106C100070BD1A78052A11D1DA68032A28BF1046F8
:106C200004D22468A45C0470501CD860032805D1E9
:106C30000120C3F80CC0087003201870012070BD3B
:106C40002DE9F04103F00702D64C0025D64E012A6B
:106C500002D0022A56D052E0FCF734FF05213170F1
:106C6000002122685554491C0E29FADB2268AC2108
:106C700011702168020A4A702168887003F0BAFA1C
:106C800000283BD0C94F386803F09AFB002835D064
:106C900038682168807CC87038682268017C11716E
:106CA000017E11F0040F0ED0C18A2268090A5171C9
:106CB0002268817D9171818A2268090AD1712268D6
:106CC000017D11720DE0818A2268090A51712268E2
:106CD000017D9171C18A2268090AD1712268817D82
:106CE000117222682021517222680221917221685A
:106CF000CD7221680D732168007E4873F560002015
:106D0000BDE8F0813278052A10D1F2680E2A28BF3A
:106D1000104604D223689B5C0370501CF0600E2860
:106D200004D10120F5600870032030700120BDE817
:106D3000F08103F00702022A1CBF002070472022C6
:106D400002700120087070472DE9F041964F0D4602
:106D5000064613F0070F04D003F00700022808D0FE
:106D600004E012F0040F1CBF0020B8700020BDE842
:106D7000F08101F029FF002814BF0124002401F054
:106D800026FF002814BF0222002242EA0403B8783A
:106D9000002814BF0422002242EA030030700120C0
:106DA0002870BDE8F08170B503F0070C00267E4C1A
:106DB0007C4DBCF1010F0AD0204613F0070F00787C
:106DC0000DD0BCF1040F08BF062818D029E0E660FA
:106DD00028680670286846700520207021E0052884
:106DE0001FD1E068022803D22B681A54401CE060CF
:106DF000022816D10120E6600870062010E02868FD
:106E0000007855280BD128684078AC2818BFBC28DA
:106E100005D128680122411C062001F0BBFE032099
:106E20002070002070BD10B403F0070C00235D4AF1
:106E30005D4CBCF1010F03D0BCF1020F37D033E041
:106E4000052020704FF42F30E3600168880AC0F1FC
:106E5000000C11EB8C2C18BF401C404201EB800051
:106E6000C01C20F0030041F6E8710144B0F5283F52
:106E700014D891F803C008686CF31F60DFF830C1C4
:106E8000604508BF002009D10B18D2F800C01B795B
:106E90000CF80030401C1428F6D305E000201168DF
:106EA0000B54401C1428FAD310BC0020704794F8EF
:106EB00000C0BCF1050F14D1D4F80CC0BCF1140F04
:106EC00028BF604606D2126812F80C2002700CF13E
:106ED0000100E060142804D10120E3600870032061
:106EE000207010BC0120704710B403F0070C002381
:106EF0002C4A2D4CBCF1010F03D0BCF1020F59D02C
:106F00004CE0052020704FF42F30E3600168880AC0
:106F1000C0F1000C11EB8C2C18BF401C404201EB5F
:106F20008000C01C20F0030141F6E8700844B1F570
:106F3000283F2DD890F803C001686CF31F61DFF87B
:106F400070C0614524D11368017C19701368417CBD
:106F500059701368817C99701368C17CD97013686B
:106F6000017A19711368417A59711168837A8B71AA
:106F70001368C17AD9711368017D19721368417D54
:106F800059721368817D99721168C07DC87205E0DD
:106F9000002011680B54401C0C28FAD3002010BCB0
:106FA00070470000FC2B010004010110DC010110FE
:106FB00034CD12AB94F800C0BCF1050F14D1D4F855
:106FC0000CC0BCF10C0F28BF604606D2126812F844
:106FD0000C2002700CF10100E0600C2804D10120AB
:106FE000E3600870032020700120D8E770B503F03B
:106FF00007020025FD4CFE4E012A02D0022A36D09F
:1070000033E003F041F940B3D0E906212368C068BA
:107010001A70D4F800C0130A8CF80130D4F800C0FC
:10702000130C120E8CF802302368DA70226811718A
:1070300023680A0A5A7123680A0C090E9A71226899
:10704000D171216808722268010A51722268010C0C
:107050009172010E2068C17204E021680D54401C39
:107060000C28FAD305203070F560002070BD32780E
:10707000052A10D1F2680C2A28BF104604D22368D2
:107080009B5C0370501CF0600C2804D10120F5605B
:10709000087003203070012070BD30B403F0070287
:1070A000D24BD34C4FF0000C012A02D0022A4ED012
:1070B0004AE0052020704FF42F30C4F80CC001685E
:1070C0000025880A424211EB822218BF401C404230
:1070D00001EB8000C01C20F0030101F50050B1F568
:1070E000283F98BF10F0030F27D1C24A0168914290
:1070F00004BF0022114620D150F82140491C2244EF
:107100000729F9D302B1C5B11A68017C11701A6858
:10711000417C51701A68817C91701A68C17CD17071
:107120001A68017D11711A68417D51711A68817D5B
:1071300091711968C07DC87106E00020196801F8D6
:1071400000C0401C0828F9D330BC002070472278CA
:10715000052A11D1E268082A28BF104604D21B680C
:107160009B5C0370501CE060082805D10120C4F826
:107170000CC008700320207030BC012070472DE93E
:10718000F04103F0070C0027994E4FF00508BCF1C1
:10719000010F0DD013F0070F0FD03246BCF1020FD4
:1071A000127810D0BCF1040F08BF062A26D065E083
:1071B00086F800807770F76060E072708E48306308
:1071C000062030705AE0052A15D1F268042A28BF3B
:1071D000104609D2C2F10303D6F830C0DB002CFA06
:1071E00003F30370501CF060042804D10120F76001
:1071F0000870032030700120BDE8F081737801250C
:10720000002413F0010F1FD04FF42F300168880ABB
:10721000424211EB822218BF401C404201EB800029
:10722000C01C20F00302B2F5283F23D800204FF401
:107230000051B0EB920F07D251F804CB401C6444CC
:10724000B0EB920FF8D3ADB113F0020F0ED003F0F4
:107250001BF878B182680021B1EB920F06D250F88A
:10726000043B491C1C44B1EB920FF8D3002D18BF0E
:10727000346300D13763777086F800800020BDE862
:10728000F08170B503F0070C0026584C584D82B0C1
:10729000BCF1010F06D013F0070F11D0BCF1020FA3
:1072A00020D01CE001A9684601F021FF05202870CC
:1072B000216801980870216800984870EE600EE01F
:1072C000E868022803D221680A54401CE8600228BA
:1072D00005D1EE6020680178407801F0FFFE02B031
:1072E000002070BD2A78052A10D1EA68022A28BF3A
:1072F000104604D223689B5C0370501CE86002288F
:1073000004D10120EE6008700320287002B0012033
:1073100070BD08B503F0070001280AD102F06AFF2A
:1073200038B101208DF80000024669460D2001F0B9
:1073300031FC002008BD08B503F0070001280AD180
:1073400002F058FF38B100208DF800000122694694
:107350000D2001F01FFC002008BD08B503F0070058
:10736000012809D102F046FF30B103208DF800005A
:107370000122694601F00EFC002008BD08B503F0AB
:10738000070001280AD102F035FF38B10B208DF833
:10739000000001226946032001F0FCFB002008BD2B
:1073A00008B503F0070001280AD102F023FF38B125
:1073B00001208DF8000002466946032001F0EAFB37
:1073C000002008BD1FB513F0070F0ED102F012FF09
:1073D00058B19DF80800F02813D002F00BFF20B13F
:1073E000012202A9092001F0D5FB07E0FC2B0100D6
:1073F0000401011054464953EFBEADDE04B0002035
:1074000010BDFEF7CBFAF0E71FB513F0070F07D159
:1074100002F0F0FE20B1012202A9042001F0BAFB23
:1074200004B0002010BD10B503F00700012808BF0C
:1074300002F01AFA002010BD10B503F0070CF94C49
:10744000BCF1010F06D013F0070F09D0BCF1020FF9
:1074500018D015E00020E06004F0FFFAE0610FE0D2
:10746000E068002804BF1002E06106D0012804D1C2
:10747000E0691043E06104F0E9FAE068401CE06074
:10748000002010BDE26812B1012A04D007E0A18BF0
:10749000090A017003E0237F037001200870501C6B
:1074A000E060012010BD70B5064603F00700DD4C1A
:1074B0000D46012808BF00200DD013F0070F02D0A1
:1074C00002280BD008E0E068002804BF104608F04E
:1074D00095FFE068401CE060002070BD08F093FF5D
:1074E00030700120287070BD2DE9F047064603F08A
:1074F0000700CC4F8946012808D0DFF82C83CB4DFC
:1075000013F0070F06D0022839D035E00020F860CC
:10751000386131E0F868002808BF7A7029D0012866
:1075200004BF1002F86124D0022822D1F869104368
:10753000F8617E7884B202F05DFED0B1062E18D2DA
:10754000DFE806F00306090C1014A8F80E4010E05E
:10755000A8F80C400DE0286884860AE02868A0F8A6
:107560000C4106E02868A0F8504002E02868A0F826
:107570005240F868401CF8600020BDE8F087386988
:1075800002282CD297F801A0002402F033FED8B1D3
:10759000BAF1060F18D2DFE80AF00306090C10143E
:1075A000B8F80E4010E0B8F80C400DE02868848E62
:1075B0000AE02868B0F80C4106E02868B0F85040AE
:1075C00002E02868B0F852403869002804BF200A59
:1075D000307004D0012802D1347089F80000386975
:1075E000401C38610120BDE8F0872DE9F0411C46C0
:1075F00015460E46074602F0FDFD80B18A4814F09C
:10760000070F04D004F0070102290BD007E0002D7A
:107610001ABF90F86C00C008002008F0F9FE0020A6
:10762000BDE8F08190F86C00C0083870012030701F
:10763000BDE8F08170B503F0070200267C4C794D5F
:10764000012A02D0022A15D012E004F081FD21683F
:107650000870FDF70FFF2168487002F02FFB2168CA
:107660008870FDF70AFF2168C87005202870EE6059
:10767000002070BD2A78052A10D1EA68042A28BFA4
:10768000104604D223689B5C0370501CE8600428F9
:1076900004D10120EE60087003202870012070BD25
:1076A00070B503F00702624C00255E4E012A02D03D
:1076B000022A42D03FE0FEF74FF9002828D0416966
:1076C000FF292CBFFF21C9B2226811708169FF29EF
:1076D00034BFC9B2FF2122685170C169FF2934BF8C
:1076E000C9B2FF21226891702268017CD1702268A2
:1076F00090F820101171018C2268090A5171016AF9
:107700002268090C9171006A2168000EC87111E0AD
:1077100020680570206845702068857021685020B9
:10772000C8702168FF20087121684871216888713C
:107730002168C871F560002070BDF268082A28BF72
:10774000104604D223689B5C0370501CF06008282C
:1077500002D10120F5600870012070BD70B503F002
:107760000701304D0646012904BF0020686301D09F
:10777000022901D0002070BD95F8340010F00704F4
:1077800004BF2C4808F049FE2A48005D3070686B41
:10779000401C6863012070BD10B5044603F007006B
:1077A00002281CBF002010BD08F03CFE2070012004
:1077B00010BD70B503F0070200251A4C012A02D053
:1077C000022A11D00EE00520207000210846E56055
:1077D00001F08DFC4FF6FF7101EA4000606101F09D
:1077E00092FCA062002070BD2278052A17D1D4F83F
:1077F00014C0E268624528BF104607D212F0010F9C
:107800001CBF6378037017D0501CE060604506D140
:107810000120E56008700320207001F080FC012049
:1078200070BD000004010110BC7B0110DC010110DF
:10783000FC2B010040010110A66A22F00103F35A5B
:107840001E0A06706370DFE770B503F007020025BB
:10785000F74C012A02D0022A0AD007E00520207046
:10786000D020E560606101F0C5FDA062002070BD20
:107870002278052A17D1D4F814C0E268624528BFDF
:10788000104607D212F0010F1CBF637803700CD0B2
:10789000501CE060604506D10120E56008700320BF
:1078A000207001F0B5FD012070BDA66A22F0010331
:1078B000F35A1E0A06706370EAE77FB51C460E464F
:1078C000054613F0070F08D102F094FC28B10122FD
:1078D00002A90C2001F05EF903E004F00700022881
:1078E00002D004B0002070BD04F032FC28700120EA
:1078F000307004B070BD10B503F00702CC4C012A03
:1079000002D0022A0DD00AE002F069FE00212062B6
:1079100000281ABF4FF4056060626162E1600020D8
:1079200010BD636AE2689A4228BF104607D2D4F8B5
:1079300020C01CF802C080F800C0501CE0609842D3
:1079400004BF01200870012010BD10B4DFF8E4C2AC
:1079500013F0070F04D003F00702022A18D014E036
:10796000012A01D04AB110E0DCF800004069DCF8DF
:10797000001040F00100486107E0DCF800004069B9
:10798000DCF8001020F00100486110BC00207047B6
:10799000DCF80020526902F0010202700120087038
:1079A00010BC704770B514460E46054613F0070F1D
:1079B00004D003F00700022814D011E0002C14BFFB
:1079C0000120002001F042FF54B19A480168096B80
:1079D000006821F4405141F4BE0141F020410163AF
:1079E000002070BD01F039FF002814BF01220022E1
:1079F0002A700120307070BD70B503F007008C4D07
:107A00001446012808BF002017D013F0070F15D126
:107A1000E868002808BF6A700DD001280BD168788B
:107A2000FBF7D8FA844968780B6800EA04021A6305
:107A30000968A0434863E868401CE860002070BD06
:107A400070B50D46044613F0070F04D003F007008D
:107A5000022805D002E0104604F005FB002070BDAE
:107A600004F004FB20700120287070BD70B50D4635
:107A7000044613F0070F04D003F00700022805D0D6
:107A800002E01046F9F7F4F8002070BDF9F7F3F8BA
:107A900020700120287070BD70B503F0070C644D94
:107AA0000E460446BCF1010F04BF0020E86015D06B
:107AB00013F0070F03D0BCF1020F11D00EE0E868FD
:107AC0005E4902283CBF0B681A54401CE86002283B
:107AD00004D102220968102001F05CF8002070BD7A
:107AE00005F059FBEA68002A04BF000A207004D0A0
:107AF000012A02D1207001203070501CE860012062
:107B000070BD70B503F0070C494D0E460446BCF13C
:107B1000010F04BF0020E86015D013F0070F03D059
:107B2000BCF1020F11D00EE0E868444902283CBFC6
:107B30000B681A54401CE860022804D1022209682C
:107B4000112001F027F8002070BD05F032FBEA6833
:107B5000002A04BF000A207004D0012A02D120703C
:107B600001203070501CE860012070BD70B503F03A
:107B7000070C2F4D0E460446BCF1010F04BF002038
:107B8000E86015D013F0070F03D0BCF1020F11D03D
:107B90000EE0E868294902283CBF0B681A54401CD3
:107BA000E860022804D102220968122000F0F2FFE6
:107BB000002070BDEA6812B1012A05D009E005F085
:107BC00018FB000A207004E005F013FB2070012070
:107BD0003070E868401CE860012070BD70B503F0AB
:107BE000070C134D0E460446BCF1010F04BF0020E4
:107BF000E86015D013F0070F03D0BCF1020F11D0CD
:107C00000EE0E8680D4902283CBF0B681A54401C7E
:107C1000E860022804D102220968132000F0BAFFAC
:107C2000002070BDEA685AB1012A0ED012E00000AF
:107C300004010110DC2B0100D42B0100FC2B0100FE
:107C400005F0CBFA000A207004E005F0C6FA2070B7
:107C500001203070E868401CE860012070BD10B55C
:107C600003F00702F84C012A02D0022A27D024E0B0
:107C700002F0B5FC0023002804BF236263621BD01E
:107C800000F1500121624168B1F5887F90F8201021
:107C90000CD390F8212001EB020C01FB02C190F8FB
:107CA000222090F823001044084404E090F82200B9
:107CB0000A1801FB00206062E360002010BD636AC7
:107CC000E2689A4228BF104607D2D4F820C01CF8B8
:107CD00002C080F800C0501CE060984204BF012040
:107CE0000870012010BD10B513F0070F04D003F089
:107CF0000702022A05D002E0104601F01DFA00201A
:107D000010BDD24A127802700120087010BD10B563
:107D100013F0070F04D003F00702022A05D002E097
:107D2000104601F082FB002010BDC94A1278027093
:107D30000120087010BD1FB513F0070F07D102F026
:107D400059FA20B1012202A90B2000F023FF04B050
:107D5000002010BD70B503F00700BB4C154601288C
:107D600004BF0020E06027D013F0070F24D102F0F9
:107D700041FA08B3E068B74E03283CBF31680D54A0
:107D8000401CE060032817D1F9F71DFF3068B0F8F8
:107D9000010045BAF9F728FE040018BFFAF787F882
:107DA00030680078002818BF01202946F9F7D0FA7A
:107DB000002C18BFFAF77EF8002070BD70B503F0F4
:107DC0000700A14C1646012804BF0020E0602BD01C
:107DD00013F0070F28D102F00DFA28B3E0689D4D8B
:107DE00002283CBF29680E54401CE06002281BD1C9
:107DF000F9F7E9FEF9F7F8FD040018BFFAF757F8AC
:107E00002868007800282868417808BF002005D03D
:107E10000120F9F714FB286841781120F9F70FFBCE
:107E2000002C18BFFAF746F8002070BD7FB51C463D
:107E30000E46054613F0070F08D102F0DBF928B112
:107E4000012202A9142000F0A5FE03E004F00700BF
:107E5000022802D004B0002070BD04F03CF90028D4
:107E600014BF012200222A700120307004B070BDBE
:107E70007FB51C460E46054613F0070F08D102F0E9
:107E8000B9F928B1012202A9152000F083FE03E010
:107E900004F00700022802D004B0002070BD04F0F6
:107EA0000BF928700120307004B070BD70B503F07C
:107EB0000700654C1546012804BF0020E06019D07A
:107EC00013F0070F16D102F095F998B1E0686149F7
:107ED00003283CBF0A681554401CE060032809D100
:107EE00008680968B0F80100097840BA00B219B111
:107EF000FEF7BDFC002070BDFEF7B6FCFAE770B5DA
:107F000003F00700504C1546012804BF0020E06034
:107F100017D013F0070F14D102F06CF988B1E068A4
:107F20004C4B03283CBF19680D54401CE0600328EB
:107F300007D11868B0F8010041BA18680078FAF75C
:107F400031FB002070BD10B503F007023E4C012A42
:107F500002D0022A07D004E00020E060FBF76DFCAD
:107F6000E061002010BDE268042A07D2C2F10303D9
:107F7000D4F81CC0DB002CFA03F30370501CE06043
:107F8000042804BF01200870012010BD7FB51C46E5
:107F90000E46054613F0070F0DD102F02BF950B134
:107FA0009DF8080010F0010F09D0012202A9162047
:107FB00000F0F0FD03E004F00700022802D004B056
:107FC000002070BD04F034F928700120307004B036
:107FD00070BD2DE9F0411C4617460E46054613F0CC
:107FE000070F06D102F006F918B1384608F01FFA5B
:107FF00003E004F00700022802D00020BDE8F08171
:1080000008F0D4F9287001203070BDE8F0812DE926
:10801000F0411C4617460E46054613F0070F1BD1CC
:1080200002F0E8F8C0B108F007FA0446384608F054
:1080300008FA012F14D1012C12D000221146012080
:1080400000F0A8FD0CE00000040101105101011036
:1080500056010110FC2B010004F00700022802D099
:108060000020BDE8F08108F0E7F9287001203070A9
:10807000BDE8F0812DE9F0411D4614460F46064645
:1080800013F0070F11D102F0B5F870B103F0DBFF68
:108090000546204603F0D4FFA5420AD04CB9002281
:1080A0001146022000F076FD03E005F007000228EB
:1080B00002D00020BDE8F08103F0C5FF3070012040
:1080C0003870BDE8F081002070477FB51C460D4632
:1080D000064613F0070F08D102F08CF828B10122F0
:1080E00002A9082000F056FD03E004F00700022872
:1080F00002D004B0002070BDFDF7BCF9022808BF13
:1081000000200BD0032808BF022007D0042808BF96
:10811000032003D0052814BFFF2001203070012068
:10812000287004B070BD2DE9F0411C4617460E467C
:10813000054613F0070F0BD102F05CF840B138464A
:1081400003F084FF00221146012000F023FD03E02C
:1081500004F00700022802D00020BDE8F08103F0FF
:1081600078FF287001203070BDE8F08110B510460E
:1081700013F0070F08BF03F0CDFF002010BD10B5AE
:10818000104613F0070F08BF03F0D0FF002010BD0A
:1081900070B5044603F007000D4602281CBF0020FE
:1081A00070BD03F0D0FF20700120287070BD03F077
:1081B000070230B4FB4B4FF0000C012A05D0022A15
:1081C00004BF1A78022A0BD01EE002201870F6486D
:1081D000C3F80CC06FF07F410068081AD86113E043
:1081E000DA68042A28BF104606D2DD69D40025FAD1
:1081F00004F40470501CD860042805D10120C3F891
:108200000CC008700320187030BC0120704713F0B8
:10821000070F04BFE54802700020704710B503F057
:108220000700E049012804BF0020C86013D013F004
:10823000070F10D1C868DE4B04283CBFD3F800C03C
:108240000CF80020401CC860042804D104220F2030
:10825000196800F09FFC002010BD2DE9F04716467C
:1082600003F007020024CF4F012A04BFFC603C61E9
:1082700064D0DFF8408313F0070F07D0022A33D011
:10828000042A04BF387806284FD058E0FD68002D36
:1082900008BF3E6225D0012D06D0D7F81490AC1E41
:1082A0004C4516D284B908E0701C7861396A0844DC
:1082B000B0F5807F88BF7C6113E04FF480724FF48B
:1082C0002A31BD4808F036F8B949386A09682044AF
:1082D0000E54601C484504D1B748C0F8FC80062005
:1082E0003870681CF8602AE0FF2202707B69CBB10D
:1082F000D7F820C03A699444BCF5807F10D2AF4DC6
:108300002D68454518BF047005D10CF5283C9CF834
:1083100000C880F800C0501C984204BF01200870BB
:10832000501C38610120BDE8F0874FF42A30FAF77D
:10833000CDFCA1494FF42A30FAF775FD3C700020BE
:10834000BDE8F08770B503F00700964C154601288C
:1083500004BF0020E06014D013F0070F11D101F02A
:1083600049FF70B1E068924902283CBF0A68155481
:10837000401CE060022804D102220968052000F0B8
:1083800009FC002070BD70B50D46044613F0070FC0
:1083900004D003F00700022805D002E0104603F0E5
:1083A00043FE002070BD03F042FE207001202870C3
:1083B00070BD1FB513F0070F04D1012202A91720C9
:1083C00000F0E8FB04B0002010BD03F00700754981
:1083D000012806D013F0070F04BF0878012806D043
:1083E00014E0012008700020C86088610DE0C868B2
:1083F000042805D28B69401C42EA03228A61C860C6
:10840000042803D10320087088690862002070479F
:1084100003F00700DFF88CC1012807D013F0070F25
:1084200004BF9CF80000022809D01EE002208CF84E
:1084300000000020CCF80C00CCF81C0015E0DCF8A3
:108440000C00022808D2DCF81C10401C42EA012172
:10845000CCF81C10CCF80C00022806D1DCF81C006B
:10846000CCF8240003208CF800000020704770B482
:1084700003F0070200254B4C012A02D0022A06D045
:1084800002E002202070E56070BC00207047227876
:10849000022A1CD1D4F824C0E268624528BF1046E5
:1084A0000ED212F0030F04D1236A53F8046BC4E90F
:1084B0000763237F0370E069000AE061501CE060FD
:1084C000604504D10120E56008700320207070BC75
:1084D0000120704770B503F007000025314C0E46AF
:1084E000012806D013F0070F04BF2078022805D01A
:1084F0002BE002202070E560E56126E0616AE0681B
:10850000884219D2E169090A41EA0262401CE2612B
:1085100010F0030FE0600FD1206AB0F5303F28BFA4
:10852000026006D2B0F5005F03D304222449FAF7B3
:10853000DFFC206A001D2062616AE068884204D185
:108540000120E560307003202070002070BD30B441
:1085500003F007040025DFF84CC0012C08BFCCF85D
:108560000C5047D013F0070F02D0022C45D041E049
:10857000042A08BF4FF42C303AD025DC002A08BF6B
:108580004FF4005034D0012A08BF4FF42F302FD0C1
:10859000022A08BF4FF410302AD0032A08BF094826
:1085A00026D022E0040101108C00011025000110EA
:1085B000FC2B0100554E564D842F0110FCA80200E3
:1085C0002001011000AF0200052A08BF4FF42A3035
:1085D0000ED0F748102A00680AD0112A08BFF548C3
:1085E00006D0202A08BFB43002D0CCF8185001E0E1
:1085F000CCF8180030BC00207047DCF80C20042AAE
:1086000007D2C2F10303DCF81840DB0024FA03F3BD
:108610000370501CCCF80C00042824BF0120087003
:10862000012030BC704770B403F0070CE24DBCF180
:10863000010F07D0E14C13F0070F07D0BCF1020F78
:1086400021D01DE00020E860286119E0E8680528D5
:108650003CBF21680A54042810D123682268D4F84A
:1086600000C0D3F80130A96912781BBA9CF804C085
:1086700023F0FF0343EA0C0341F82230401CE8607A
:1086800070BC002070472B6973B1042B07D222689D
:10869000032B1A445278027004BF01200870581C42
:1086A000286170BC012070472268D5F818C0127884
:1086B0005CF8222026684FEA126C86F801C0266812
:1086C0004FEA124C86F802C026684FEA122C86F850
:1086D00003C0D4F800C08CF80420D8E710B503F02C
:1086E0000700012804D1002211460E2000F052FAA2
:1086F000002010BD2DE9F04103F00704AE4E1746EF
:1087000088460546012C04BF0020F06017D013F006
:10871000070F12D101F06EFD78B1F068A749022869
:108720003CBF0A681754401CF060022807D102229F
:108730000968072000F02EFA01E0022C02D0002088
:10874000BDE8F081F26812B1012A04D009E0FCF71B
:1087500091FE287005E0FCF790FE2870012088F853
:108760000000F068401CF0600120BDE8F08170B5A9
:1087700003F007000025904C012808D013F0070FE4
:108780000BD0042804BF2078062825D02DE0A56151
:10879000E5616570E560257027E0E068022807D292
:1087A000A16942EA0121A16161781144617010E080
:1087B000042807D2E16942EA0121E16161781144AC
:1087C000617006E0052804D261788A4204BF062160
:1087D0002170401CE06008E0D4E9060101F094F843
:1087E000002804BF0120A0702570002070BD10B5C6
:1087F000714C13F0070F07D003F00700042804BFE3
:10880000207806281FD028E0E068022807D2A16956
:1088100042EA0121A16161781144617010E0B0F574
:10882000817F08D265490968014401F8022C61780A
:108830001144617004E001BF61788A420621217011
:10884000401CE06009E05E49A06901F07FF8002863
:1088500004BF0120A07000202070002010BD03F094
:10886000070CBCF1010F00D0C1E75349002088611B
:108870004870C8600870704730B403F007050024E2
:10888000DFF834C1012D07D013F0070F0DD0022DF2
:108890003CD0042D54D06FE0CCF81840CCF81C40EC
:1088A000CCF80C408CF8004066E0DCF80C000228A4
:1088B0000BD2DCF8181042EA0121CCF818109CF811
:1088C000011011448CF8011019E0042817D2DCF8CB
:1088D0001C10032842EA0121CCF81C109CF801303E
:1088E0001A448CF801200AD106228CF80020DCF80A
:1088F0001820114304BF4FF43071CCF81C103149DB
:10890000401CCCF83010CCF80C0035E0DCF80C2022
:10891000042A28BF10460AD2C2F10303DCF8305003
:10892000DB0025FA03F30370501CCCF80C0004287C
:1089300003D10120CCF80C40087030BC01207047F6
:108940009CF80000062815D1DCF81800002201026E
:10895000DCF81C0003021046B2EB930F06D251F86C
:10896000045B401C2A44B0EB930FF8D3CCF83020C2
:108970008CF80040CCF80C4030BC002070472DE94A
:10898000F04103F00700DFF834C000250A4E01284B
:108990001AD013F0070F4FF001071ED0042801BFB3
:1089A0003078062800244FF4103836D032E000002A
:1089B000DC010110BC7B011004010110FC2B010043
:1089C000842F0110EFBEADDEF560DCF8000005700D
:1089D000DCF80000457035701CE0F068022804D215
:1089E000DCF800301A54401CF060022812D159A063
:1089F0000068F5600F70DCF80010C2B2097891428F
:108A000008D1DCF80010C0F307204978814204BF88
:108A1000062030700020BDE8F08108EB0430FAF742
:108A2000B1F9022804D0601CC4B2062CF5D3384634
:108A3000012807BFB7717571B770B5713570E9E777
:108A400003F00702022A1CBF00207047424A9279B5
:108A500002700120087070472DE9F041002103F0F9
:108A600007003E4E3C4D0C46012803D013F0070F83
:108A70000CD06CE0EC702C81EC622C71002046F87C
:108A80002040401CC0B24028F9D360E0E8780528B7
:108A90003CBF401CE870C0B2012808BF100220D0C3
:108AA000022804BF688910441BD050D92889B5F822
:108AB0000AC084454BD92A4B00F00307DA55471CFE
:108AC0004FF41032674508BF00200CD1401CC0B2E3
:108AD0000428FBD3E86A214902EB0020FAF7A3F946
:108AE0002CE0688133E04FF0030C3CEA000025D114
:108AF00013F800C0C7000CFA07FC401CC0B24CEAD7
:108B000001010428F4D3287900F03F03401CC0B2CF
:108B100046F823102871402810D1E86A0F4902EB6B
:108B20000020FAF780F92C71E86A401CE862002006
:108B300046F82040401CC0B24028F9D32889401C88
:108B400080B228816989884204BF012068710020B1
:108B5000BDE8F08155AC000004010110842F011024
:108B60003C010110F94800220270427082700271CB
:108B70004271C270DFF8D8C3114601EB41030020F7
:108B80000CEB43031A54401C0628FBD3491C08294C
:108B9000F3D3704707F05ABC2DE9F04115460E4655
:108BA0000746FAF758FD00F008040820FAF74EFDD2
:108BB0002A463146384607F049FC05462046FAF772
:108BC00041FD2846BDE8F081E04880787047DF48E5
:108BD00040787047DD49002048707047DB49062027
:108BE0008871704770B50026F9F7ECF8044610F06C
:108BF0000F051AD02846F9F7E8F8012D17D0FCF731
:108C00003CFC44EA006422461421022002F02BFFBF
:108C100014F0060F09D00126FCF72CFC044603F0E3
:108C20006AFA022C08BFFBF719FE304670BDFCF74C
:108C300021FCC6498A79904218BF8871DFD1E7E7E5
:108C40002DE9F04F83B00026FBF745FAFCF712FC44
:108C5000022804D101F09AFA002818BF0126FFF774
:108C6000C1FF002818BF0126DFF8E08298F8020053
:108C7000002800F0EF81E9464FF0FF34FAF7EBFCF3
:108C800000F0080A0820FAF7E1FC98F80300002534
:108C900008B398F80500AE4900EB4002401CC0B292
:108CA00001EB420188F80500082828BF88F8055024
:108CB00098F80300401E88F803004C780F780020D5
:108CC000002C06DD0A18927809F80020401C844226
:108CD000F8DC0D704D705046FAF7B4FC002CC0F271
:108CE000A981F8B20024182880F06C81DFE800F038
:108CF000962E0C1823310F3EFC45967C8287C7FBCD
:108D0000FAF9F8F797A6AEB3FBF7A8FD1EE09DF8B9
:108D10000000AC280CBF01200220FCF76CFC15E021
:108D20009DF800100120FCF7B7FB012088F8010036
:108D3000044600F047B99DF8000001F04DFC012108
:108D40000320FCF7A9FB012088F80100012400F0B2
:108D500039B9BDF8000040BA03F06CF902210320D4
:108D6000FCF79AFB012088F80100EFE79DF801105D
:108D70009DF80000FCF790FBE8E74FF0010A88F847
:108D800001A098F8000060BBF9F705F848B39DF81A
:108D9000009088F800A019F0040F18BFFDF7AFFD90
:108DA00019F0020F07D0FF210F20FCF702FEFBF79E
:108DB0003AFE49F0010919F0010F10D0FCF75AFBF7
:108DC000022802D103F097F948B1FCF753FB0528BC
:108DD00002D100F0F6FD10B10020FBF713FE88F879
:108DE000005088F80150EDE09DF80000401E01F0B1
:108DF0000BF8ABE79DF8000003F0AFF9A6E79DF88C
:108E00000000002871D0FCF735FB022818BF0124B0
:108E100003F07AF901460220FCF73EFBD2E09DF810
:108E20000000002818BF012003F04BF99DF8000056
:108E3000002818BF012000F0AFFDC3E09DF800003E
:108E4000002818BF012003F01EF9BBE09DF80000C8
:108E500003F09CF97AE79DF8000020B1012873D057
:108E6000022805D0AEE04FF42F30F9F72FFFA9E02C
:108E700001F003FA00210420FCF70EFB66E7FAF785
:108E8000EAFB00F008090820FAF7E0FB98F8030075
:108E9000002808BF88F802504846FAF7D3FB4FF085
:108EA000000AD14672B6FAF7B8FE48B1FAF78FFF5A
:108EB0008246FAF76CFFFAF790FF8146FAF777FFE0
:108EC000F8F781FEF8F790FD0190F8F702FFFAF746
:108ED0006DFC5FEA000B18BFFAF74CFC06E06CE093
:108EE00065E05EE057E04CE038E047E04FF4935037
:108EF000FAF7B5FB62B61748056017480168D1F864
:108F0000CC10006841F4BE0141F02041C0F8C81007
:108F100007F05BFA72B6019818B1F8F754FEF8F74B
:108F200062FFFAF77AFE48B1BAF1000F18BFFAF7FC
:108F30007AFEB9F1000F18BFFAF7C1FEBBF1000FBE
:108F400018BFFAF7D2FB62B63CE0000048010110FE
:108F5000843001105C000110E42B01009DF800003A
:108F6000012804BF0421052086D0022806D003284A
:108F700007BF00210420022108467DE700210320CD
:108F80007AE79DF80300009A1E2160F31F6201201A
:108F900002F069FD16E0BDF8000040BA04F001F9E6
:108FA00010E0BDF8000040BA04F009F90AE0BDF88D
:108FB000000040BA04F020F904E0BDF8000040BA17
:108FC00004F00EF90CB1012634E0E9464FF0FF340D
:108FD000FAF741FB00F0080A0820FAF737FB98F887
:108FE000030008B398F805001E4900EB4002401C3E
:108FF000C0B201EB420188F80500082828BF88F8B4
:10900000055098F80300401E88F803004C780F784C
:109010000020002C06DD0A18927809F80020401C78
:109020008442F8DC0D704D705046FAF70BFB002CB3
:10903000BFF657AEFAF70FFB00F008040820FAF766
:1090400005FB98F80310002908BF88F80250204655
:10905000FAF7F8FA002E14BF0120002003B0BDE893
:10906000F08F00008430011002460020022928BF42
:10907000704752B1012A18BF704701EB810000EB25
:10908000C100F74901EB0010704701EB0110F549F1
:1090900001EBC010704770B5FAF7DDFA00F0080672
:1090A0000820FAF7D3FAF04C00256078302806D271
:1090B0004FF48851EB4807F042F9A570E570A079AC
:1090C000302806D24FF4D071E54807F038F9E57141
:1090D00025723046BDE87040FAF7B4BA00FB01F2E1
:1090E000B2F5886F9CBFE04AC2E9030170470028CF
:1090F000DD4AD26818BF0260DB480029006918BF4A
:10910000086050437047D848012101710078D54963
:1091100080F0010000EB001001EBC0107047D24856
:109120008278002132B1C27822B9027882F001023D
:109130000270817001717047CB491E284A784870CF
:1091400008BF002003D01F2808BF012000D10870ED
:1091500010467047C4480078C24980F0010000EB17
:10916000001001EBC0107047F0B4BF4E96F800C07D
:10917000BC4CF5680CEB0C1C04EBCC1C03FB05F49D
:109180000CEB440C8D4234BF2C460C463669F31A66
:10919000934238BF1A460026002A9CBFF0BC704795
:1091A0000023002C06D930F813702CF813705B1CC8
:1091B0009C42F8D8761C0CEB450C00EB4100964223
:1091C000EED3F0BC70472DE9F041A74F14468C4612
:1091D00001467A7806981D468A4218BFBDE8F0819C
:1091E0000121F970012802D0022823D028E0387824
:1091F0009C49FE6800EB001001EBC011A64234BF91
:10920000324622463869A84238BF05460023002D61
:1092100016D90020002A06D91CF8007021F8107019
:10922000401C8242F8D85B1C01EB4601A444AB42CF
:10923000EFD305E000232A4621466046FFF794FF5E
:10924000BDE8F04100F08EBA002808BF704786499B
:10925000864B4A7886491B78002A097818BF022A6B
:1092600005D0042A18BF092A01D001227CE7814ACF
:109270001278012A84BF804A1378012200F08CBA48
:109280002DE9F04F784C83B00121E1707B49794D95
:10929000794E0F78754991F800A06178112932D084
:1092A0000EDC002918BF02291ED0042918BF092985
:1092B0001AD0A0B1002352463946FFF755FF0EE001
:1092C000122918BF13291ED0212918BF2229F0D135
:1092D00028B100230AF102023946FFF745FF03B027
:1092E000BDE8F04F00F03EBA2978012903D964495E
:1092F00096F800A00F780028F1D000235246394696
:1093000000F04AFAEBE7F8F75EFCF8F76DFB009027
:10931000002818BFF8F7CBFD2878012888BF96F8F9
:1093200000A0F8F740FD10F0040F18BF0AF1010A81
:109330005448006800F5804001906078A0F1110960
:109340002078484900EB001001EBC015E068B842F6
:1093500038BF07462069504538BF8246F8F7E4FD1C
:1093600083460020F9F7A0F90026BAF1000F34DD9A
:109370000024002FC4BF019800EB861826DD1BF9DE
:109380000400202824BF002025F814001BD200EB85
:10939000D0714910C00758F82110C00E21FA00F012
:1093A00081B24FF0FF30B9F1000F1CD0B9F1010FBD
:1093B00008BFC8B205D0B9F1020F04BF0846F9F7DB
:1093C00079F925F81400641CBC42D8DB2648761CC9
:1093D0005645C06805EB4005CADB0098002818BF59
:1093E000F8F768FD7BE711F4005FC1F3042018BFB4
:1093F0004042E6E71C4801214172407980F00100BB
:1094000000EB800101EBC000154901EB0010704733
:109410001548C279002132B1027A22B9427982F02C
:1094200001024271C171417270470F491E288A7949
:10943000887108BF002003D01F2808BF012000D179
:109440004871104670470848407980F0010000EBF1
:10945000800101EBC000024901EB001070470000E1
:10946000B4410110B430011050010110CB000110C3
:10947000D1000110CC000110CE000110CA00011073
:10948000CD000110F82B01002DE9F04FE44985B023
:10949000012291F80080E34991F80090E2490A72B4
:1094A0008979E24C11291CBF1229132938D008B33D
:1094B000DD49497901EB810202EBC10104EB0112A4
:1094C0000021B9F1000F06D930F8113022F811301F
:1094D000491C8945F8D80021B8F1000F0AD909EBD9
:1094E000010302EB410C30F81330491CACF8683032
:1094F0008845F4D8FAF7AFF800F008050820FAF725
:10950000A5F8C94C607A002818BF01217ED0E1710E
:109510002846FAF797F80020207205B0BDE8F08FD2
:10952000F8F751FBF8F760FA0190002818BFF8F738
:10953000BEFCBD488179A1F11106416900914079D5
:1095400000EB800101EBC00004EB0015F7F799FB7D
:10955000B7494FF0110B0028096801F5804101F56A
:109560000C6701F5046104BF8A46012004D0BA46A5
:1095700058460F464FF0010BF9F796F8F8F7D2FC72
:1095800000240390B9F1000F29D9009880010290BE
:1095900003980057202824BF002025F814001BD270
:1095A00000EBD0720299521001EB8201C00751F812
:1095B0000A10C00E21FA00F081B24FF0FF30002EE9
:1095C0004AD0012E08BFC8B204D0022E04BF0846FC
:1095D000F9F770F825F81400641C4C45D8D35846A8
:1095E000F9F762F8F8F7A0FC00248246B8F1000F02
:1095F0002CD90098A3464FEA80191AF904002028B4
:1096000024BF05EB4400A0F868B000E032E01AD2B5
:1096100000EBD071491009EB8101C007C959C00E98
:1096200021FA00F081B24FF0FF30E6B1012E08BF01
:10963000C8B204D0022E04BF0846F9F73BF805EB88
:109640004401A1F86800641C4445D6D30198002861
:1096500018BFF8F72FFC4DE711F4005FC1F30420A9
:1096600018BF4042B6E711F4005FC1F3042018BFF1
:109670004042E4E7607980F001006071002146E734
:1096800070B50D4668490122CA706A4A4978167851
:10969000694A212914781EBF2229232970BD002878
:1096A00018BF002D11D0002322463146FFF75CFD84
:1096B000631C012221462846FFF756FD05EB4400B6
:1096C000A31C01223146FFF74FFDBDE8704000F0BA
:1096D00049B870B5544D0446687890B9E06868B1EF
:1096E00056490978012994BF534955490B78554982
:1096F0000122097800F050F8687810B9A068FFF7E7
:10970000BFFD6878112804BF0020FFF7B9FD687815
:10971000122804BF0020FFF7B3FD6878132804BFA8
:109720000020FFF7ADFD206910B1A97921B105E056
:10973000606918B1A97909B9FFF7A6FEA8791128BF
:1097400004BF0020FFF7A0FEA879122804BF002064
:10975000FFF79AFEA879132818BF70BD0020BDE856
:10976000704091E670B5F9F776FF00F00806082022
:10977000F9F76CFF2C4C20790025002801BF2078D8
:1097800080F001002070A5701CBF0120A070304641
:10979000F9F758FFE57070BD2DE9F0479946164678
:1097A0000D460446F8F7C5FB5FEA000C1BD01E49C6
:1097B0000878254AD1F80C8000EB001002EBC010AD
:1097C00009FB08F200EB4200454594BF2F4647468F
:1097D0000969A1EB0901B14238BF0E460021002EF4
:1097E00008D8BDE8F0874B46324629462046BDE8FA
:1097F000F047B9E40023002F08D91CF9032034F8FE
:10980000122020F813205B1C9F42F6D8491C00EB65
:10981000480004EB4504B142ECD3BDE8F0870000FA
:10982000CF000110D000011050010110B44101100F
:10983000F82B0100CA000110CB000110CC00011070
:10984000CE000110D1000110B43001102B490028C6
:1098500014BF0020012008707047284800780028B5
:109860000CBF0120002070472448017899B1244999
:109870000A6852690B6842F001025A610A689269EB
:1098800012F0010F07D00A68126B1E4B096822F410
:1098900040521A430A63002141608160C160016146
:1098A00041617047E0E700B50178C27983B01143A8
:1098B00041F040018DF8001041788DF80110418889
:1098C00009098DF80210818809098DF80310817843
:1098D00001F00F02017962F31F118DF804108179F4
:1098E0008DF80510017A8DF80610407A8DF8070082
:1098F000684606F0B0FD03B000BD0000680101102D
:10990000DC2B010000205FA070B50E460446FBF77B
:10991000B1FD042811D1A4F5107080280DD2A01932
:10992000A0F24120802808D225020024002E04D96C
:109930002846F9F7CBF9012801D0002070BD641C3E
:1099400005F58075B442F3D3012070BD70B50D46A6
:109950000446FBF78FFD04280AD1A4F51070802877
:1099600006D220022946F9F75EFA012808BF70BD29
:10997000002070BD10B5074CFFF762F9012808BF41
:1099800010BD206800F01CFD002818BFFBF7C4FDC7
:10999000F2E70000DC010110B14A0028516814BF51
:1099A00041F0010021F0010050607047AC4B596854
:1099B0000A0E120721F07F4142EA00600843586016
:1099C0007047A7484068C0F303607047A4484068E8
:1099D000000F7047A24800697047A1490120086143
:1099E00070479F490020086170472DE9F043AFB0F0
:1099F000002706F035FD0646A02102A806F09FFCD0
:109A0000002425464FF003084FF00109305D10F0A7
:109A1000800F17D0601CC1B28DF8A9108DF8AF501F
:109A20008DF8A880ADF8AC50ADF8AA508DF8AE50C6
:109A30003555CDE90091002201272AAB114602A835
:109A4000F6F742FD601CC4B20A2CDFD3012F06D109
:109A5000102302AA06210120009505F071FF06F0EF
:109A600004FD2FB0BDE8F0832DE9F04F7D4F87B0A6
:109A70003868B0F90E11B0F90C0106F0B5FCFAF730
:109A8000EDFE06F0F7FC3868D0F8F800C0F30340AC
:109A9000FAF7CAFEFBF7EEFC052835D1DFF8C8B1AE
:109AA000DFF8C8916E4D4FF00008ABF1070A686807
:109AB000C0F303643868A100D0F8F800C5F8088046
:109AC000C84000F00F0621460520C5F80C8002F0C2
:109AD0004BF8002C7ED0022C1FD0042C7BD0686861
:109AE0000A2C4FEA106120F07F404FEA017118BF45
:109AF00041F0007108436860FFF7A2F8012803D025
:109B0000FBF7B8FC0528D2D006F0AFFCFAF7A5FEAB
:109B100007B0BDE8F04F06F0B2BC0D213046FBF7B0
:109B20009CFD0028E8D006F0AFFC06F0B2FCFAF786
:109B30003CFE06460020F7F7EAFB4D48F7F79DFF8D
:109B40000120F7F78FFFF9F7ADFD4A48F9F75FFEFF
:109B5000F9F744FEF9F771FE41003868B0F80621C4
:109B6000B1FBF2F1491CC1F34F01698090F8080183
:109B7000287050B1F9F761FE39684000B1F804115E
:109B8000B0FBF1F0401CC0F34F010846F9F7D2FDDD
:109B9000D9F80000C0F818B0F8F715F8F8F76BF925
:109BA000287838B1401E10F0FF00287004BF688884
:109BB000F9F7C0FD6868C0F3036421460520F6F795
:109BC0008AFBFFF73DF8012809D06868C0F30360FD
:109BD000A04201E03CE03FE008BF002E1AD0D9F8D7
:109BE0000000C0F818A0F9F7C5FDF9F703FE002042
:109BF000F9F70DFEF9F763FDF7F7E5FFF7F7F6FE66
:109C00000020F7F73AFF06F044FC06F047FCFBF7AC
:109C100090FE71E76846F8F7CBFA70B16846FFF737
:109C200058FD0198FAF7B0FA684606F03CFC064683
:109C3000F8F70DFBFBF791FCC3E73868406E10F0B6
:109C4000704F02D0FBF768FCBBE7FBF78DFCB8E771
:109C5000304606F02DFC4FE7304602F066FC4BE73D
:109C600080010110DC01011007005FA0DC2B010066
:109C700027EB001007E600107047002808BF704768
:109C800080220146014806F055BB7047344401105C
:109C9000704708283CBFFE49087070470020FC4907
:109CA00088604860FB48006890F88100082838BF49
:109CB000087070470020F64948607047F448007803
:109CC000704770B5F34D0024286890F86C0010F0D0
:109CD000020F0BD0FBF7CEFB022807D1EC48296816
:109CE000007801EB8000B0F8840084B2204670BD9B
:109CF00070B5E84D4FF48054286890F86C0010F06F
:109D0000020F0DD0FBF7B6FB022809D1E048296805
:109D1000007801EB8000D0F88400000CC0F313043D
:109D2000204670BDDA488078002818BF01207047AF
:109D30002DE9F041FBF79EFB022803D102F0DBF98D
:109D4000022803D04FF48050BDE8F0814FF48055D5
:109D50002E4602F0FDF9CF4F0446DFF83483386811
:109D600090F86C1011F0010F0ED0B0F87600D8F812
:109D700008104042814207DC34B10020641EC8F85C
:109D80000800204602F0E9F9396891F86C0010F0FB
:109D9000040F18BF002C0AD0B1F87C00621E90405E
:109DA000B1F87E20824238BF1046C0F31306D1F8C6
:109DB000A40010F0020F1CBF98F80210002902D076
:109DC000000CC0F31305B54298BF354602F060FAA7
:109DD000B8B106F0EBFA012803D006F0E7FA08283C
:109DE0000FD1FBF71EFC01463868B0F85800C0F3ED
:109DF000033081421CBF4FF40050B5F5005F38BFFF
:109E000005462846BDE8F0812DE9F04FDFF884A231
:109E100087B0DAF8001091F86C2012F0020F0DD024
:109E20009B4A91F88090DFF870B21778002809DB20
:109E3000484503D2B84218BF06463DD107B00020BE
:109E4000BDE8F08F3E464FF0FF38F7F7CFFDF8F74B
:109E50006DFC0025B9F1000F2ED9DAF800000024BE
:109E600000EB8500B0F8840081B22046F7F770FA65
:109E7000F8F701F86846F8F79BF900285FD00298D8
:109E800078B1014685489BF8002000785043421E77
:109E900007D331F9020B0028B8BF40420444521ED8
:109EA000F7D2F8F7D4F9F7F7A1FDA04584BF2E4605
:109EB000A0466D1C4D45D0D3B74243D0082E3CBFC1
:109EC00073490E70DAF80000B0F8821039B300EB75
:109ED000870200EB8600B2F88420B0F8840092B2CA
:109EE00080B2801A484340F30F34FAF79DF96C4B67
:109EF0009BF80020002193F800C002FB0CF2002A1E
:109F00000DD930F81120224420F811209BF80020B0
:109F100093F800C0491C02FB0CF28A42F1D84FF0C2
:109F2000806002F0DDF9DAF80000022100EB860023
:109F3000B0F8840082B2032001F095FD09E0FBF740
:109F4000EBFA97E702F004F903283CBF401C02F04B
:109F500004F9012007B0BDE8F08F4E484C49006875
:109F6000B0F87600424288688242BCBF401E8860DA
:109F700070472DE9F04F91B093460E4604464FF0DE
:109F8000000A02F0E5F8DFF80C81414F0500D146E8
:109F900010D106F092FAD8F80010B1F87810884283
:109FA00008D30120C7F8089002F0D7F811B00120BB
:109FB000BDE8F08F002E1FDDB8680028B8BFC7F8D5
:109FC000089007DBD8F80010B1F874108842BCBFC5
:109FD000401CB860D8F80000B968B0F87400884236
:109FE00015DC032D13D2681CC7F8089002F0B5F8F1
:109FF00011B00120BDE8F08F09D1D8F80000B0F809
:10A0000076004142B8688842C4BF401EB860B87844
:10A0100050B1D8F8000090F8A40010F0040F1EBF53
:10A02000002011B0BDE8F08FD8F80000B0F9721030
:10A030008C420EDD796821447960B0F86E00884268
:10A0400010DC4FF0FF30C7F80490FFF7DDFE8246CA
:10A0500008E07868002805DD002CD4BF01212146E6
:10A06000401A7860DFF83C9099F8000007283BD14F
:10A070000D48594600784200684606F06AF9ADF886
:10A080000040ADF80260ADF8045038890EE00000E1
:10A09000C8010110DC010110CA000110CE0001103E
:10A0A000CB00011051010110D1000110ADF80600E4
:10A0B000B888ADF80800D8F80000B0F87210ADF814
:10A0C0000A10B0F87410ADF80C10B0F86E10ADF8BE
:10A0D0000E10B0F87600ADF8100099F800000728CF
:10A0E00004BF6846FFF7B0F8504611B0BDE8F08FE6
:10A0F0003D4810B50068D0F8A40010F4807F06D069
:10A10000C0F30330012101FA00F0F8F76AFF374984
:10A1100000204870887010BD70B5344D0024A878B8
:10A12000002814BF01260026687828B902F029F813
:10A13000002808BF002100D001218E4224D00A1C33
:10A1400018BF0122AA7028480068D0F8A43013F084
:10A15000040F0ED021B1C3F30310082808D206E083
:10A160000021A960696090F88100082800D2287059
:10A17000012413F0020F18BF0124002A18BF012286
:10A180000421032001F06FFC204670BD1649002019
:10A190000968D1F8A41011F4807F08BF7047DFF878
:10A1A0004CC09CF80120131C18BF012330B4104C84
:10A1B000C1F303322468E46B012505FA02F2224060
:10A1C00011F4007F01D00AB102E00AB1002100E0E1
:10A1D00001218B4204BF30BC7047081C18BF01200E
:10A1E0008CF8010030BC97E7DC010110C8010110B8
:10A1F000D42B01005F48007870475E48406800F546
:10A20000407070475B48406800F58070704770B5DB
:10A21000584C4FF41032584962601068884204BFAD
:10A220005068B0F5087F26D1D2F808C0BCF5D04FF1
:10A2300021D85249D06888420DD0002311461846D3
:10A24000B3EB9C0F07D251F8045B401C6B40B0EBA2
:10A250009C0FF8D37BB9012502F5807000F0B0F8AF
:10A2600048B1606800F5407000F0B9F800281EBFE2
:10A270002570012070BD002070BD3E49002008708F
:10A280004FF41030F8F722BD3A48017841B14068E8
:10A29000394A0168914202BF4168B1F5087F7047B1
:10A2A00000207047334B5B6803F580731844F8F760
:10A2B0001FBE304B5B6803F540731844F8F718BEB7
:10A2C0002C484068006970472A4949680A698242F7
:10A2D0009CBF00207047C0EBC00001EBC00000F540
:10A2E00080607047234A526802EB80035B6A1A441D
:10A2F000234B53F82000FF3020F0FF0000FB01202B
:10A300007047F0B41B4B00221D4E5C681746831843
:10A3100093F928C0BCF1000FB8BF41F822700DDBE3
:10A32000D3B204EB830556F823306D6AFF3325441E
:10A3300023F0FF0303FB0C5341F82230521C102A78
:10A34000E5D3F0BC704794460029B8BF7047094A6E
:10A35000526802EB80035B6A1344094A52F82020DA
:10A3600002F1FF0020F0FF0001FB00306146F8F72A
:10A37000BFBD0000D401011054465053EFBEADDE06
:10A38000002C010010B5FFF742FFA8B1FFF735FF21
:10A390000146D022174805F0CDFFFFF733FF164CDA
:10A3A00001464FF4C272206805F0C4FF2068406D7A
:10A3B000BDE8104001F05DBE0220FBF71CF9E2E7AA
:10A3C00058B10E4A0168914207D1406820F00F0051
:10A3D000B0F5087F04BF012070470020704730B1FE
:10A3E000006820F00F00602804BF012070470020A3
:10A3F00070470000BC7B0110DC010110415053523A
:10A4000010B572B60120F8F731FBF9F7F7FAF9F752
:10A4100025FB4FF0FF30F9F719F9694880234FF415
:10A420000052002152F821C040F821C0491CB1EB74
:10A43000930FF7D3F9F71CF9F9F706FEF9F730FE99
:10A440000120F9F702FEF8F7D3FB1E20F9F7F0FD23
:10A45000F9F728FBF8F7D4FDF9F7A6FDF9F778FB33
:10A46000F9F71CF9F8F758FEF7F7D3FAFFF78AFF68
:10A47000F9F795F8F9F74EF8FEF774FBFCF78EFB49
:10A48000FFF710FA62B64F4806F01CF84E4C2068F1
:10A49000B0F90C0106F01BF8F5F703FFFFF7F8FB26
:10A4A000F9F734FEFBF77DFA2068418A008AFEF74F
:10A4B00015FE2068806EC0F34E0161F35F0001F06D
:10A4C000C5FAFFF7D9FB06F007F8FBF7BCF82068E0
:10A4D00090F8640000F00F00F8F7B8F9206890F8E1
:10A4E000200010F0010F04BF0021032003D001F071
:10A4F0000BFE01460220FAF7CFFF344800680069DE
:10A500000C2100F07002012001F0ADFAFFF7F0FD20
:10A51000002010BD2E4CFEF793FB012806D0FAF761
:10A52000A9FF032802D101F04AFB08B3002C05DC87
:10A5300001F0EAFD01460220FAF7AEFF0126254DA3
:10A54000FAF798FF0446FAF798FF0146204601F013
:10A550000BFBFAF792FF01462046F5F7BCFEFEF72B
:10A560003DFB062C29D2DFE804F028180722251528
:10A57000641E002CCFDCDBE7287840B9FCF77AF9C1
:10A5800028B900221E21022001F06DFA2E7002F07F
:10A5900075FAD5E7FFF768FAD2E7FCF796F8FAF70D
:10A5A00069FF012804BF0220FAF773FFC8E701F032
:10A5B0000FFBC5E7FFF7DEF9C2E7FBF714F8BFE7CB
:10A5C000007F0110BC7B0110DC010110DC2B0100BD
:10A5D000FF700200E0010110FE490870704710B4DE
:10A5E0004FF42C30FC4A016891421CD14168B1F50E
:10A5F000007F18D3836800228446B3F5056F88BFB7
:10A600004FF405630021B1EB930F24BF10BC7047DA
:10A610005CF82140491C2244B1EB930FF8D3002A87
:10A6200004BF10BC7047002010BC704770B54FF4D9
:10A630002C310446E84D0868A84217D14868B0F5A7
:10A64000007F13D38B6800228C46B3F5056F88BF5B
:10A650004FF405630020B0EB930F08D25CF8206044
:10A66000401C3244B0EB930FF8D302B1002149B142
:10A670008A68B2F5056F88BF4FF40562204605F081
:10A6800059FE1CE0FF224FF40561204605F0B1FEA3
:10A690004FF40070C4E900504FF40560A060002042
:10A6A000E06084F8200084F8210084F8220084F817
:10A6B000230040F2FF71C4E90410A061E0610120B1
:10A6C00070BD70B50021C160D0F808C00B460446CB
:10A6D000BCF5056F88BF4FF4056C0022B2EB9C0FF0
:10A6E00006D254F82250521C2B44B2EB9C0FF8D3E4
:10A6F0005942C1604FF42C304FF405622146F8F7FF
:10A70000F7FB012818BF002070BDFF2270B500259F
:10A71000044605614FF40061503005F06AFEA584DF
:10A72000E584A562E56225636563A563E563256449
:10A730006564A5640120E56470BD70B402684FF4DF
:10A7400000715160016801F1500291F821C091F847
:10A7500020300CFB03F102EB41010022BCF1000FA1
:10A7600008D900EB4204521CB4F88A4021F8024B8D
:10A770009445F6D80022002B08D900EB4204521C65
:10A78000B4F8CA4021F8024B9342F6D80022BCF13B
:10A79000000F07D900EB4204521CA48821F8024B99
:10A7A0009445F7D80022002B08D900EB4204521C34
:10A7B000B4F8444021F8024B9342F6D8B0F8862012
:10A7C00021F8022BB0F8882021F8022BB0F8842061
:10A7D00021F8022B00240022BCF1000F88BF00EBFF
:10A7E000841508D905EB4206521CB6F80A6121F817
:10A7F000026B9445F6D80022002B88BF00EB84152D
:10A8000008D905EB4206521CB6F8CA6121F8026B62
:10A810009342F6D8641C032CDDD370BC70472DE93D
:10A82000F74F88B000250A992C462E4609680491F6
:10A8300001F150030999002984BF6849D1F80080CB
:10A840001CD90022002888BFB8F9CE700DD933F981
:10A85000021B0029B4BFC1F1000C8C46BC45BCBF33
:10A860000D44641C521C8242F1D30999761C8E421D
:10A87000E7D3002CC8BF95FBF4FA08DC4908414334
:10A8800001EB5002049901EB4201B1F950A0002103
:10A89000029101910499503100910021039109998D
:10A8A00000296CD94D49009E069609684FF0000BAF
:10A8B0004FF00109B1F9C0E0D1F8B4105F46C1F31F
:10A8C0000741D846CDF814B00791002829D9B6F928
:10A8D00000204FF0000C06999344634600280DD9E0
:10A8E000B1F90040A51A48BF151B7545B8BF0CF15A
:10A8F000010C01EB49015B1C8342F1D307998C45A4
:10A9000003D305997F1C1144059108F1010806EB5A
:10A9100049068045DBD3002FC4BF059991FBF7F1B1
:10A9200001DC9BFBF0F1039B0A9A09B202EB4302A4
:10A9300091802A4A1268B2F9BA30AAEB030399420D
:10A940000ADDB2F9B82052448A4205DD019A114469
:10A9500001910299491C02910099099A01EB400169
:10A9600000910399491C039191429BD302990029BC
:10A9700005DDDDE9011291FBF2F1019102E05146A2
:10A98000CDF804A00A9AA2F8861000210291039142
:10A990000499503100910021049100286FD90F498A
:10A9A000009F069709684FF0000B099EB1F9BCE0C3
:10A9B000D1F8B410D846090ED946CDF814B0079195
:10A9C000002E32D9B7F900204FF0000C93446346B3
:10A9D000069905E0E101011053454C46DC010110E8
:10A9E000002E0DD9B1F90040A51A48BF151B7545B9
:10A9F000B8BF0CF1010C01EB40015B1CB342F1D379
:10AA000007998C4504D3059908F101081144059173
:10AA100009F1010907EB4007B145D3D3B8F1000FA5
:10AA2000C4BF059991FBF8F101DC9BFBF6F1049B97
:10AA30000A9A09B202EB4302A2F84410FE4A1268D5
:10AA4000B2F9BA30AAEB030399420ADDB2F9B82091
:10AA500052448A4205DD039A114403910299491C2C
:10AA600002910099891C00910499491C049181422A
:10AA700095D302980028C4BF039991FBF0FA0A9875
:10AA8000A0F888A001980A99504400B200EBD07059
:10AA90004010A1F884000BB0BDE8F08F2DE9F04F15
:10AAA000BBB016460D460446F6F7A0FFF6F7E9F8E8
:10AAB00001004FF011001DBF029001200390012101
:10AAC00008BFCDE90210CDE93654F7F72BFA002282
:10AAD000002D88BF04A904D9835C8B54521C954275
:10AAE000FAD8F7F721FA0021002C88BF04AA07D969
:10AAF000435C02EB010C491C8CF820308C42F7D8E7
:10AB0000F7F751F940F2012135900840F7F743F883
:10AB1000CA480DF1D80B007810F0200F6AD0F6F774
:10AB2000B0F8C74A44F6C00144F640031268002852
:10AB300011441A440CBFCDE90021CDE9001206F101
:10AB40008A00389040303990FF210F20FAF731FF0A
:10AB5000F6F74CFF0025EA460DF1E00902A85BF884
:10AB6000257050F82500F7F79FFD0024002F84BFC3
:10AB700004A800EB45181AD918F90400202828BFAA
:10AB800000200DD25AF8251000EBD072521051F867
:10AB90002210C007C00E21FA00F080B2F7F78AFD3C
:10ABA00059F8251021F81400641CBC42E4D36D1C34
:10ABB000022DD3D3A34805781D2D1BD100210A46B1
:10ABC00014AC5BF822C00020BCF1000F88BF59F81C
:10ABD000223007D933F8107024F81170401C491C3A
:10ABE0008445F7D8521C022AEBD31D2D04BF204602
:10ABF000FEF74AFC9148007810F0040F00F0E7815E
:10AC0000F6F73FF88E490028096801F52C6201F536
:10AC100004610CBFCDE91412CDE914218A48F6F77E
:10AC2000BAFF0120F6F786FB2C900120F6F7CEFB49
:10AC30002B900120F6F733FE23900298F6F7F0FBF5
:10AC400024900398F6F7ECFB17900120F6F775FCBB
:10AC50002A901120F6F771FC27900120F6F79CFC52
:10AC600028901120F6F798FC259020A800901EABA4
:10AC70001CAA1AA90298F6F765FD21A800901FAB3F
:10AC80001DAA1BA90398F6F75DFD0298F6F7D6FDFD
:10AC900022900298F6F7D2FD674C01902068B0F838
:10ACA000E4100120F6F754FB00210120F6F7E2FD45
:10ACB000206890F8E6100298F6F7C1FB206890F83B
:10ACC000E6100398F6F7BBFB00210120F6F74BFCDA
:10ACD00000211120F6F747FC00210120F6F772FC55
:10ACE00000211120F6F76EFC2068B0F8E8100298F9
:10ACF000F6F755FD2068B0F8E8100398F6F74FFD19
:10AD00000020F6F7E5FD29902068B0F8EC100091DE
:10AD100090F8EB3090F8EA200B210298F6F7E6FC69
:10AD20002068B0F8EC10009190F8EB3090F8EA2031
:10AD30000B210398F6F7DAFC0020F6F7C9FD2EADDB
:10AD4000F7F799F8FDF77CFF012805D02846F7F7BB
:10AD50002FFA002800F04181F6F748FE32990022D0
:10AD600000205BF822C0BCF1000F84BF02EB42035D
:10AD700006EB831308D931F8025B03EB4007401C54
:10AD8000A7F80A518445F6D8521C022AE8D3029843
:10AD9000F5F7D3FC18900398F5F7CFFC16900298BE
:10ADA000F6F7BEFB26900398F6F7BAFB224C1990F3
:10ADB0002068B0F8EE10009190F8EB3090F8EA209F
:10ADC0000B210298F6F792FC2068B0F8EE10009183
:10ADD00090F8EB3090F8EA200B210398F6F786FC08
:10ADE00000250020F6F774FD00210298F5F790FC8D
:10ADF00000210398F5F78CFC0DF10808012158F8A3
:10AE00002500F5F785FC36A8002450F8257014A815
:10AE1000002F50F825A03ED904A800EB451905EBFA
:10AE2000450006EB8018002119F804B00846F6F733
:10AE300068FD01200AE00000DC010110E1010110C1
:10AE4000F82B01005601011001000E0000FA0BF171
:10AE500002A88B4650F82500F6F755FB6FEA0B0168
:10AE60000920F6F74EFD0DF1B80BF7F704F8FDF7E2
:10AE7000E7FE012804D05846F7F79AF900287CD05D
:10AE8000F6F7B4FDBAF8000008EB4401641CA1F821
:10AE90004A01BC42C7D300210846F6F732FD6D1CBB
:10AEA000022D9ED318990298F5F732FC1699039853
:10AEB000F5F72EFC26990298F6F725FB19990398C9
:10AEC000F6F721FBFE4C2068B0F8F010009190F8E6
:10AED000EB3090F8EA200B210298F6F707FC206887
:10AEE000B0F8F010009190F8EB3090F8EA200B21C8
:10AEF0000398F6F7FBFB0120F6F7EAFC2EACF6F719
:10AF0000BAFFFDF79DFE012804D02046F7F750F95F
:10AF1000002868D0F6F76AFD3299002236AC00208E
:10AF200054F822C0BCF1000F84BF02EB420306EBD1
:10AF3000831308D931F8025B03EB4007401CA7F8E4
:10AF40008A518445F6D8521C022AE8D301202C9954
:10AF5000F6F7FEF901202B99F6F740FA0120239924
:10AF6000F6F788FC24990298F6F769FA179903987E
:10AF7000F6F765FA01202A9900E031E0F6F7F3FAD6
:10AF800011202799F6F7EFFA01202899F6F71AFB16
:10AF900011202599F6F716FB209800901E9B1C9A0D
:10AFA0001A990298F6F7A2FB219800901F9B1D9A10
:10AFB0001B990398F6F79AFB22990298F6F7EFFB94
:10AFC00001990398F6F7EBFB2998F6F781FC359881
:10AFD000F6F7E1FD3BB0BDE8F08FFAF79DFAB1E678
:10AFE000FAF79AFA43E7FAF797FA8AE72DE9F04F6A
:10AFF000ADF6F42DFF224FF4056102A805F0F9F932
:10B00000FF224FF423710DF6580005F0F2F902A863
:10B01000CDF85808FFF70AFBAA4C207810F0080F6B
:10B0200015D0002516A8FF224FF40061069505F003
:10B03000E0F9ADF82C50ADF82E500C950D950E950D
:10B040000F95109511951295139514951595DDF89A
:10B0500058080DF6580290F820C090F82110503092
:10B0600001FB0CF300EB43000023002908D902EB9D
:10B07000430630F8025B5B1CA6F88A509942F6D86A
:10B080000023BCF1000F08D902EB430630F8025B45
:10B090005B1CA6F8CA509C45F6D80023002907D9A6
:10B0A00002EB430630F8025B5B1CB5809942F7D88F
:10B0B0000023BCF1000F08D902EB430630F8025B15
:10B0C0005B1CA6F844509C45F6D830F8023BA2F829
:10B0D000863030F8023BA2F8883030F8023BA2F804
:10B0E000843000250023002988BF02EB851608D98B
:10B0F00006EB430830F8027B5B1CA8F80A71994202
:10B10000F6D80023BCF1000F88BF02EB851608D9E2
:10B1100006EB430830F8027B5B1CA8F8CA719C451B
:10B12000F6D86D1C032DDDD36046FFF778FB27783A
:10B13000012517F0800F7DD161480DF658090025D3
:10B14000006890F8B40000F00F0600F03EFD012802
:10B1500009D00F213046FAF780FA012814D00020D8
:10B1600000F030FD77E000210846F6F73BFDF5F7EB
:10B170007CFD60B154480168D1F8B012006841F418
:10B180008031C0F8B01202E0012000F01BFD4F48F2
:10B1900090F800804E480678002E18BFB8F1000FD6
:10B1A00057D0DDF85808002180F8208080F8216011
:10B1B00080F8221080F82310F7F7AAFA17F0240F6E
:10B1C00004D04A4631464046FFF768FC17F0030FAB
:10B1D0003ED0B246F6F7E7FD054600F48170F6F77B
:10B1E000DAFCFF210F20FAF7E4FBF6F7FFFB284615
:10B1F000F6F7D1FCDDF85878002107F150000090F7
:10B20000534642460846F7F789F90020F7F74CFA0B
:10B2100000250AFB08FBBBF1000F0AD907EB450626
:10B22000B6F85000F7F746FA6D1CA6F85000AB458B
:10B23000F4D800E00FE0274800781D2804BF07F18C
:10B240005000FEF71DF84A4651464046FFF7E7FA20
:10B250000125F6F763FD9DF828009DF82910CDF82B
:10B26000E40A002D19BF002800290DF6F42DBDE8D1
:10B27000F08F14480078CDF8EC0A10F0020F00F0BF
:10B28000E780DDF85858DDF8E42A47F6FF7A2869A8
:10B2900005F1500820F00F002861CDF8F00A0020D9
:10B2A0006FEA0A09009006460190002954D9044823
:10B2B0000068CDF8E80A06FB02F038F910300BE020
:10B2C000DC010110E1010110E02B0100CA000110B6
:10B2D000CB000110510101101F460124BC464FF064
:10B2E000000B012A17D906FB024038F9100060450F
:10B2F000C8BF84469842B8BF0346B0EB070E48BFAC
:10B30000A7EB000E0FFA8EF75F45C8BFBB46074696
:10B31000641C9442E7D3CC45C8BFE1465345B8BF4F
:10B320009A46BCEB030048BFA3EB0C0000B2DDF86B
:10B33000E83AB3F9C030834205DBDDF8E80AB0F93A
:10B34000C200834505DD012000FA06F30198184389
:10B350000190761C8E42AED30026002A45D9FE48C5
:10B360000068CDF8E80A38F9163001241F46BC46BB
:10B370004FF0000B012917D904FB026038F91000C7
:10B380006045C8BF84469842B8BF0346B0EB070E7D
:10B3900048BFA7EB000E0FFA8EF75F45C8BFBB464C
:10B3A0000746641C8C42E7D3CC45C8BFE1465345F1
:10B3B000B8BF9A46BCEB030048BFA3EB0C0000B239
:10B3C000DDF8E83AB3F9BC30834205DBDDF8E80A82
:10B3D000B0F9BE00834505DD012000FA06F30098B0
:10B3E00018430090761C9642BDD30198E86220B1C4
:10B3F000DDF8F00A40F0080028610098A86218B152
:10B40000286940F004002861A5F824A0A5F826903A
:10B41000BDF9DC28B9EB020048BFA2EB0900CE4A17
:10B420001368B3F9B820904203DD286940F00200A8
:10B430002861BDF9DC28B2EB0A0048BFAAEB020084
:10B44000B3F9BA20904203DD286940F00100286179
:10B45000DDF8EC0AC14C10F0050F05D00DF65802CE
:10B46000DDF8E40A00F050F8207810F0400F2FD1FA
:10B470000798401C07900698002814BF0998089860
:10B4800000F1010014BF099008900DF65800FFF775
:10B4900054F9002002460590049802A98C46B0F5A4
:10B4A000056F94BF03464FF405630020B0EB930F84
:10B4B00006D25CF82040401C2244B0EB930FF8D336
:10B4C0005042C8604FF42C304FF40562F7F710FD7E
:10B4D0000A208DF800009DF818008DF801009DF8F5
:10B4E00019008DF802009DF81A008DF803009DF8F0
:10B4F0001B008DF8040005226946012000F0DAFAED
:10B500000DF6F42DBDE8F08F2DE9F05F14680646C6
:10B51000DFF844922069154620F4FE6020618F48D0
:10B520000F464FF00108007810F0010F52D030465E
:10B5300000F09EF92B680020002E186388BFD9F810
:10B54000002014D905EB4001B1F944100029B8BF1F
:10B55000494209B2B2F9CCC08C4505DD196B08FA35
:10B5600000FC41EA0C011963401CB042EAD34FF0E1
:10B57000000C012E1CBFA6F1010ED9F800B029D095
:10B5800005EB4C00B0F94620B0F94410501A48BF02
:10B59000881A00B2BBF9C4A0824517DAB5F9880051
:10B5A000B1EB000A48BFA0EB010A0FFA8AFA111AA0
:10B5B00048BF811A08B28245186BAEBF08FA0CF179
:10B5C0000CF1010108FA01F1084318630CF1010CB8
:10B5D000F445D5D3614890F800C01CF0040F00F08A
:10B5E000148129684FF0000B5846C1F83CB0002F79
:10B5F00088BFD9F8003014D905EB4002B3F9D8A0C0
:10B60000B2F90A21924503DCB3F9DAA0924505DAD2
:10B61000CA6B08FA00FA42EA0A02CA63401CB8423E
:10B62000EAD329680020002EC1F838B088BFD9F8C5
:10B63000003014D905EB4002B3F9D8A0B2F9CA2101
:10B64000924503DCB3F9DAA0924505DA8A6B08FA71
:10B6500000FA42EA0A028A63401CB042EAD329682F
:10B660000020002FC1F844B088BFD9F8003014D9A9
:10B6700005EB4002B3F9DCA0B2F94A21924503DCA4
:10B68000B3F9DEA0924505DA4A6C08FA00FA42EAFC
:10B690000A024A64401CB842EAD329680020002EFE
:10B6A000C1F840B088BFD9F8003014D905EB40028A
:10B6B000B3F9DCA0B2F90A22924503DCB3F9DEA0AB
:10B6C000924505DA0A6C08FA00FA42EA0A020A64AC
:10B6D000401CB042EAD328680021002FC0F84CB0CB
:10B6E000C0F848B088BFD9F8003014D905EB410242
:10B6F000B3F9E0A0B2F98A21924503DCB3F9E2A0E4
:10B70000924505DAC26C08FA01FA42EA0A02C264FA
:10B71000491CB942EAD30021002E88BFD9F8003075
:10B7200014D905EB4102B3F9E090B2F94A229145F0
:10B7300003DCB3F9E290914505DA826C08FA01F96D
:10B7400042EA09028264491CB142EAD3A56B206C2B
:10B7500030EA050204E00000DC010110E101011003
:10B7600042EA0503226413D000210846002E0FD9B7
:10B7700008FA00F912EA090F18BF491C401CB04230
:10B78000F6D3012904D145EA0200C4F840B0A06311
:10B79000A06C984340EA0301A06404D0E06C002848
:10B7A00008BFC4F848B01CF0010F02D0206B8843DA
:10B7B0002063E56B606C30EA050242EA05036264CF
:10B7C00012D000210846002F0ED908FA00F63242A6
:10B7D00018BF491C401CB842F7D3012904D145EADF
:10B7E0000200C4F844B0E063E06C984340EA03010F
:10B7F000E06404D0A06C002808BFC4F84CB01CF072
:10B80000010F02D0606B88436063206B18B1206920
:10B8100040F010002061606B18B1206940F02000FA
:10B820002061A06B18B1206940F040002061E06BFE
:10B8300018B1206940F080002061206C18B12069A7
:10B8400040F480702061606C18B1206940F4007091
:10B850002061A06C18B1206940F480602061E06C28
:10B8600018B1206940F4806020610120BDE8F09F9C
:10B870002DE9F74F13684FF0000883B0724CC3F8FE
:10B880003480DDF810C00127D4F800B04146BCF187
:10B89000000F1BD902EB410CBCF904C0BCF1000F36
:10B8A000B8BFCCF1000C0FFA8CFCBBF9CC4064455E
:10B8B00007DDD3F834C007FA01F44CEA040CC3F8EE
:10B8C00034C0DDF810C0491C6145E3D30021BCF150
:10B8D000010F1CBFDDF810C0ACF101092FD002EB45
:10B8E000410CBCF90650BCF90440B5EB040C48BF50
:10B8F000A4EB050C0FFA8CFCBBF9C66066451BDA9D
:10B90000B2F986C0B4EB0C0648BFACEB040636B205
:10B91000B5EB0C0448BFACEB05040FFA84FC66459C
:10B92000D3F834C0AEBF07FA01F44C1C07FA04F494
:10B930004CEA040CC3F834C0491C4945CFD39BF8EA
:10B94000CA20002A7CD09BF8CB108A4288BF1146BF
:10B950000022DDF810C0BCF1000F84BF491C00912B
:10B960006ED94FF0010EDDF800C04FF00008012144
:10B97000C146BCF1010F48D902FB0004BBF9CEC09F
:10B9800002940EFB0004019402FB001403EB440438
:10B99000B4F95060002EB4BF74423446A44534DB81
:10B9A0000EFB001403EB4404B4F95050002DB4BF57
:10B9B0006C422C46A44528DB029C641A03EB440429
:10B9C000B4F94E40002CB4BF67422746BC451CDB8F
:10B9D000019F7F1A03EB4707B7F94E70002FB4BFE2
:10B9E000C7F1000ABA46E2450FDCAE1BBBF9C850EE
:10B9F000B542B8BF08F101083C1BAC42C8BF09F111
:10BA00000109491C009CA142BED3B9EB080148BF03
:10BA1000A8EB09019BF8CAC0614506DB0121D3F8F8
:10BA200034C091404CEA010159630499521C8A4286
:10BA300006D2002A18BFA2F1010E94D191E7FFE7C8
:10BA400006B00120BDE8F08FDC0101105949C2B2F7
:10BA5000C0F307200A804880704756484188008814
:10BA600061F31F207047DFF84CC101238340BCF80D
:10BA700000C013EA0C0F08BF704700B583B000F098
:10BA80003F008DF800008DF801108DF80220100A9B
:10BA90008DF80300100C8DF80400100E8DF80500D1
:10BAA00000208DF806008DF80700684604F019FDA7
:10BAB00003B000BDDFF8FCC001238340BCF800C028
:10BAC00013EA0C0F08BF704710B582B000F03F00BA
:10BAD0008DF80000072A88BF072200206B46002A45
:10BAE00009D911F800C01C18401C84F801C090420C
:10BAF000F7D3072805D200211A18401C51700728D7
:10BB0000FAD3184604F0EDFC02B010BDDFF8A4C073
:10BB100001238340BCF802C013EA0C0F08BF704732
:10BB200010B582B000F03F0040F080008DF80000BA
:10BB3000072A88BF072200206B46002A09D911F87E
:10BB400000C01C18401C84F801C09042F7D307289D
:10BB500005D200211A18401C51700728FAD3184644
:10BB600004F0BFFC02B010BD70B5124E40EA0125D2
:10BB70000228B488224618BF052803D1002918BF1F
:10BB8000022900D12C46A24208D049B1F0880121F7
:10BB900044EA00420320FFF766FFB480F58070BDE1
:10BBA000F7F74BFE44EA004201210320FFF75BFF59
:10BBB000F3E70000E2010110FE4908707047FD48FC
:10BBC00000787047FB4948707047FA4840787047E2
:10BBD0002DE9F04F93B0F6F7EFF811900020F6F74B
:10BBE000E5F8F44D002420466C70F6F795F9FDF762
:10BBF00027F8012804D1F9F73DFC032840F008821A
:10BC0000EC4C207810F0010F07D0FFF7EFF9207807
:10BC100020F001002070FCF7DDFF207810F0020F0B
:10BC200000F0F281E448E34900684978B0F8580030
:10BC30000229C0F303200DD0DE4CA17801F00F01E2
:10BC4000F9F70BFD01280CBF02200020607011D015
:10BC500000F0D1B900210846F5F7C4FFF5F705F863
:10BC600040B1D6480168D1F8B012006841F4803183
:10BC7000C0F8B012F6F797F8DFF838A310909AF8EA
:10BC8000020010F0100F18BFF6F73FFDFF210F2044
:10BC9000F9F78FFECA4800780C90CA4800780D90DA
:10BCA000C94890F800B0C94800780F900D98002856
:10BCB0001CBF0C98002813D004F0E6FB04F0E9FB4D
:10BCC0000020F8F71DFE0020F8F78BFE9AF802001E
:10BCD00010F0100F0CD00120F8F794FE01200BE0BB
:10BCE0000F98002818BFBBF1000FE5D100F083B911
:10BCF0000020F8F787FE0020F8F784FE0120F5F712
:10BD000006FBF6F770F81E20FDF716FA002108462C
:10BD1000FDF7AAF9814601210020FDF7A5F9DDE92B
:10BD20000C128046002001FB02F7002F84BFA849B7
:10BD30004A0C06D929F8101028F81020401C874218
:10BD4000F8D81E20FDF771FB00210120FDF78CF9CA
:10BD5000054601210846FDF787F904460F990020A2
:10BD60001BEB01061CBF9A494A0C06D025F810109F
:10BD700024F81020401C8642F8D800200E908D48F0
:10BD8000808800287ED9701C40081290FCF758FF6C
:10BD9000012877D005A8F6F70BFA002873D006988B
:10BDA000F8F7F2F90798E0B38248807810F0100FA6
:10BDB00008D0DDF81CA004F099FB514604F0DCFB30
:10BDC000824615E000200023019002900390049029
:10BDD00000901A461946079804F08DFB8246754874
:10BDE000807810F0200F03D004F080FB824609E039
:10BDF000F8F71AFA0D9A00925246014610460C9B2B
:10BE000004F0ECFBBAF1000F1CBF0020002F12D988
:10BE10003AF9101039F910208A42B8BF29F81010E9
:10BE200000E008E038F910208A42C8BF28F8101056
:10BE3000401C8742ECD8109810F0010F1CBF0A98E4
:10BE4000002832D05B48807810F0200F0AD0002202
:10BE500011460A9804F054FB04F099FA5FEA000ACC
:10BE600023D00BE0DDF828A0F8F7A7F90222009212
:10BE7000524601461046129B04F0B0FB0020002EF3
:10BE800013D901E01FE016E03AF9101035F910203F
:10BE90008A42B8BF25F8101034F910208A42C8BF72
:10BEA00024F81010401C8642EBD8F6F7D0F90E9813
:10BEB000401C0E9002E0F9F72FFB0E983D4989884F
:10BEC0008842FFF463AFF5F791FD04F0E2FA04F065
:10BED000E5FA38490E98898888427BD3109810F08B
:10BEE000020F26D000224FF6FF731046002F0ED906
:10BEF00039F9101038F910C0A1EB0C019142C8BFFC
:10BF00000A469942B8BF0B46401C8742F0D80B2026
:10BF10008DF80000100A8DF801008DF80220180A33
:10BF20008DF803008DF80430052269460120FFF7E3
:10BF3000C1FD109810F0010F57D000224FF6FF738B
:10BF40001046002E0ED935F9101034F910C0A1EBAF
:10BF50000C019142C8BF0A469942B8BF0B46401C2B
:10BF60008642F0D80020BBF1000F84BF0F9901EB8F
:10BF70000B0616D9A6EB000C05EB4C0104EB4C0CA0
:10BF800031F8027CABEB000105EB410804EB410109
:10BF9000A8F866703CF802CC401CA1F866C0834546
:10BFA000E8D80D208DF80000100A8DF801008DF8FA
:10BFB000022010E0EA010110DC010110E02B010079
:10BFC000CA000110CB000110CF000110D0000110F9
:10BFD0000080FFFF09E0180A8DF803008DF8043097
:10BFE000052269460120FFF765FD3020FDF7A4F822
:10BFF0003020FDF71AFAF5F791FE1048017821F08C
:10C0000002010170FCF7E6FDF9F734FA032808D0C5
:10C010000120F5F781FF119813B0BDE8F04FF5F757
:10C02000C5BEF9F779FAE2E504498870704703481C
:10C03000807870470149888070470000EA0101104C
:10C04000FE4908707047FD4800787047FB4948700A
:10C050007047FA4840787047F84840797047F74988
:10C06000002048717047F54988717047F34880791E
:10C070007047F24982B26FF30F00C1E904027047C2
:10C08000EE48C0787047ED4A0028516914BF41F06E
:10C09000020021F0020050617047E848007DC0F3C3
:10C0A00040007047E54AF02303EA0010516921F08F
:10C0B000F001084350617047E048007DC0F3031071
:10C0C0007047DE4A0028516914BF41F0010021F099
:10C0D000010050617047D948007D00F001007047B1
:10C0E000D64B19690A0E120721F07F4142EA00601F
:10C0F000084318617047D1480069C0F30360704776
:10C10000CE480069000F7047CD480068406DC0F30D
:10C1100003607047012101FA00F04FF47F0101EA4A
:10C120000041C6480269114301617047012101FACB
:10C1300000F04FF47F0101EA0041C048026922EAA1
:10C14000010101617047BD480069C0F307407047B5
:10C15000BA48008AC0F303307047B84910B50246A8
:10C1600008694FF47043C0F3033420F4704003EACD
:10C1700002331843086103210846FFF774FC204688
:10C1800010BDAE48808AC0F38020704770B5AB4EBA
:10C190000446C0F380007569C5F30021884210D0C1
:10C1A000F8F75CFB14F0040F05D004F0FFF8012849
:10C1B00008BF002003D0A34890F86C00C00804F02A
:10C1C00027F9C4F3C010C5F34031884218BFF8F70F
:10C1D00045FB14F0010F14BF45F0400025F040006E
:10C1E00014F0040F14BF40F4807020F4807014F039
:10C1F000080F14BF40F4007020F4007014F0100F0A
:10C2000014BF40F4806020F4806014F0200F14BF4D
:10C2100040F4006020F4006014F0800F14BF40F47C
:10C22000005020F400507061BDE87040FDF774BF0D
:10C2300082484169002011F0400F18BF012011F021
:10C24000200F18BF40F0020011F4807F18BF40F0AB
:10C25000040011F4007F18BF40F0080011F4806F53
:10C2600018BF40F0100011F4006F18BF40F020001C
:10C2700011F4005F18BF40F0800070476F48007DE8
:10C28000C0F3801070476D48007DC0F340107047C8
:10C290006A48808AC0F3002070476848808AC0F3EB
:10C2A00040207047FDF73EBD6448808AC0F34030AF
:10C2B00070476248808AC0F3C02070475F48808A18
:10C2C000C0F3003070475D484069C0F3003129B1C8
:10C2D000C0F34010002804BF0120704700207047C1
:10C2E00056498A6910438861704770B5534EB069EA
:10C2F00040F400740020B061756915F0400F1CBF58
:10C3000015F0040F44F0010415F0200F1CBF15F0C8
:10C31000080F44F0020415F4807F18BF44F00404B1
:10C3200015F4007F18BF44F00804FDF7FBFC00285B
:10C3300018BF44F0100415F4006F18BF44F0200437
:10C3400015F4805F18BF44F04004308AC0F3033115
:10C3500044EA0140002918BF40F4806070BD3749AD
:10C36000C86170473548007F00F0010070473348CE
:10C37000007FC0F3400070473048007FC0F380006A
:10C38000704703463048520000EB4100194603F065
:10C39000E0BF2D48704710B5284C002818BF00207A
:10C3A00001D0207210BD26480068B0F85800C0F3D4
:10C3B0000320FDF789FF002818BF4079F1D110BD97
:10C3C0002DE9F043002487B0A046F9F753F81C4943
:10C3D000052808680CBF90F8F80090F8580000F0A5
:10C3E0000F09484604F091F8144F064616F0100F56
:10C3F000387DC0F303150ED0F5F7DEFC38B116F426
:10C40000801F04BF25F00C0040F0020503D007B0E8
:10C410000020BDE8F08329464846F9F71EF90028B8
:10C4200004BF07B0BDE8F0830120F4F770FFF5F713
:10C4300022FDFCF705FC01286FD007E0F001011098
:10C44000DC010110BC7B0110808401106846F5F707
:10C45000AFFE00285DD06846FDF73BF90198F7F77D
:10C4600093FE029888B1FE48FE49007809784000A2
:10C4700000FB01F2FC48029903F06BFFFB480078D7
:10C48000492804BFF848FCF7FBFE059800283BD07C
:10C49000F748F849059C007809784518F7F7C1FE78
:10C4A000DFF8D483B0B1397A00EB410698F8000088
:10C4B000022804BF3046FCF7E7FF0022002D09DD0B
:10C4C00034F8120036F81210401A24F81200521CE8
:10C4D0009542F5DCF5F770FC30B1F5F764FC10F42B
:10C4E000801F08BFE54801D0F7F767FE397A6A0078
:10C4F00000EB4100214603F02CFF98F800000328D0
:10C5000004BF2046FCF7C0FFF5F7A1FE4FF001087D
:10C5100003E0F9F701F8002C8BD0F5F767FAF9F78B
:10C5200008FA07B04046BDE8F0832DE9F04387B034
:10C530000446052802D1FDF74DFA08B9FFF740FF80
:10C54000F8F798FF8046F8F798FFDFF8349307462E
:10C55000B8F1050F0CBFCB4ECB4E99F81400C0F3C9
:10C56000031218BF052F05D1FFF7ADFE002818BF35
:10C5700042F0020211462046F9F76FF8002804BF86
:10C5800007B0BDE8F08303F07FFFF8F70EF905462A
:10C59000F7F756F90124F4F768FB0020F4F7B7FE2B
:10C5A0002046F5F739FCC9F83040A4F10109FCF741
:10C5B00047FB012809D0F8F75DFF404505D1F8F7A2
:10C5C0005CFFB84208BF002D0AD0F5F70FFA03F060
:10C5D00065FFF9F7AEF9F7F76FF907B0BDE8F0833B
:10C5E0006846F5F7E5FDC0B16846FDF772F80198B9
:10C5F000F7F7CAFD6846B0470546F5F728FE002D57
:10C60000D5D114B901984845D1D1F5F7EDF90028F5
:10C6100004BF2046F5F700FCC9E7F8F772FFC6E74C
:10C620002DE9F14F002688B08D48039605960696B1
:10C63000049604788B480899374605780A4604FB27
:10C6400005F001EB40090290B0460095234686496B
:10C65000484603F0C3FFDFF814A29AF80000492807
:10C6600004BF8148FCF70CFE804800784C2804BFCA
:10C670004846FCF705FE02994FF0000A09EB41031A
:10C680009C46002D2DD90020611E13D009EB410BD3
:10C6900039F811203BF802BCA2EB0B0212B2002ABF
:10C6A000B8BF524212B22CF811208242C8BF1046C5
:10C6B000491EEBD10CEB440131F9022C142AB9BF0D
:10C6C00031F9042C142A01260596ACF8000009EB78
:10C6D00044098C46B842C8BF07460AF1010AAA4578
:10C6E000D1D36749B1F90C904845A4BF012003900C
:10C6F0004F45A4BF01260596002E37D16048C0796A
:10C7000000281CBF0022002D88BFEC462ED902FB5A
:10C7100004F003EB4000018EADF80010818EADF8FF
:10C720000210018FADF80410B0F93CA0ADF806A0DE
:10C7300000210CEB410B3CF81100BBF802B058444F
:10C7400000B2484503DB0126074604960BE0491C6E
:10C750000329EEDB3EB9BAF1140F04DB0126BDF963
:10C760000670049602E0521CAA42D0D302994FF000
:10C77000000A03EB410C002D28D90020611E02297C
:10C7800012D903EB410233F811B032F802EC32F85F
:10C79000042CF3445A4412B22CF811208242C8BF30
:10C7A0001046491E0229ECD80021ACF80000ACF874
:10C7B0000210ACF8041003EB44030CEB440C4045AE
:10C7C000C8BF80460AF1010AAA45D6D32C4BB3F95B
:10C7D0000E209042A4BF012003909045A4BF0126E3
:10C7E0000696002E14BF586B986B00F1010014BF21
:10C7F000586398631D480078FF285BD00299089819
:10C8000020F83160DDF808C00898059900EBCC00ED
:10C810004180069981800499C18003990181596BF7
:10C820004FEAE17C01EB1C5C6FF30B0CA1EB0C01FC
:10C830004181996B4FEAE17C01EB1C5C6FF30B0CBF
:10C84000A1EB0C018181C781A0F81080D9794182C8
:10C85000A0F814900127C2824FF00208002E15E0C4
:10C86000CA000110CB000110807F0110510101109E
:10C87000D0000110CF00011056010110808401107A
:10C88000F001011089E400100BE80010089907EB93
:10C8900085032246CDF800800CBF4E204D20FCF7CA
:10C8A00092FC07EB85032246CDF8008047200899CB
:10C8B000FCF789FC039828B103F0A5FD002818BFF8
:10C8C000FDF78FF8304609B0BDE8F08F2DE9F04F45
:10C8D000DFF8B8B383B004460025BBF90C90EC48F0
:10C8E000EC490095007809782E464718F5F75BFA71
:10C8F0000190F7F796FC8246F5F75EFA30B1F5F74E
:10C9000052FA10F4801F08BFE34801D0F7F755FC36
:10C910009BF8081000EB4108E0480078032804BFAA
:10C920004046FCF7B1FDBAF1000F3BD09BF8080080
:10C930000AEB400AD9480078022804BF5046FCF7A9
:10C94000A3FD0020002F0CD93AF8101038F8102061
:10C95000114434F81020511A24F81010401C87425A
:10C96000F2D8DFF8388398F80000062804BF204684
:10C97000FCF78AFD019810F4007FA7F101001FD099
:10C98000002818BFBBF90E3033D034F9101000293D
:10C99000B4BF4A420A469A42BCBF0D44761C401EB0
:10C9A000F3D126E00020002FDBD934F8101038F83E
:10C9B0001020891A24F81010401C8742F5D8D0E7BF
:10C9C000002818BFBBF90E3013D004EB400234F836
:10C9D000101032F8022C891A09B224F8101000291C
:10C9E000B4BF4A420A469A42BCBF0D44761C401E60
:10C9F000EBD1002EC8BF95FBF6F52EB2268098F835
:10CA00000000072804BF2046FCF73EFD0025781EE5
:10CA10000ED034F81010891B09B224F81010002928
:10CA2000B8BF494209B28D42B8BF0D46401EF0D191
:10CA30002580BBF81400C0F3002048B103F0B6FC19
:10CA4000012803D003F0B2FC082801D14FF00509FA
:10CA50004D4508DD0120009098F80000402804BFF3
:10CA60002046FCF711FD98F80000012804BF20467D
:10CA7000FCF70AFD009803B0BDE8F08F2DE9F04FF8
:10CA800087B0FDF70BF9DFF818B2DBF80000B0F95A
:10CA90003610B0F9340003F0A7FCF7F7DFFE0420EE
:10CAA00000F0D9F8794E78B1307DC0F3401010B95C
:10CAB000FFF709FC40B9DBF80000806DC0F30340CC
:10CAC0000F2818BFF7F7B0FE052000F0C4F858B1E2
:10CAD000FFF7F9FB40B1DBF80000806DC0F30350B5
:10CAE0000F2818BFF7F7A0FEFF203071FAF740F8C3
:10CAF00003F010FDF8F7BEFC022873D1DFF8A49113
:10CB0000DFF8A481DFF8A4A100273069C0F3036532
:10CB1000DBF80000A900806D7762C840B76200F0C2
:10CB20000F04F762B08AC0F3403080B103F084FC98
:10CB300001280CD0DBF80000B0F85800C0F3032146
:10CB4000C0F303308C4202D10F2818BF0446294697
:10CB50000220FFF709F8062D6BD2DFE805F063032A
:10CB60000303676730692246C0F30364307D022CFB
:10CB7000C0F303130ED019461046F8F76EFD0028D7
:10CB800057D003F081FC03F084FCF7F70EFE05009C
:10CB900009D024E0FFF797FB002814BF43F00203FD
:10CBA00023F00203E7E7707800281CBF0001F4F7C8
:10CBB0000DFBF5F718F9B770FCF742F801280AD019
:10CBC000F8F758FC022806D13069C0F30360A04290
:10CBD00008BF002D07D003F05CFC03F05FFCF8F702
:10CBE000A8FE26E02EE06846F5F7E2FAB8B16846FE
:10CBF000FCF76FFD0198F7F7C7FA684603F08FFC62
:10CC0000054699F8000038B1D8F800008068CAF8E5
:10CC10000000D8F800000760F5F719FBCCE7F8F73B
:10CC20007BFCC9E7204603F043FC02E02046FFF707
:10CC30007CFCFCF705F8012804D0F8F71BFC02285F
:10CC40003FF463AF03F011FCF7F707FE07B0BDE850
:10CC5000F04FFDF723B80D4A0228117D1269C1F388
:10CC60000311C2F3074205D0012808BF11F0020FDB
:10CC70000AD002E011F0040F06D0012101FA00F001
:10CC8000104018BF0120704700207047F0010110CC
:10CC9000D0000110CF000110808401105601011056
:10CCA000DC01011025000110C02B01008C000110D7
:10CCB000FC4800787047FC490968B1F8B410884313
:10CCC000F849C04388607047F6488068C0437047A1
:10CCD0008446F5480B4600688179C079490001FB1C
:10CCE00000F2F248614600EBC32003F032BBF0498A
:10CCF0004FF6FF7221F8202001EB80014A80ED4AB7
:10CD000000211154921C1154EB4A42F8301002EBEE
:10CD1000C0025160E94A1154D21D02F8101002EB12
:10CD200040004170704700B50020FFF7E0FF012090
:10CD3000FFF7DDFFDB490020087000BDDE4A00215F
:10CD400002EBC0035B682E2B84BF52F83020202AF0
:10CD500009D9DB4A02EB40035B78042B22BF12F8AF
:10CD600010000428012108467047F0B4D049D54D81
:10CD700031F82210AB5C401A00B2002808BF1946F7
:10CD8000B8BF0121C8BF02214FF00106CC4CDFF82B
:10CD900028C313B38B425CF832300BD10028B8BFE4
:10CDA000404218444CF8320014F81200401C04F8B9
:10CDB00012000EE00CEBC20700287B60B8BF4042B7
:10CDC0004CF8320004EB420314F81200587004F8D7
:10CDD0001260A954F0BC012070470028B8BF40423F
:10CDE0004CF83200F3E72DE9FF4FAF48A3B00068DD
:10CDF000837990F8079000200090019003900290B2
:10CE00000490059006900890079009900A900B9066
:10CE10000D900C900E900F90109012901190139016
:10CE20001490159017901690189019901A901C90C5
:10CE30001B901D901E901F902190A9F101001FFAD8
:10CE400080FA2090994800EBC12B09B1012970D0DC
:10CE500000224FF0010E0026334635463446B446D4
:10CE6000724598BF10AF24D8219951451DD802FBB7
:10CE70000910DDF88C8038F810803BF81000A8EB22
:10CE8000000000B232280CDD2DF8110000FB015526
:10CE900000FB0244761C27F8120003446045C8BF1B
:10CEA0008446481C81B25145E1D9501C82B272457A
:10CEB000DAD9209A00210120012AC8BFE84615DDF1
:10CEC00008EB400738F9102037F902AC5245A2BFF1
:10CED000B7F90270BA42322A03DD801C491C80B2C5
:10CEE000C9B2401C209A80B29042E9DBBDF9000033
:10CEF000BDF902209042A8BF3228C4BF481CC1B26D
:10CF0000684600EB490030F9022C30F9040C8242EB
:10CF1000A8BF322AC4BF481CC1B2002E18BFBCF142
:10CF2000320F01DD01290AD027B00020BDE8F08FC3
:10CF3000FFE7981E82B2581E1FFA80FE8BE705EBB2
:10CF400085004000B0FBF3F004EB84014900259A12
:10CF5000B1FBF3F110802698018027B00120BDE8D5
:10CF6000F08F2DE9F04F89B08068002406AB05AA48
:10CF700021460090FFF737FF054603AB04AA0121C5
:10CF80000098FFF730FFDFF838A107900AF1040995
:10CF90002800494FA9F10F08A3464FF0010608F1F8
:10CFA000040535D02878002853D198F800000028CF
:10CFB00008BF88F8006022D00022BDF81810BDF824
:10CFC0001400FFF7D2FE00284FF0000011D079685E
:10CFD0002E2984BF3968202907D99AF8011004291D
:10CFE00022BF9AF8001004290120002818BF2E70D3
:10CFF00005E0FFF77CFE00210098FFF769FEBDF811
:10D000001400A9F80000BDF81800A9F8020020E0FB
:10D0100098F80000012804BF2878012812D11120B7
:10D020008DF804008DF805B038788DF806008DF87D
:10D0300007B038798DF80800052201A90120FEF714
:10D0400065FD01240020FFF752FE00210098FFF744
:10D050003FFE0798002847D06878002866D198F8E6
:10D060000100002808BF88F8016034D00122BDF813
:10D070000C10BDF81000FFF778FE28B30E49002011
:10D08000C9682E2984BFB968202907D90C49C978F5
:10D09000042922BF9AF8021004290120002818BF91
:10D0A0006E7018E0BC02011004030110A88F01107B
:10D0B000CC020110BD020110988F0110C1020110B5
:10D0C000C8020110BF0201100120FFF710FE01216C
:10D0D0000098FFF7FDFDBDF81000A9F80400BDF8A9
:10D0E0000C00A9F8060021E098F80100012804BF0F
:10D0F0006878012813D111208DF804000D218DF8D6
:10D100000510387A8DF806008DF80710387B8DF8F9
:10D110000800052201A90120FEF7F8FC01240120E6
:10D12000FFF7E5FD01210098FFF7D2FD0E485CB145
:10D130006978012919BF297801290670012004BFE7
:10D1400009B0BDE8F08F00E02CB180F800B009B064
:10D150000020BDE8F08F6978012919BF29780129DD
:10D1600002210170F1D1F2E7BC020110FE48026811
:10D17000FE48B2F8C61081810181B2F8C410C181A5
:10D180004181232101820721418240F6C41181613E
:10D19000322181827047F54800897047F3488089C1
:10D1A0007047F2490A28088184BF0A2008818881D3
:10D1B0007047EE4840897047EC48C0897047EB499A
:10D1C0002828488184BF28204881C8817047E748C3
:10D1D000008A7047E54908827047E448408A7047F2
:10D1E000E249B0F5C87F488284BF4FF4C8704882D6
:10D1F0007047DE48808A7047DC49B0F5967F8882A8
:10D2000084BF4FF49670888280B2404364225043BA
:10D2100088617047D5488069704770B503F084F91C
:10D2200003F087F9044690F8DC04D04E002538B9A5
:10D2300094F8DD0418B92021CD4803F07FF9B580BA
:10D2400094F8DD04002808BFF58070BD10B503F028
:10D250006BF903F078F9F323002100288CBFC44A4E
:10D2600010BD12F801C00CEA030C02F801C0491C01
:10D27000C9B28842F5D810BD70B5054603F054F91F
:10D2800003F061F9012D08BFFE2402D0022D08BF72
:10D29000FD24002100288CBFB54A70BD535C23409B
:10D2A0005354491CC9B28842F8D870BD70B51446B1
:10D2B0000D46064603F038F903F04AF90023012E23
:10D2C00002D0022E08D00EE0042C08BF01230AD0A1
:10D2D000052C08BF042306E0042C08BF022302D05B
:10D2E000052C08BF082305EB8501C1EB851100EB78
:10D2F0008101887A0A7B82422CBF9D4A70BD12F858
:10D3000000C04CEA030C02F800C0401C91F80CC0AD
:10D31000C0B28445F3D270BD2DE9F04116460D46EA
:10D32000074603F001F903F013F903F016F98046FC
:10D3300003F009F901468C482C46B5420068B0F963
:10D340000E308B4810D837F914209A4208DD025D60
:10D350000C2C42F00402025524BF42F01002025588
:10D36000621CD4B2B442EED9A8F1010251438AB290
:10D37000B54228BFBDE8F081511937F91110994223
:10D3800008DD415D0C2D41F00801415524BF41F0FD
:10D3900020014155691CCDB2B542EDD3BDE8F08105
:10D3A00010B503F0D0F8002100288CBF704B10BDE1
:10D3B0005A5C12F0100F1CBF22F010025A54D2B265
:10D3C00012F0200F1CBF22F020025A54D2B212F0E9
:10D3D000040F1CBF42F010025A54D2B212F0080FD0
:10D3E0001CBF42F020025A54491CC9B28142DFD30B
:10D3F00010BD2DE9F74F03F097F8044603F0A8F8A5
:10D40000054603F0AFF8584E94F841403068B0F844
:10D410001A8003F0A2F8306890F8CD90002084467E
:10D4200003460746002C88BFA8F125083BD903EB2B
:10D430008301C1EB831105EB810181F8C97081F88B
:10D44000CB703268B1F8AEA0B2F81AB0528A0AFBBB
:10D450000BFA9AFBF2F291F88DA092B2BAF1000F9A
:10D4600001BF91F8DAA0BAF1010F91F872A0BAF1F8
:10D47000000F14D1252A98BF012203D94245A8BF25
:10D4800002220CDB81F8C920012A04BF401CC0B273
:10D4900005D0022A04BF0CF1010101F0FF0C591C58
:10D4A000CBB2A342C3D3334A4FF0000411780844EF
:10D4B00010F0FF0150786044C2B218BF002A0AD0B1
:10D4C0008818814507D8DDE900010124029AFFF799
:10D4D00023FF2648478003B02046BDE8F08F2DE9A2
:10D4E000F04703F021F8044603F032F8054603F054
:10D4F00039F8DFF874801D4994F84140D8F80000ED
:10D50000B1F80CC00022408B002C86BFA0EB0C06AB
:10D510000627BDE8F08702EB8200C0EB8210D8F846
:10D52000003005EB8001B1F8AE00B3F81A905B8AC9
:10D5300000FB09F090FBF3F083B291F88D00002816
:10D5400004BF91F8E70002280DD163459CBF81F824
:10D55000C870012005D99E42DCBF81F8C870022046
:10D5600001DC81F8C90007E004030110D4020110B6
:10D57000B29F0110DA020110501CC2B2A242CAD3FB
:10D58000BDE8F0872DE9F04116460C46054602F04D
:10D59000CBFF02F0E2FF804602F0D5FFFE49B44225
:10D5A0000968B1F90E3088BFBDE8F081A8F1010724
:10D5B000A8F1020CDFF8E48335F9142001199A422E
:10D5C000BCBF35F91110994205DA18F8041021F0A2
:10D5D000040108F8041007FB004189B20CFB00426B
:10D5E00035F9111092B29942BCBF35F91210994227
:10D5F00005DA18F8041021F0080108F80410611C7D
:10D60000CCB2B442D8D9BDE8F0812DE9F04F85B055
:10D6100002F08AFF044602F09BFF019002F0A2FF95
:10D620000090DF48DC4A4FF0000C816902911168DC
:10D6300091F8CE3003938789C589488B94F841804F
:10D64000C11B401B1FFA81F986B26446B8F1000F76
:10D6500040F2078104EB8400C0EB8411019800EBD9
:10D66000810292F8920000EB8001C1EB80110098DA
:10D6700000EB8103C848B2F8AC100068B0F818A0FD
:10D68000B0F81AB001FB0AF1B0F810A0408A91FB83
:10D69000FAF11FFA81FAB2F8AE1001FB0BF191FB1F
:10D6A000F0F081B292F88D00002872D192F8C80093
:10D6B00006286ED04FF0000B82F8C8B092F8E70051
:10D6C000022818BF032804D092F8DA00012874D089
:10D6D000C2E082F8C9B0A94282BF8E42022082F81D
:10D6E000C80008D892F89000022802BF93F8C8003A
:10D6F000022882F8C80092F8E700032804BF92F8D5
:10D7000090E0BEF1020F06D193F8C8E0BEF1010F20
:10D7100008BF01207DD092F8C8E0BEF1020F18BF0B
:10D72000BEF1010F35D002280AD092F890000228ED
:10D7300004BF93F8CA00002802D0A94204D917E018
:10D74000B94203D9A94201D8012004E089451CD976
:10D750008E421AD8022082F8C90092F8E7E0BEF1A2
:10D76000020F17D092F890E0BEF1020F03D00CE048
:10D770008E42EFD909E093F8CAE0BEF1000F09D05C
:10D7800093F8C8E0BEF1030F18D082F8C8B082F851
:10D79000CAB061E0A2F8CCA0A2F8CE10B2F8AC00FA
:10D7A000A2F8D000B2F8AE00A2F8D200032082F8AE
:10D7B000C800012082F8CA004EE03DE0B3F8CCB0CA
:10D7C000B3F8CEE0AAEB0B0AA1EB0E010AFB0AFAB2
:10D7D00001FB01A1DDF808A0514527DCA2F8CCB07F
:10D7E000B3F8CE10A2F8CE10B3F8D010A2F8D01033
:10D7F000B3F8D210A2F8D21093F8CA10491CC9B2DB
:10D8000082F8CA10039B994238BF03200BD304212E
:10D8100000E008E082F8C8100A462146FFF746FDFE
:10D820004FF0010C18E082F8C80015E0012082F8E2
:10D83000C80082F872000FE0B3F8CC00A2F8CC0068
:10D84000B3F8CE00A2F8CE00B3F8D000A2F8D00012
:10D85000B3F8D200A2F8D200601CC4B24445FFF471
:10D86000F9AE05B06046BDE8F08F2DE9F05F4C4899
:10D8700000273C46B0F810A0408A0FFA80F902F069
:10D8800053FE054602F064FE95F84160002580468F
:10D890004FF0040B002E59D905EB8500C0EB851025
:10D8A00008EB800090F88D1000294BD190F8C8103B
:10D8B000042918BF062945D090F8E710022902D0A4
:10D8C000032909D03EE090F8C910002904BF681C64
:10D8D00060F3070404D135E090F8C910002931D075
:10D8E000017C827BC37B891ACAB2417CC91AC9B246
:10D8F0008A428EBF13460B461146828A524506D293
:10D90000591A4945A4BFB0F90210A02909DD80F8D1
:10D91000C8B090F8C90004222946FFF7C7FC0127C8
:10D9200010E090F8CA1001290CD190F8C900012824
:10D9300004BF681C60F30F2404D0022804BF681CD5
:10D9400060F31744681CC5B2B542A5D30025002E6C
:10D9500039D904F0FF0AC4F30729C4F3074405EBDF
:10D960008500C0EB851008EB800090F88D1031BB6E
:10D9700090F8C810042918BF062920D090F8E710A5
:10D98000022918BF03291AD190F8CA10012916D903
:10D99000BAF1000F06E0000004030110B29F01106D
:10D9A000D402011018BF514610D041B180F8C8B060
:10D9B00090F8C90004222946FFF778FC0127681C6B
:10D9C000C5B2B542CBD33846BDE8F09FB9F1000FE0
:10D9D00005D090F8C910012908BF4946E5D0002CB0
:10D9E000EDD090F8C910022908BF2146DDD0E6E746
:10D9F0002DE9F05F9A4691460E4607460A9D02F0D1
:10DA0000A2FD804602F0A9FD8346FE48022354464B
:10DA100000684FF0010CAA4590F8CC0098BFA8F11F
:10DA2000010215D803FB084139F9111081420BDBC3
:10DA300007F804C0002C1CBF391901F801CC94422E
:10DA4000BCBF391981F801C0611CCCB2AC42E9D924
:10DA5000ABF10301CAB2AA4594BFA8F10103BDE826
:10DA6000F09F02FB08A189B239F9111081420EDB47
:10DA700006F80AC0BAF1000F1CBF06EB0A0101F854
:10DA800001CC9A45BCBF06EB0A0181F801C00AF13E
:10DA9000010101F0FF0AAA45E3D9BDE8F09F2DE995
:10DAA000F0471C4615460F468046089E02F041FD91
:10DAB00002F053FD824602F046FDB44288BFBDE845
:10DAC000F087DFF84493AAF101034FF0000C19F836
:10DAD0000420211812F0050F07D025F814C018F8FB
:10DAE0000420002A08BF25F811C003FB00418AB2B8
:10DAF000111A19F804A089B21AF00A0F06D025F8F5
:10DB000012C03A5D002A08BF25F811C0611CCCB2D2
:10DB1000B442DCD9BDE8F0872DE9FF4F81B01D4646
:10DB20000F46804602F000FD02F003FD90F8DC1481
:10DB3000B448012900680CBFB0F90E6090F8CC60C1
:10DB400002F00BFD009002F0FEFC01460020039A5B
:10DB5000DFF8B4B2034604468446AA4298BFA1F156
:10DB6000010A29D818F802E0BEF1000F20D037F9D9
:10DB70001290B1451CDB1BF8029019F0010F10D177
:10DB800032B10BEB020E1EF801EC1EF0010F08D1B2
:10DB9000524508DA0BEB020E9EF801E01EF0010F71
:10DBA00001D0641CE4B219F0040F1CBF401CC0B2C9
:10DBB000521CD2B2AA42D5D9039AAA4239D8DDF86A
:10DBC0000090A1F1010AA9F10109CDF80090DDF85A
:10DBD000009009FB01291FFA89F918F809E0BEF144
:10DBE000000F22D037F91990B1451EDB1BF80290C7
:10DBF00019F0020F10D132B10BEB020E1EF801EC3E
:10DC00001EF0020F08D152450ADA0BEB020E9EF805
:10DC100001E01EF0020F03D00CF1010C0CF0FF0C20
:10DC200019F0080F1CBF5B1CDBB2521CD2B2AA4217
:10DC3000CDD976490870881C4B70047080F801C0FB
:10DC400005B0BDE8F08F70B592B006460020029096
:10DC500003900490059006900790089009900A9010
:10DC60000B900C9014460D460D900E900F90109056
:10DC7000119002F059FC90F8DC1401291FBF90F8B4
:10DC8000DD04012812B070BD2B4632460AA902A855
:10DC90000094FFF7ADFE2B4632460AA902A8009475
:10DCA000FFF7FDFE12B070BD2DE9F04102F03CFC23
:10DCB000044602F03EFC804654480023871C01784D
:10DCC0003A7840781144CAB2797884F8DC34084450
:10DCD000C1B284F8DD3498F8DC0401264A4D0128ED
:10DCE00014D1002A1CBF002984F8DC640ED102F094
:10DCF0001BFC02F028FCF3220021002806D96B5CF3
:10DD000013406B54491CC9B28842F8D898F8DD0416
:10DD1000012818BFBDE8F08138787978014401F016
:10DD2000FF0870B902F000FC02F00DFCFE22002199
:10DD3000002806D96B5C13406B54491CC9B2884259
:10DD4000F8D8787870B902F0EFFB02F0FCFBFD2206
:10DD50000021002806D96B5C13406B54491CC9B2E2
:10DD60008842F8D8B8F1000F18BF84F8DD64BDE828
:10DD7000F0812DE9F05F17468846814602F0D9FB15
:10DD8000064602F0D1FB054602F0CEFB02F0D1FBC5
:10DD9000044690F8DC04DFF878A04FF0000B40B99F
:10DDA00094F8DD0418B92021174802F0C7FBAAF83F
:10DDB00004B094F8DD04002808BFAAF806B096F86D
:10DDC000DC04012806BF95F8DB040028BDE8F09FBD
:10DDD0003A4641464846BDE8F05FFFF7D3BB70B511
:10DDE00092B01C4615460E46FFF796FEFFF75CFF05
:10DDF00000200290039004900590069007900890F0
:10DE0000099007E004030110B29F0110D80201102D
:10DE1000D40201100A900B900C900D900E900F9070
:10DE20001090119002F080FB90F8DC1401291FBFC4
:10DE300090F8DD04012812B070BD2B4632460AA9C5
:10DE400002A80094FFF7D4FD2B4632460AA902A887
:10DE50000094FFF724FE12B070BD2DE9F04F85B09D
:10DE60004FF00008CDF80080CDF80480CDF8088090
:10DE700002F05AFB044602F05CFB039002F068FBE0
:10DE8000064602F06FFB054694F841000022012788
:10DE90004FF002094FF0030A00285CD94FF00A0B3B
:10DEA0000DF1FF3002EB8201C1EB821106EB810123
:10DEB00091F8923003EB830CCCEB831391F88DC077
:10DEC00005EB8303BCF1000F3FD191F8E7C0BCF133
:10DED000020F18BFBCF1030F08D091F8DA30012B04
:10DEE00004BF91F8911001F800B02EE091F8CAC07B
:10DEF000BCF1000F0BD091F8C830042B91F8913091
:10DF00000CBF03F800901F5481F8B3A01DE091F8F6
:10DF1000C8C0BCF1010F18BFBCF1020F15D191F8B8
:10DF200090C0BCF1020F0CD193F8CAC0BCF1000F35
:10DF300007D0B3F8D0C0A1F8ACC0B3F8D230A1F884
:10DF4000AE3091F8911001F80090511CCAB294F8CB
:10DF500041109142A6D884F8DE84DFF858844FF04F
:10DF6000000BBA4618F80B0001281CBF0328042830
:10DF700074D11DF80B106F4621B10A2908BF07F8AC
:10DF80000B006BE00399002091F84130002B88BF13
:10DF90000BF1010262D900EB8001C1EB801105EBAE
:10DFA000810191F88DC0BCF1000F04BF91F8911070
:10DFB00091424FD194F8411001EB8102C2EB8111E3
:10DFC00006EB810900EB8001C1EB801005EB8001BD
:10DFD000EC22484602F0AEF994F84100401C84F867
:10DFE000410094F84200401C84F8420094F8DE049A
:10DFF000401C84F8DE04B9F8D000A9F8AC00B9F8E8
:10E00000D200A9F8AE00002089F8CA0018F80B0069
:10E01000012807D0032806BF042007F80B000428B6
:10E020000BD014E0032007F80B0089F8B3A00220FE
:10E0300089F8E70089F8E6A009E0022089F8B30032
:10E0400089F89000032089F8E70089F8E6A089F8AC
:10E05000D9A003E0401CC0B283429CD80BF1010060
:10E0600000F0FF0BBBF10A0FFFF47CAF0098C8F87B
:10E0700000000198C8F80400BDF80800A8F80800DE
:10E0800005B0BDE8F08F2DE9F74F002782B0BB4601
:10E090004FF0020902F048FA804602F059FA0646AB
:10E0A000C54898F84140006890F8CE5002F055FA03
:10E0B000824698F8DC04012843D1C0480088A84271
:10E0C00008D8DDE90201049AFFF726F9BB480021D0
:10E0D000418036E00025002C84BFAAF102000090A8
:10E0E0002FD905EB8500C0EB851006EB800090F87A
:10E0F0008D10002901BF90F8DA10012990F87210F4
:10E1000000291AD14178012909D80378AC4AD25C98
:10E1100012F0100F03D00522294601200BE0009ACF
:10E1200091420ADB0178A648405C10F0200F04D031
:10E13000052229460220FFF7B9F8681CC5B2A5429E
:10E14000CFD30020002C88BFAAEB090319D900EB1C
:10E150008001C1EB801106EB810191F88D2062B93D
:10E1600091F8E720022A18BF032A06D149784945C9
:10E1700003D39942BCBF791CCFB2401CC0B2A042AD
:10E18000E5D3002F1CBF0025002C84BFAAF1010796
:10E190004FF0040932D905EB8500C0EB851006EB82
:10E1A000800090F88D1029BB90F8DA10012905D174
:10E1B00090F8E710022918BF032905D190F8C8107C
:10E1C000062918BF032915D14178002908BF01236A
:10E1D00003D0B94208BF02230CD180F8C89098F848
:10E1E000DC0401280ED0042229461846FFF75EF809
:10E1F0004FF0010B681CC5B2A542CCD305B0584600
:10E20000BDE8F08F052229461846FFF74FF8F1E7E1
:10E210002DE9F04F83B0064602F086F9044602F07D
:10E2200088F9804602F094F98346634894F8417077
:10E23000006890F8CE1089000291B0F90E50A079D4
:10E240000190207A009002F088F9814602F07BF973
:10E25000824602F08CF900281CBF17200090FFF7BF
:10E260003EF994F8DB04012808BF98F8DC0407D0D5
:10E2700094F8DC0430B9DDE900213046FFF7B9F845
:10E2800084F8DC04C0B201285CD1DDE9002130460D
:10E29000FFF742F80023002F50D9A9F10208A9F195
:10E2A0000100DFF81C9100FB0AFC03EB8300C0EBCC
:10E2B00083110BEB810292F8DA0001283AD1D07A6F
:10E2C00010B1507B404535DD917A107B884214D3E4
:10E2D00036F91100A8420BDD19F801000C2920F0D5
:10E2E000040009F8010024BF20F0100009F8010023
:10E2F000481CC1B2107B8842EAD2917AC0B21FFAA0
:10E300008CFA884216D30AEB010036F91000A842B5
:10E310000BDD19F801000C2920F0080009F80100B4
:10E3200024BF20F0200009F80100481CC1B2107B76
:10E330008842E8D2581CC3B2BB42B6D394F8DC047E
:10E3400001281FD01D49002008804880FFF75DF993
:10E3500094F8DD14084384F8DD04DDE9002130463B
:10E36000FFF791FE94F8DD14084384F8DD04FFF70D
:10E370007CFA94F8DD14084384F8DD0403B0BDE8AA
:10E38000F04F6AE50D4D2888401C80B22880B0F51A
:10E39000167F84BF4FF4167028806888401C80B2B6
:10E3A000688002998842D1D3FEF7FAFF0020688086
:10E3B000CCE70000A89F011004030110D402011053
:10E3C000B29F01102DE9F04100240F460646254674
:10E3D00002F0BEF80022002E13D902EB8201C1EB3D
:10E3E000821100EB810393F88D10012905D1B3F957
:10E3F00002301D44A342C8BF1C46511CCAB2B242DF
:10E40000EBD3012F84BF95FBF7F004B2F948B0F9C4
:10E4100000108C42D8BFBDE8F081611041801E2100
:10E4200081800480BDE8F0812DE9F05F16460F463B
:10E43000054602F08DF8024600208446002D98BF64
:10E44000BDE8F09F4FF00109DFF8A8834FF0020A02
:10E4500003210CEB8C03C3EB8C1302EB830393F8C7
:10E460008D40012C04BF93F8DA40012C1DD1012FFF
:10E4700019D093F801B0B3F9024036F91BB0A4EB00
:10E480000B04B8F902B05C4504DD401C83F88E90A3
:10E49000C0B20AE0B8F904B05C4504DD401C83F862
:10E4A0008EA0C0B201E083F88E100CF1010303F0DE
:10E4B000FF0CAC45CDD3BDE8F09F2DE9F84F0546E4
:10E4C00045F25650484301140024A1EBE07007B216
:10E4D000009402F038F8064602F03FF85FEA0009BF
:10E4E000A6F102004FF01808C3B2224632D0A3EBC7
:10E4F000080000F1010EA8F1010BC7F1000A414626
:10E50000984511D802FB061080B235F910C005EB12
:10E510004000B0F902006044B842C4BF601CC4B2FD
:10E52000481CC1B29942EDD9A6450ED102FB06B0F6
:10E5300080B235F9101005EB4000B0F90200084434
:10E54000504502DD0120009004E0501C0024C2B2BE
:10E550004A45D4D30098BDE8F88F2DE9F04F99B023
:10E5600000268146032012900A2018900520119061
:10E57000039608960E2001960D9600960696179023
:10E5800005960B961E20029604960A9615900796FD
:10E5900009960F960F200D463746B0460C960E96FC
:10E5A000149001F0D5FF824601F0BEFF109001F0FB
:10E5B000C0FF139001F0C7FFDFF83CE200220EF12C
:10E5C0000E0B169012990020002960D91EF8003019
:10E5D0001BF802C016990CFB013189B239F81130D1
:10E5E00009EB4101498819440CB215998C4240F35A
:10E5F000D4800A2D80F0D18005EB8501C1EB851315
:10E600000AEB83014FF0010C81F8DAC01EF800C05C
:10E610000AF823C01BF802304B704C801EF8003003
:10E6200003EB83035B008B801BF8023003EB830357
:10E630005B00CB80714B0C8133F81030A1F8A8300F
:10E640006F4B33F81230A1F8AA30012381F88D30D6
:10E650002346FA2CC8BFFA2381F88B3081F88C301E
:10E6600081F88A30711CCEB2691CCDB24445C8BF56
:10E67000A0461BF802106B463DF911C0A445C8BF67
:10E6800023F81140401C1299C0B288429ED3501CFE
:10E69000C2B21898904295D80A2D5CD211980022E7
:10E6A000002884BF4FF01E0CEE4654D9554C1698E6
:10E6B000A15C48431E3080B239F8101009EB4000CD
:10E6C00040880844159900B2884271DD0A2D6FD246
:10E6D00005EB8501C1EB85130AEB83014FF0010BBC
:10E6E00081F8DAB00AF823C0A35C4B7048804FF47D
:10E6F00096738B80A35C03EB83035B00CB80088164
:10E7000045F6D043A1F8A83004F12903FA2833F8DC
:10E710001230A1F8AA3081F88DB0CCBFFA2303469D
:10E7200081F88B3081F88C3081F88A30711CCEB240
:10E73000691CCDB24045C8BF804633497346895CE9
:10E740003EF911408442C8BF23F81100501CC2B2E8
:10E7500011988242AAD31398052190F8DF0400286B
:10E7600030D0002E18BF0421109880F8DF1437D065
:10E77000042E03D231462846FFF724FE4146484680
:10E78000FFF79BFE18B1139890F8E004F0B36A46C7
:10E7900000212846FFF748FE28E0002CB4BF614264
:10E7A0002146149B9942C4BF791CCFB25EE7FFE7B4
:10E7B0000028B4BF41420146149B9942C4BF791C52
:10E7C000CFB2B7E73EB91798874204D31098062115
:10E7D00080F8DF1404E01098002E80F8DF14C7D111
:10E7E00004490020322208804A80888019B02846D7
:10E7F000BDE8F08FF0020110002F0100082F01008A
:10E80000182F0100032F01000E2F0100FFE76A46B9
:10E8100001212846FFF708FEE8E700002DE9F04F48
:10E82000DFF800C4DDE90959DCF800A0FC4C1E4605
:10E830009AF8A1E09AF8A0B04B4518DC9446AA4299
:10E84000D8BF9AF807800CDC06FB08C730F91770B0
:10E85000A742C8BF3C460CF1010C0FFA8CFCAC453A
:10E86000F2DD06F1010C0FFA8CF64E45E6DD9AF862
:10E87000A200EC4E844226DDDFF8ACC3BCF90000F8
:10E8800000FB0EF747FA0BF7BC421CDDA042B8BFF5
:10E89000ACF800404B45D8BF4FF6FF7C10DC10466B
:10E8A000AA4209DC3468E47903FB0404401C00B28A
:10E8B00021F814C0A842F5DD581C03B24B45EEDD2B
:10E8C0000120BDE8F08F0020BDE8F08F2DE9F001B8
:10E8D00045F25656DDE90554002C35F914C0027096
:10E8E0000CFB06FC4FEA2C46A6EBEC7C0FFA8CF6F0
:10E8F0000B70BCBFBDE8F0017047A446A24221DA0C
:10E9000035F91C70B74209DA05EB4C0838F9028C6E
:10E91000B04503DA0CF10102027013E0B74205DBE7
:10E9200005EB4C0838F9028C464505DD05EB4C0833
:10E9300038F9028C4745EDDBACF1010C0FFA8CFC89
:10E940009445DDDCA342DCBFBDE8F001704735F93A
:10E950001400B0420ADA05EB4402B2F90220B242D6
:10E9600004DA601E0870BDE8F0017047B04205DBB4
:10E9700005EB4402B2F90220964205DD05EB4402A4
:10E98000B2F902209042ECDB601C04B29C42DEDB58
:10E99000BDE8F00170472DE9FF4F91B04FF000093D
:10E9A000CDF84090CDF80090CDF80490CDF80890C7
:10E9B000CDF80C90CDF81090CDF814901E46CDF8FF
:10E9C0001890CDF81C90CDF82090CDF82490CDF87B
:10E9D00028900546CDF82C90CDF83090CDF83490A5
:10E9E000CDF83890CDF83C9030788A464200C84641
:10E9F0004F46684601F0ADFC31780020491E0029E1
:10EA0000C8BFEE465CDD0AEB40023AF91040B2F9AD
:10EA100002C040F2E7310B46A346A4450EDB35F9B0
:10EA200014208A4203DC0B461146A14602E09342C1
:10EA3000C8BF1346621C14B2A445F0DA1E9A35F919
:10EA40001C30012A35F91B2027D09A42B8BF1A463C
:10EA50005210914227DB0EEB40023EF91010B2F942
:10EA600002C035F9113035F91CC09C45AABF002100
:10EA7000518000280CDB3EF911303EF910C063458F
:10EA800004BF53882EF81130491C09B28142F2DDCF
:10EA90001099491CC9B210910CE09A42A8BF1A46BD
:10EAA00052109142D7DA139921F8189008F1010118
:10EAB00001F0FF083178401C00B2491E8142A2DCFF
:10EAC00030784FF0FF324100504601F092FC307830
:10EAD00000210028C8BF6A461DDD4FF0000C6046CB
:10EAE0000029C8BF32F911300ADD32F91040A342C3
:10EAF0000CD0401C00B28842F7DBBCF1000F05D1FE
:10EB000032F811002AF81700781CC7B2481C01B26D
:10EB100030788842E1DCC1B21098081A307015B024
:10EB2000BDE8F08F2DE9F04F87B04FF0000CDFF813
:10EB3000FC90CDF810C04FF0FF35644604AE0DF1E7
:10EB4000140809F1040A09F1080BCDF814C0012BCF
:10EB500008BF4FF0000C07D0022B04BF4FF0000C91
:10EB6000DFF8CCE010D01EE039F81C7026F81C70DD
:10EB70003AF81C7028F81C700CF1010C0FFA8CFC90
:10EB8000BCF1020FF0DB0EE03BF81C7026F81C70A5
:10EB90003EF81C7028F81C700CF1010C0FFA8CFC6C
:10EBA000BCF1020FF0DB0027002A72DDBDF910C0B6
:10EBB000CDF800C0BDF912C0CDF804C0BDF914C035
:10EBC000CDF808C0BDF916C0CDF80CC0DFF854C0B0
:10EBD000DCF800E031F91780B8F1000F30F918C007
:10EBE00000EB48060BBFB6F9026036F9026CDDF89F
:10EBF0000090DDF804900CBFDDF808A0DDF80CA053
:10EC0000B9EB0C0B48BFACEB090BBAEB060948BFDC
:10EC1000A6EB0A09D9440FFA89F90DF1180A09E09F
:10EC200019FCFFFF040301101C0301101E03011057
:10EC30002A0301102AF81790B9F1000FC4BF9EF8FB
:10EC40009F90CC4505DD9EF89E904CFA09F9B145A0
:10EC500003DDBEF99C90E14502DA641C3D46E4B256
:10EC6000012B02D0022B26D00DE0B8F1000FDFF807
:10EC7000C88614BFA8F802C0A8F800C0DFF8BCC658
:10EC800025D0ACF8026007F1010C0FFA8CF797421F
:10EC9000A0DB012C0BD9B1F90020B1F9021030F939
:10ECA000122030F911008242ACBF00250125284610
:10ECB00007B0BDE8F08FB8F1000FDFF8848614BF0D
:10ECC000A8F802C0A8F800C0DFF878C6D9D1ACF81F
:10ECD0000060D8E72DE9F05F0446DDE90B05DDF8BB
:10ECE0002880994617460E464FF0000A012802D0A8
:10ECF000022803D005E001F026FC01E001F02DFC24
:10ED0000824600204FF0FF31BAF1000F08DD34F9E0
:10ED100010208A42C8BF1146401C00B25045F6DBA5
:10ED200045F2565048430114A1EBE0708542B8BF4C
:10ED300005B20020B4F90210B4F90030024699423D
:10ED4000A4BFB4F90430994207DBB4F906308B4212
:10ED5000D8BF8D4201DA01203080AAF1020B4FF0BA
:10ED6000020CBBF1020F1EDD04EB4C0334F91C1046
:10ED700033F902EC7145A4BFB3F902E071450CDB35
:10ED800033F904EC8E45DEBFB3F904308B428D427B
:10ED900003DA26F810C0401CC0B20CF101010FFAD2
:10EDA00081FCDC45E0DBB4F90010B4F902308B42A1
:10EDB000DEBFB4F904308B428D4203DA002127F81C
:10EDC0001210521C04EB4A0131F9043C31F902CC17
:10EDD0006345A4BF31F906CC634509DB31F908CCA2
:10EDE0009C45D8BF9D4203DA26F810B0401CC0B243
:10EDF00031F9023C31F904CC6345A2BF31F9061C5C
:10EE00008B42AB4204DDAAF1010127F81210521C1B
:10EE1000002818BF002A0AD0B6F90010B7F9003050
:10EE200034F9111034F913309942B8BF002089F831
:10EE3000000088F80020BDE8F09F2DE9F74FADF500
:10EE4000296D9346044601F07EFBCDF8600A01F07F
:10EE500084FB039001F068FB0025CDF8740ACDF81F
:10EE6000704A0398CDF8A058CDF89058CDF8945832
:10EE7000CDF8B458CDF89858CDF89C58CDF8A45892
:10EE8000CDF8A858CDF8C858CDF8AC58CDF8B05842
:10EE9000CDF8B858CDF8BC58CDF8DC58CDF8C058EE
:10EEA000CDF8C458CDF8CC58CDF8D058CDF8F0589E
:10EEB00004EB4000CDF8D458CDF8D858CDF8E05840
:10EEC000CDF8E458CDF80459CDF8E858CDF8EC5811
:10EED000CDF8F458CDF8F858CDF8800ACDF8FC58A4
:10EEE000CDF80059CDF808594FF40061CDF80C5910
:10EEF00004A801F024FACDF89859CDF89059CDF82E
:10EF0000AC590020CDF8A459CDF8C059CDF894598A
:10EF1000CDF89C59CDF8A059CDF8B859DDF8601A54
:10EF2000CDF8A859CDF8B059CDF8B459CDF8CC5991
:10EF3000CDF8BC59CDF8C459CDF8C8590646074696
:10EF4000CDF86C0A0029C4BF0DF50161FE4B0FDD41
:10EF5000DDF8802A33F810C032F81020A2EB0C0242
:10EF600021F81020401CDDF8602A00B28242EFDC5C
:10EF7000039900200029C4BF0DF50561F34B0EDD98
:10EF8000DDF8702A33F810C032F81020A2EB0C0222
:10EF900021F81020401C039A00B28242F0DCEC4CB5
:10EFA0000DF67820012122680DF6642392F89F2047
:10EFB0000090CDE901120DF51D620DF511610DF501
:10EFC0000160FFF787FE20684FF002080DF67C21F4
:10EFD00090F89F00CDE9001802900DF668230DF51A
:10EFE00021620DF515610DF50560FFF773FE9DF8C3
:10EFF000780A9DF87C1A084340D12046DDF8801A33
:10F000000068B1F9001090F89F004008814235DA9D
:10F01000DDF8602ADDF8801A01EB420131F9021CAB
:10F0200081422BDADDF8701AB1F90010814225DA3D
:10F03000039ADDF8701A01EB420131F9021C81429A
:10F040001CDADDF8600A4100BF4801F077FA039846
:10F050004100BE4801F072FAB74A0020111D0B1D95
:10F0600001F1080C22F8105021F8105023F810502C
:10F070002CF81050401C00B20228F3DB9DF8642AE3
:10F08000002A1CBF9DF8680A002800F0DA800120E1
:10F09000CDE900B00DF664230DF509620DF511619F
:10F0A0000DF50160FFF777FCCDE900B80DF6682398
:10F0B0000DF50D620DF515610DF50560FFF76BFCA3
:10F0C0000020CDF8840A9DF8640A002840F38A8263
:10F0D000DDF8840A0DF50961DDF8843A31F9101084
:10F0E0000DF51160DDF86C2A30F913008142DCBFA8
:10F0F000DDF8601A491EC9B2CDF86C1A0DF5016130
:10F10000CDE90010CDF808B00DF65421081FDDF848
:10F110006C3AFFF7DBFB9DF8680A4FF00008002807
:10F1200006DC81E0DDF8880A002818BF024600D11D
:10F1300000220DF50D6030F91810803030F91800FC
:10F140008142DCBF0399491EC9B2CDF8881A0DF57A
:10F150000561CDE900100DF65C21CDF808B0081F5F
:10F16000DDF8883AFFF7B2FB9DF8506A9DF8545AD3
:10F170009DF8644A01F0E7F9012C03D1A91B401F57
:10F18000814248DC0DF1100A9DF8509A9DF8584ACA
:10F190009DF8545A9DF85C6A01F0D5F9009001F091
:10F1A000DCF9002CB8BF0024B9F1000FB8BF4FF054
:10F1B00000090099491E8D42C8BF0D46401E864277
:10F1C000C8BF0646B442DCBF614B4FF6FF7110DC8E
:10F1D0004846A94509DC1A68D27904FB0202401CA2
:10F1E00000B22AF81210A842F5DD601C04B2B44245
:10F1F000EEDDDDF8740A9DF8501A00EB870081758A
:10F200009DF8581AC1759DF8541A01769DF85C1A3C
:10F210004176781CC7B208F101000FFA80F89DF81A
:10F22000680A8045FFF67EAFDDF8840A9DF8641A0F
:10F23000401C00B2CDF8840A8842FFF649AF00F0C6
:10F24000D1B99DF8780A9DF87C1A50EA010300F0C4
:10F25000C9814FF0FF394C4600281CBF002A8DF8A9
:10F26000785A00291EBF9DF8680A00288DF87C5A3C
:10F270009DF8782A3AB101230DF51D610DF5016065
:10F28000FFF750FC81469DF87C2A3AB102230DF528
:10F2900021610DF50560FFF745FC0446B9F1FF3F1C
:10F2A0000DF5216A7ED00DF51D600DF5016130F977
:10F2B0001900B4F1FF3FCDE90010DDF8600ACDF888
:10F2C00008B0A0F10100C3B24FF000020DF65421C6
:10F2D0000DF5256056D0FFF7F9FA3AF914000DF54F
:10F2E0000561CDE9001003980DF65C21401EC3B204
:10F2F000CDF808B00022081FFFF7E8FA9DF8506A21
:10F300009DF8544A9DF8645A01F01DF9012D04D16D
:10F31000A11B401F814200F365819DF85C1A9DF896
:10F32000540ACDE900019DF8583A9DF8502A04A9E5
:10F33000DDF8940A0EE000001E0301102203011004
:10F34000260301102A030110DEBC01101EBD0110AE
:10F3500004030110FFF762FA002800F04381DDF892
:10F36000740A9DF8501A00EB87007F1C81759DF888
:10F37000581AC1759DF8541A01769DF85C1A4176A9
:10F3800000F030B9FFF7A2FACDE900B80DF6682316
:10F390000DF50D620DF515610DF50560FFF7FBFA32
:10F3A000002400E093E09DF8680A002840F31A81E9
:10F3B0000DF50D60324630F91410803030F914002C
:10F3C0008142DCBF0399491ECEB20DF50561CDE93E
:10F3D00000100DF65C213346CDF808B0081FFFF78A
:10F3E00075FA9DF850AA9DF8549A9DF8648A01F028
:10F3F000AAF8B8F1010F04D1A9EB0A01401F81421C
:10F400003DDC9DF85C1A9DF8540ACDE900019DF899
:10F41000583A9DF8502A04A9DDF8940AFFF7FEF93E
:10F42000A0B3DDF8740A9DF8501A00EB87008175CF
:10F430009DF8581AC1759DF8541A01769DF85C1A0A
:10F440004176781CC7B29DF8500A9DF8542A904224
:10F45000D8BF0DF5196104DC0D54401C00B2904278
:10F46000FADD9DF8580A9DF85C1A8842D8BF0DF560
:10F470001B6204DC1554401C00B28842FADD601C9B
:10F4800004B29DF8680A844292DBABE0FFE777B9EB
:10F490009DF8500A9DF8543A9842DCBF01220DF5C0
:10F4A000196104DC0A54401C00B29842FADD9DF850
:10F4B000580A9DF85C3A9842DCBF01210DF51B62A9
:10F4C000DDDC1154401C00B29842FADDD7E7B4F1FC
:10F4D000FF3F7DD03AF914000DF50561CDE900102C
:10F4E00003980DF65C21401EC3B2CDF808B000228F
:10F4F000081FFFF7EBF90126CDE900B60DF66423EE
:10F500000DF509620DF511610DF50160FFF743FA84
:10F510009DF8640A0024002864DD0DF5016A0DF5EC
:10F5200019680DF51B690DF509600DF5116130F9CC
:10F53000140031F91410DDF86C2A8842DCBFDDF8C4
:10F54000600A401EC0B2CDE900A1CDF808B0034664
:10F55000CDF86C0A0DF65421081FFFF7B7F99DF896
:10F560005C1A9DF8540ACDE900019DF8583A9DF8BF
:10F57000502A04A9DDF8940AFFF750F948B3DDF8E2
:10F58000740A9DF8501A00EB870081759DF8581A8F
:10F59000C1759DF8541A01769DF85C1A4176781C65
:10F5A000C7B29DF8500A9DF8541A884205DC08F845
:10F5B0000050401C00B28842F9DD9DF8580A9DF8C1
:10F5C0005C1A884208DC09F80050401C00B201E0D7
:10F5D00008E03CE08842F6DD601C04B29DF8640A55
:10F5E0008442A0DBDDF8602A039900204A43002A08
:10F5F000C8BF04AB0FDDDDF8941A33F810C031F842
:10F60000101001EA0C01DDF894CA2CF81010401C0F
:10F6100000B28242EFDC9DF8780A9DF87C1AC8425D
:10F6200003D1A9494FF619400880DDF8601A00207F
:10F630000029C4BF0DF51962A44B2FDD115C01290F
:10F6400020D0DDF8801A31F81010D9B120E09DF8F3
:10F65000500A9DF8541A884205DC08F80060401CE6
:10F6600000B28842F9DD002FB6D19DF8580A9DF806
:10F670005C1A8842B0DC09F80060401C00B2884285
:10F68000F9DDA9E7DDF8801A31F8101023F8101021
:10F69000401CDDF8601A00B28842CFDB03990020DD
:10F6A0000029C4BF0DF51B61894A12DD0B5C012BDB
:10F6B00004D0DDF8703A33F810302BB9DDF8703A29
:10F6C00033F8103022F81030401C039B00B29842EF
:10F6D000ECDBDDF8740A47750DF69C2DBDE8F08F64
:10F6E0002DE9F04F89B0044600F01EFF054600F0FA
:10F6F0002FFF4FF0000B024605F11600CDF800B0C9
:10F70000CDF804B0CDF808B0CDF80CB0CDF810B0FD
:10F71000CDF814B0CDF818B00790687D4FF0FF3ADF
:10F720000121D846D146089002283FD94FF0000C5D
:10F73000002851DD67480021002CC4BF079B03EB64
:10F740008C032BDD01EB8105C5EB811502EB8507F1
:10F7500097F8DA60012E1DD13DF81160D6B9DDF8B9
:10F760001CE012F825607D781EF82CE0B6459CBFA1
:10F7700093F802E076450DD85E78B54224BFDE7876
:10F78000AE4207D3B7F90250854203DD2846012572
:10F790002DF81150491C09B2A142D3DB0CF1010034
:10F7A0000FFA80FC08988445C4DB15E00020002C8B
:10F7B000C8BF6B4610DD00EB800CCCEB801C02EB6D
:10F7C0008C0C9CF8DAC0BCF1010F08BF23F81010B4
:10F7D000401C00B2A042EEDB0020002CC8BF6B46EC
:10F7E0001ADD33F81010012912D100EB8001C1EBB2
:10F7F000801102EB8101B1F90210594504DDD846B0
:10F80000D1468B46824603E08845BCBF8846814688
:10F81000401C00B2A042E4DB0021002CCEBF00203F
:10F8200009B0BDE8F08F514518BF494507D001EB3D
:10F830008103C3EB811302EB830383F8DA00491CD5
:10F8400009B2A142EFDB09B0BDE8F08F70B50C46FC
:10F8500000F06AFE064600F07BFE054600F07DFEE5
:10F860000023002C86BF0021801E70BD03EB8302A5
:10F87000C2EB831205EB820292F8DAC0BCF1000FF2
:10F8800018D092F801C0BCF1020F01D3844511DDFC
:10F89000B2F880C0BCF1030F02D282F8DA1009E09E
:10F8A00096F8DCC4BCF1010F04BF92F883C0BCF130
:10F8B000010FF2D05A1CD3B2A342D7D370BD084671
:10F8C000022998BF70470BE71C030110DEBC011032
:10F8D0001EBD011019FCFFFF002808D0002906D02A
:10F8E000002B04D08B4202D8194600F082BD70472D
:10F8F0002023002219461148EEE7104870472020C7
:10F900007047F0F793BEF0F795BEF0F796BEF0F7AC
:10F9100099BEF0F798BE30B4144600280CD00029E8
:10F920000AD0002C08D0002B06D08B4204D82146E8
:10F9300030BC1A4600F00DBD30BC70475EBD0110F2
:10F9400030B41D46029B144658B101280DD0022840
:10F9500011D0032813D1C8B22A46214630BC00F08A
:10F96000ACB830BCC8B200F01BB8C8B2AAB22146CD
:10F9700030BC00F030B830BC084600F071B830BC84
:10F98000704705A070470420704709207047052084
:10F9900070477047704700004E3933300000000058
:10F9A00010B504466348644904700020088020466E
:10F9B00000F0DAF8204600F0CFF8204600F0D0F84A
:10F9C000204600F0C5F8204600F0BEF82046BDE80D
:10F9D000104000F0CDB870B50446564815460E46A6
:10F9E000007865280FD1062C0DD15349B1F90000DC
:10F9F000421C08D0401C00B20880C62803DBE01F70
:10FA00000880FFF77EFF072C29D2DFE804F0040A04
:10FA100010161C28220029463046BDE8704000F030
:10FA2000A4B829463046BDE8704000F096B8294693
:10FA30003046BDE8704000F094B829463046BDE835
:10FA4000704000F086B829463046BDE8704000F0AE
:10FA50007CB829463046BDE8704000F029BA70BD38
:10FA600070B5040015D1FFF748FF0078334DC0F39F
:10FA700040002870FFF741FF0078C0F38001304854
:10FA800001702A780A4304D12B49501E0880FFF7E1
:10FA900038FF204600F06AF8204600F05FF8204664
:10FAA00000F060F8204600F055F8204600F04EF8CF
:10FAB0002046BDE8704000F00EBB2DE9F0411D4628
:10FAC00016460F4604000ED11A4932201D4A08700E
:10FAD000194900200880062111701949087017493A
:10FAE0000870FFF705FF2B4632463946204600F0E6
:10FAF0003EF82B4632463946204600F030F82B4679
:10FB000032463946204600F02EF82B46324639461A
:10FB1000204600F020F82B4632463946204600F0B9
:10FB200016F82B46324639462046BDE8F04100F033
:10FB3000E8BA00002F030110300301103203011056
:10FB4000330301102E030110704770477047704750
:10FB500070477047704770477047704770477047ED
:10FB600070477047704770477047704770477047DD
:10FB7000002164281AD0652818D1FF4B002201EB20
:10FB80004100491C23F8102003EB40000229428069
:10FB90008280F4DBF94842700270C2828282C270B5
:10FBA000F7480280F448123800F0C4BA704710B524
:10FBB000FFF7A3FEF14944888C808388CB80C288FC
:10FBC0000A81008948818A81C88122440A821844B6
:10FBD000488210BD70B5E9480D46144681898D42B2
:10FBE00016D3018A8D4213D8C1898C4210D3408A22
:10FBF00084420DD8FFF781FE0646FFF77EFE0146E0
:10FC0000042070704D818C81BDE87040FFF77DBE8F
:10FC100070BD70B50546FFF770FED84CE078401C0B
:10FC2000C1B2E17021290AD9A078012807D1E28A5E
:10FC3000A18A2846FFF7CEFF0020E070A07070BDBB
:10FC40002DE9F05FDFF834930446484699F8001038
:10FC50004078C94FDFF8288300266FF00B0B4FF078
:10FC6000010A00EB4005C9B348464FF0020C8289F7
:10FC7000437801209843012957D0022953D1617854
:10FC800000296CD001294ED1D646B8F90010CB46D8
:10FC900000EB400A27F8151007EB450907EB4A036C
:10FCA000B9F802C05C88BCEB040201D5A4EB0C02DD
:10FCB00012B2642A7DDAB9F804209B88B2EB030CF7
:10FCC00001D5A3EB020C0FFA8CF2642AF2DA37F9B1
:10FCD0001A30D946CA1A6DD55C1AB4E0FFE76078CD
:10FCE000002820D1A8F8006027F81560608800F08F
:10FCF000D9FD5E46594600F04CFFA24900F01AFEBD
:10FD000000F0B0FD07EB45056880A08800F0CAFD53
:10FD1000314600F03EFF9C4900F00CFE00F0A2FDD1
:10FD2000A88089F800A0BDE8F09F61780129FAD188
:10FD300007EB45014B88934261D3B9F810209342F9
:10FD40005DD88988B9F80E20914258D3B9F81220AD
:10FD5000914254D889F8010089F800C0E3E71046C1
:10FD600000F0A0FD8246608800F09CFD5D4659468B
:10FD700000F00FFFDFF80C82414600F0DBFD51463A
:10FD800000F0A4FD3BD3B9F8100000F08BFD8246D3
:10FD9000608800F087FD294600F0FBFEC34641461F
:10FDA00000F0C8FD514600F091FE28D3B9F80E00CE
:10FDB00001E076E046E000F075FD8246A08800F0A4
:10FDC00071FD294600F0E5FEDFF8BC81414600F0F8
:10FDD000B1FD514600F07AFD11D3B9F8120000F0E0
:10FDE00061FD8246A08800F05DFD294600F0D1FE4D
:10FDF000414600F09FFD514600F068FE02D289F8AE
:10FE0000006090E7608800F04DFD294600F0C1FEDB
:10FE1000594600F08FFD00F025FD014699F80100DC
:10FE200000EB400007EB40067180A08800F03AFD2F
:10FE3000294600F0AEFE414600F07CFD00F012FDC8
:10FE4000B08070E7144624B2032C2ADDF246002A63
:10FE500000D55A1A11B2212923DAFFF74EFD0446C4
:10FE6000FFF74BFD99F8013001462AEA030289F8B1
:10FE70000120A8F8006089F800600420607002EB9F
:10FE8000420007EB400042884A81808888813E809A
:10FE90007E80BE80FE803E817E81BDE8F05FFFF700
:10FEA00034BDA8F8006027F815608BF801003AE728
:10FEB0002DE9F05F814604460A20FFF76BFD2178AB
:10FEC0000B20FFF767FD61780C20FFF763FD60886A
:10FED00000F0E8FC6FF00B0A5546514600F059FE61
:10FEE000284900F027FD00F0BDFC81B20D20FFF78E
:10FEF00051FDA08800F0D6FC294600F04AFE2249B8
:10FF000000F018FD00F0AEFC81B20E20FFF742FDBC
:10FF1000E1880F20FFF73EFD21891020FFF73AFD11
:10FF200061891120FFF736FDA1891220FFF732FD0C
:10FF3000DFF84CB0BBF8000081B21320FFF72AFDB8
:10FF40001420EE21FFF726FD104D15202978FFF72C
:10FF500021FD287865287DD14FF00008464609EB41
:10FF6000061528780F2875D0688800F09BFC51464C
:10FF700000F00FFE03490BE090BD011034030110A7
:10FF8000300301100000B444000020452F0301108D
:10FF900000F0D0FC00F066FC87B2A88800F082FC7C
:10FFA000514600F0F6FD5D4900F0C4FC00F05AFC3B
:10FFB000791E80B2A12903D340F2FE418F4209D9B4
:10FFC00039460820FFF7E6FC69880920FFF7E2FCC4
:10FFD000AA211AE038430FD008F10100C0B28046D0
:10FFE000012816D901460820FFF7D4FCBDE8F05FD0
:10FFF000CC210A20FFF7CEBC39460820FFF7CAFC07
:020000021000EC
:1000000069880920FFF7C6FCBB210A20FFF7C2FC64
:1000100000E02C46761C0A2EA1DBFFF76EFC06469C
:100020003F480025007840B149463E4800F08EF830
:1000300018B101280ED002280FD03B4800780028C4
:1000400008D0B07B400901280DD0022802D1607889
:10005000364E00E03EE050B10CE002207070BDE88A
:10006000F05FFFF752BC2046BDE8F05FE8E5F570B1
:10007000ABF800502078012803D1607808B9ABF8BC
:100080000050607820B1012822D0022822D11BE044
:100090000120B070F570608800F004FC55465146B0
:1000A00000F077FD224900F045FC00F0DBFBB08258
:1000B000A08800F0F7FB294600F06BFD174900F01F
:1000C00039FC00F0CFFBF0822046BDE8F05FA0E5F0
:1000D000F570B57027E670B5134D287808B1FFF7B5
:1000E00066FD0F4C0F492078087010B1084600F0EB
:1000F00021F829782078BDE8704001430620FFF7F9
:1001000002BC10B5002808D1FFF7F7FB202181734E
:100110000549002008700349087010BD0000204503
:10012000320301107EBD01103303011034030110AE
:100130000000B4440178002907D00021418040F23A
:10014000A311C18140F24C41018270472DE9F05F5B
:10015000044608780027DFF8B0810D46012843D116
:100160006878DFF8A8B1DFF8A8916FF00B0618B136
:1001700061880129F3D133E0688800F093FBB2462F
:10018000314600F006FD594600F0D4FB00F06AFB52
:1001900086B2A88800F086FB514600F0FAFC5D4963
:1001A00000F0C8FB00F05EFB81B2A6F2F910B0F5DA
:1001B000D77F19D840F63310814215D9A680E18047
:1001C00026816181012060801420FFF7E3FB6188B4
:1001D0001620FFF7DFFB88F80070A9F800704FE0E9
:1001E000022802D0012868D088E0688800F05AFB15
:1001F000314600F0CEFC594600F09CFB00F032FB8B
:100200001FFA80FBA88800F04DFB314600F0C1FCCE
:10021000404900F08FFB00F025FB1FFA80FAE088D0
:100220006189401AA0811520FFF7B4FB6188162070
:10023000FFF7B0FBB9F800004E4681B21720FFF778
:10024000A9FBA1891820FFF7A5FB454698F80010E7
:100250001920FFF79FFB2878012809D0B4F90C007A
:10026000B4F90E1088420EDDB4F9101088420ADA93
:10027000B6F900003C2801DD2F7001E00120287054
:100280006088BDE8F09FA4F808B05146A4F80AA021
:100290001520FFF77FFB61881620FFF77BFB308876
:1002A00081B21720FFF776FBA1891820FFF772FBB8
:1002B00029781920FFF76EFBE2E798F80000E8B113
:1002C000B9F900004D46002818DD3C2816DA678091
:1002D000A78188F8007002211620FFF75BFB2888B1
:1002E00081B21720FFF756FBA1891820FFF752FBB8
:1002F000FF211920FFF74EFB0220C2E76780A7818C
:1003000088F800703846BCE74C0301100000B44484
:1003100030030110000020450446AFF30080204662
:10032000EFF7B0FF7047000001491820ABBEFEE7B1
:10033000260002004DF2BF4CC1F2000C60474DF2A6
:10034000775CC1F2000C60474DF6074CC1F2000C1F
:1003500060474DF2354CC1F2000C60474DF2ED3C68
:10036000C1F2000C60474FF64D3CC1F2000C6047F3
:100370004FF6753CC1F2000C60474FF6C52CC1F238
:10038000000C60474EF2416CC1F2000C604741F630
:100390006F3CC1F2000C60474DF6537CC1F2000C7B
:1003A00060474FF61F3CC1F2000C604745F67F7C6A
:1003B000C1F2000C60474DF6F16CC1F2000C6047D1
:1003C0004DF6315CC1F2000C60474DF6AF5CC1F2F6
:1003D000000C604740F2590CC1F2000C604740F23B
:1003E000BF1CC1F2000C604740F6911CC1F2000C2A
:1003F00060474DF2235CC1F2000C60474CF2295C6F
:10040000C1F2000C60474CF2235CC1F2000C604763
:1004100043F62F7CC1F2000C60474EF2CB0CC1F2C8
:10042000000C60474EF2012CC1F2000C604746F20E
:10043000050CC1F2000C604746F2150CC1F2000C2D
:10044000604746F20B0CC1F2000C60474DF6A57CEC
:10045000C1F2000C60474EF2352CC1F2000C60472F
:100460004CF26B5CC1F2000C60474CF2192CC1F2EB
:10047000000C60474CF2015CC1F2000C60474CF28A
:100480000F5CC1F2000C604741F6595CC1F2000CF0
:10049000604741F6455CC1F2000C604741F6835C61
:1004A000C1F2000C60474EF2894CC1F2000C60476B
:1004B0004EF6693CC1F2000C604740F23B4CC1F281
:1004C000000C60474CF2E11CC1F2000C60474CF29A
:1004D000FD4CC1F2000C604741F64F5CC1F2000CCC
:1004E00060474EF20D0CC1F2000C604740F6473CED
:1004F000C1F2000C604740F6573CC1F2000C604767
:1005000041F6733CC1F2000C60474EF6055CC1F247
:10051000000C60474AF2553CC1F2000C60474EF6B1
:100520000B0CC1F2000C604745F6157CC1F2000CC3
:10053000604745F6397CC1F2000C60474DF2335CF0
:10054000C1F2000C604745F6657CC1F2000C6047C3
:1005500045F6277CC1F2000C604745F66D7CC1F280
:10056000000C604745F64F7CC1F2000C604746F234
:100570005D0CC1F2000C60472DE9F0010246154800
:100580000F468446056B9CF806309CF80840002D09
:1005900008BFA34219D0C67917464FF0000C002EB1
:1005A000C8BF0D4D11DD0020002B08DD15F90080BE
:1005B000401C834231F8188022F8028BF6DC0CF1E3
:1005C000010C01EB4401B445EDDB3846BDE8F00118
:1005D0007047000020000110BC0301102DE9F0411C
:1005E0001D4616460F468046069CF2F762FD2146E0
:1005F0002846F2F7E0FD3A4631464046F2F738FE2B
:10060000BDE8F041F2F768BD2DE9F0411D46164600
:100610000F468046069CF2F74CFD0120F2F7DDFD07
:1006200021462846F2F7C7FD3A4631464046F2F7E2
:100630001FFE0020F2F7D1FDBDE8F041F2F74CBDFE
:10064000002B08BF704730B41CB2DDF808C0BCF105
:10065000000F13D04FF0000C002A9CBF30BC704735
:1006600031F91C5005EB5305B5FBF4F520F81C508F
:100670000CF1010C6245F3D830BC70470023002A0E
:100680009CBF30BC704731F913C09CFBF4FC20F8D0
:1006900013C05B1C9A42F6D830BC7047491058BF53
:1006A000C1F140415B1058BFC3F140438B42EFF3AF
:1006B0000080704751EA030C17D41CF5801F58BF07
:1006C000BCF5801F00F10680994218BF704708BF33
:1006D0009042704707D711F5801F58BF13F5801F50
:1006E00019D499427047894270471CF5801F08D57C
:1006F000BCF5801FF7D58B4218BF704708BF8242F8
:1007000070474FF4001C1CEB410F38BF1CEB430F2C
:1007100001D28B42704770B500F008F8922449006E
:100720004FF000514FF08053FFF7B8BF0EF1020EAB
:100730002EF0030E5EF8046B364205D4012A43EB1B
:10074000030515F5001F12D8012841EB010C1CF51B
:10075000001F0CD80ED14FEAD17C15F5001F0CEB11
:100760004C0C0CF1020C08BF4CEBD37C04E04FF0B6
:10077000080C01E04FEAD37C0CEB4C0526FA05F699
:1007800006F00706B6F1040C06D20EEB860CBDE8A7
:1007900070404CF0010C6047DFE80CF0090B0202DE
:1007A0004FF000414FF00000A1F5002170BD194647
:1007B0001046012851EB010418BFD4F5001484BF82
:1007C000002001F0004170BD0808A0F500114FEABB
:1007D0003101704753EA010C17D41CF5801F58BF34
:1007E000BCF5801F00F106808B4218BF704708BF20
:1007F0008242704707D713F5801F58BF11F5801F3D
:1008000019D48B4270479B4270471CF5801F08D556
:10081000BCF5801FF7D5994218BF704708BF9042BA
:1008200070474FF4001C1CEB430F38BF1CEB410F0B
:1008300001D2994270470FB40CBC03BCFFF76BBFE9
:10084000014800F074B900BF0000C07F401058BFDD
:10085000C0F14040491058BFC1F140418142EFF31F
:1008600000807047C10DD1F19E0206DB4FEA0023E4
:1008700043F0004323FA02F07047004207D54FEAE5
:100880004001B1F1FE4F02D24FF00000704710B5A9
:1008900000F0D1F849922480002070476FEA2000D0
:1008A00070470000B0FA80F310FA03F2C3F19D0321
:1008B0000AD0D90501EB1220530638BF704700F16A
:1008C000010008BF20F001007047000050EA010C51
:1008D00000F113801CF5000F58BFBCF5000F01D4C8
:1008E0008842704707D710F5000F58BF11F5000F69
:1008F00015D488427047894270471CF5000F04D513
:10090000BCF5000FF7D5814270474FF0807C1CEB9F
:10091000400F38BF1CEB410F01D28142704710B528
:1009200000F089F8922449004FF000504FF08051B8
:10093000FFF78CBF4FF47F0C1CEAD0121EBF1CEADD
:10094000D11392EA0C0F93EA0C0F00F0478090EA63
:10095000010F48BF42F480724FF0004C4CEA002077
:100960004CEA012102EB0302A0FB0113A2F50002F5
:10097000002918BF43F001035B0028BF4FEA33038F
:1009800042EB22425FEA132C4CEBC2502EBFBCEB71
:10099000436FB2F57C0F70474FEA036CBCF1004F18
:1009A00008BF20F00100B2F57C0F38BF70470BD5AF
:1009B00082F0FF0212F5803FC8BF704700F1C040CF
:1009C000D8BF00F00040704700F5000C5FEA4C0C07
:1009D00048BF7047B0F1C04000F073B890EA010F13
:1009E0000CEAD11348BF42F48072624538BF6345B8
:1009F00004D280EA010000F00040704710B500F01A
:100A00001AF800BF8900013E00F007B800F009B8ED
:100A10005FEA410C5FEA1C6C08D080EA010000F03C
:100A200050B85FEA400C5FEA1C6CF6D14FF0004012
:100A3000A0F5800070470EF1020E2EF0030E5EF856
:100A4000044B244204D44FEA4102B2F17F4F11D843
:100A50004FEA4003B3F17F4F0CD80ED14FEAD07C60
:100A6000B2F17F4F0CEB4C0C0CF1020C08BF4CEBBD
:100A7000D17C04E04FF0080C01E04FEAD17C0CEB94
:100A80004C0324FA03F404F00704B4F1040C06D276
:100A90000EEB840CBDE810404CF0010C6047DFE821
:100AA0000CF0070802024FF00040A0F5800010BDD6
:100AB0000846420018BFD2F1807288BF00F00040A3
:100AC00010BDFF2141EAD050C005704751EA000C2B
:100AD00000F113801CF5000F58BFBCF5000F01D4C6
:100AE0008142704707D711F5000F58BF10F5000F6E
:100AF00015D481427047894270471CF5000F04D518
:100B0000BCF5000FF7D5884270474FF0807C1CEB96
:100B1000410F38BF1CEB400F01D28842704780EA7A
:100B2000010081EA000180EA0100FFF7F8BE0CF045
:100B30000F03092B08BF082000F051800A2B0BD0AF
:100B4000082B18BF704708BF1CF0400F0AD04FF0A9
:100B500000004FF0000170471CF0400F18BF4FF02D
:100B6000004070471CF0100F08D020F0704300F0D8
:100B70007F4242EAD3014FEA4370704700F0604081
:100B800021F07F4242EA000201F07F4040EA7270A9
:100B900070474FF0FF0212EAD0521CBF92F0FF03E1
:100BA0008B42C2BFD14200EBC1507047002A0AD02D
:100BB000002B0BD0002900F00040A4BF40F0FE4005
:100BC00040F40000704700F00040704743024FF0CF
:100BD0000B0C18BF4CF0806C7FF432AE70471CF4E5
:100BE000801F11D01CF4E02F03D06FEACC314900F4
:100BF00070474FF04050EFF3008222F0704242EA1B
:100C0000000282F3008870474FF000007047000038
:100C100010E000E000E100E000ED00E0000007006F
:100C20000000004000100040003000400040004044
:100C300000500040006000400080004000900040F4
:100C400000A0004000C0004000000030842F0110D0
:100C50001C02000000010000800000008002000073
:100C6000000800000008000000080000000100006B
:100C700000010000680000006800000000000000A3
:100C80000001000068000000680000000000000093
:100C9000499A0000B39A00001D9B00008D9B000044
:100CA0004F8B00004F8B00004F8B00004F8B0000DC
:100CB0004F8B00004F8B00004F8B00004F8B0000CC
:100CC0004F8B00004F8B00004F8B00004F8B0000BC
:100CD000C3920000E7920000538B00005193000084
:100CE000759300004F8B00002FA90000F1A90000B0
:100CF000DD9D0000219E00005D9E0000AF9E000073
:100D00000B930000F79E00004F8B00002D93000016
:100D10008DA60000B9930000658B0000F18B0000E8
:100D20004F8B0000E38C0000F98C0000578D000011
:100D3000339200004F8B00003392000009AA00009C
:100D40004F8B00004F8B00004F8B00004F8B00003B
:100D5000D79300004F8B000077A000003D9F00005C
:100D60003D9F00007BA000001DA100002FA10000FE
:100D700041A100005FA10000BFA10000E9930000B5
:100D800057940000999400009B950000839F0000F9
:100D9000E59500000D97000049970000519600006E
:100DA000BF9F000025A0000063970000F997000096
:100DB0006B9800006B980000D7A000004F8B0000DC
:100DC0004F8B00004F8B00004F8B00004F8B0000BB
:100DD000A79800004F8B0000F5A2000037A3000089
:100DE000CDA100000BA20000FB9800000F9C0000AA
:100DF000FB98000055990000A9990000F1990000A6
:100E00001D9A00004F8B00004F8B00004F8B00009D
:100E1000FF220000B3230000032400004F24000041
:100E20004F8B00004F8B00004F8B00004F8B00005A
:100E30004F8B00004F8B00004F8B00004F8B00004A
:100E40004F8B00004F8B00004F8B00004F8B00003A
:100E50004F8B00004F8B0000D78D0000998E000053
:100E60009D8F00004B9000002F9100004F8B0000E1
:100E70004F8B00004F8B00004F8B00004F8B00000A
:100E80004F8B00004F8B00004F8B00004F8B0000FA
:100E90007BA30000C1A300001FA4000085A40000E4
:100EA000FFA40000D7A5000063A30000A5A60000D2
:100EB0001FA700000FA800009FA700004F8B000095
:100EC00029A800004F8B00004F8B00004F8B0000C3
:100ED0004F8B00004F8B00004F8B00004F8B0000AA
:100EE000979C0000E79C00004F8B0000059D0000D0
:100EF0006D9D00004F8B0000BF9C00004F8B0000D9
:100F00004F8B00004F8B00004F8B00004F8B000079
:100F1000000000000000000000000000402C010064
:100F2000802C0100C02C0100002D0100402D01008B
:100F3000802D0100C02D0100002E010000000000E6
:100F400000000000402E010000000000802E010083
:100F5000181A1C0304090D0E004B0051A056010382
:100F6000040608090B0D0E105004800AB00D801302
:100F70005019801C80228028802B8031800AB00D7F
:100F8000801C8028802B0000682F010000000010CA
:100F90006CFE0000E0210000D42D020000000110D2
:100FA0005003000084210000482E0200500301106D
:100FB0004CBA0000FC210000F0B4FB4EDDE905C492
:100FC0003668049DB66916F0010F04D01F464B1B0E
:100FD000CD1BDBB2EDB216F0020F06D06746A2EBD6
:100FE000040CD21B0CF0FF0CD4B216F0040F08D086
:100FF00080F800C04A1B84704270C91AC170F0BCEE
:1010000070470370857080F801C0C470F0BC7047F1
:101010002DE9F043164601FB06F90D46014685B061
:101020001F464A46E1480DF0E1F9E04C0DF01DFB8A
:101030004FF0000818B105F07EFF01281AD00DF01E
:1010400014FB18B105F077FF082842D0B7F5805F90
:101050001CBF0020B9F1000FDCBF05B0BDE8F08374
:101060002156794309132154401C8145F8DC05B011
:10107000BDE8F08300210B46002ECEBFDFF828C369
:1010800005B0BDE8F0830020002D1CDDDCF8002059
:1010900092F83E919945DCBF92F83F914B450CDCAC
:1010A00092F83C918145DCBF92F83D21904204DCEE
:1010B00062567A431213625401E004F80180401C26
:1010C000491CA842E2DB5B1CB342DCDB05B0BDE897
:1010D000F083AE428CBF701E681EC2B2B54234BFF0
:1010E000681E701EC1B20420CDE90002002303A8CF
:1010F0000292FFF761FF00210A46002EDCBF05B017
:10110000BDE8F0830020002D19DD9DF80D309342DD
:10111000DCBF9DF80F309A4209DC9DF80C30834209
:10112000DEBF9DF80E30984204F8018003DD63565F
:101130007B431B136354401C491CA842E5DB521C33
:10114000B242DFDB05B0BDE8F0832DE9F0411C467B
:1011500015460E4607460DF08DFA214628460DF03D
:101160008EFA0623914A314638460DF08DFABDE8D5
:10117000F0410DF08EBA8E4AC2E90301704730B4D7
:10118000B3F5805F11D04FF0000C002A9CBF30BC3B
:10119000704731F91C405C43241320F81C400CF1CB
:1011A000010C6245F5D830BC7047884204BF30BCA2
:1011B0007047520030BC0DF019B92DE9FF4F7D4842
:1011C00093B04FF0000906787B4890F800A076486D
:1011D000006890F8ABE0B0F9A810129190F8AA005E
:1011E000CDF80890CDF81C90CDF8309011900020EB
:1011F000CDF80090CDF80490CDF80C90CDF810907B
:10120000CDF81490CDF81890CDF82090CDF824901A
:10121000CDF82890CDF82C90CDF83490CDF83890BA
:10122000CDF83C9001460746844602461090BAF13C
:10123000000F54D94FF0000845464446002E34D9DB
:1012400002FB064B149830F91B000028B4BFC0F114
:10125000000B8346DE4524DAA8EB00080FFA88F875
:101260000028ACBF8346C0F1000B5944A8BF84449A
:1012700005DA05F10105C0F1000BEDB25F44DDF8C0
:1012800054B0BBF1010F0CD10028B8BF4042DDF8CB
:1012900048B0584505DA3DF812B00BF1010B2DF8B6
:1012A00012B0601CC4B2B442CAD3B9F1000F07D166
:1012B000B8F1000F04DD1198A842D8BF4FF0010922
:1012C000B54208BF4FF002093DF91200B0EB5A0FCA
:1012D000C4BF01201090501CC2B25245AAD3344C56
:1012E000E06A421A48BF0A1A344DA5FB0165EE08B0
:1012F0000125964287BF219A15700022219E98BF32
:101300003270B9F1010F2CD0B9F1020F08D21A785E
:10131000032A01BFC4E90B1C022017B0BDE8F08FFF
:10132000B9F1020F25D0B9F1010F2AD0002808BF6A
:10133000C4E90B1C0FD01A78002A1CBF209A002A7F
:1013400009D000EB400088423FBFC4E90B1C0320DA
:1013500017B0BDE8F08F159828B31098012839D040
:1013600041E0226B002A1CBFBCF1000FB2EB470F1B
:10137000CDD202201870C4E90B1C17B00320BDE8C1
:10138000F08F1878022838BF1D70C4E90B1C18783C
:1013900002281BD0209898B1BCF1000F18BFBCEBFD
:1013A000470F13D90EE01EE0DC010110F44C0110D0
:1013B00094010110CA000110CB000110CDCCCCCC9F
:1013C000674503D217B00220BDE8F08F17B00320A5
:1013D000BDE8F08F187800281FBFC4E90B1C05205A
:1013E00017B0BDE8F08FC4E90B1C17B00020BDE8B2
:1013F000F08FFF4900200A7A12F0060F18BF4869E3
:1014000070470020FA49097A11F0060F18BFF94811
:1014100070472DE9F007002491B0002B9EBF11B05A
:10142000BDE8F0077047561E4FF000086F464FF0BA
:10143000000C002E16D904FB02C531F8159001EB03
:1014400045056D88A9EB05052DB227F81C500E3512
:101450001C2D98BF27F81C800CF1010C1FFA8CFC86
:10146000B445E8D304FB02FC012A20F81C804FF0AD
:10147000010C13D904FB02C507EB4C0A00EB45092C
:101480003AF802AC39F8029C0CF1010CA9EB0A09FC
:101490001FFA8CFC20F815906245EBD804F1010C82
:1014A0001FFA8CF49C42C2D311B0BDE8F00770471C
:1014B0002DE9F04FADF6040D03FB02FA4FF0000CDE
:1014C000E946BAF1000F84BF0026CB4D13D931F99C
:1014D0001C4004F10F071E2F98BF29F81C6004D987
:1014E00035F81C70E41B29F81C400CF1010C0FFAB4
:1014F0008CFCE245EBD84FF0000C002B59D90CFBCB
:1015000002F44FF0000B39F9148008F11904322C61
:101510003CD901252C46012A38D90CFB024639F961
:10152000167007F10A0EBEF1140F14D907FB08FE5E
:10153000BEF1000F0FDD09EB460E3EF902ECA7EB02
:101540000E071837302F06D831F916600F361E2EC9
:1015500084BF6D1CEDB2641C24B2A242DDD8142DF0
:1015600011D900244FF0010B002A1CD90CFB0245B5
:10157000641C31F8156039F8157024B2F61B20F898
:101580001560A242F2D8BBF1000F0CD10024002A52
:1015900009D90CFB0245641C31F8156024B220F80F
:1015A0001560A242F5D80CF1010C0FFA8CFC6345D2
:1015B000A5D80021BAF1000F8EBF8F4A0DF6040D99
:1015C000BDE8F08F30F8113022F81130491C09B213
:1015D0008A45F7D80DF6040DBDE8F08F2DE9F04FE0
:1015E000DFF818C29FB00DF11008BCE8F0008DE8DC
:1015F000F000BCE8F00088E8F000BCE8F0000DF175
:10160000200888E8F000DCE9004CCDE90C4C00260D
:10161000002B9CBF1FB0BDE8F08F0DF1380BA2F17D
:10162000010AEE464FF0000C654667466446BAF183
:10163000000F31D906FB024831F8189001EB480839
:10164000B8F80280A9EB08080FFA88F82BF8148084
:1016500008F10F08B8F11E0F9CBF0CF1010C1FFA26
:101660008CFC0BD9AC4507D9BCF1000F04D0654602
:10167000A4F1010C0CF0FF074FF0000C641CA4B2A5
:101680005445D7D3AC4507D9BCF1000F04D065460B
:10169000A4EB550C0CF0FF07052D23D906FB027CAB
:1016A00031F91CC00CF10F041E2C1BD93EF8174059
:1016B000002AA4EB0C0C0FFA8CF54FF0000C11D99A
:1016C00006FB02C43EF81C8031F81470A8EB050834
:1016D0000CF1010CA7EB08071FFA8CFC20F8147022
:1016E0006245EDD806F1010C1FFA8CF69E4299D3A3
:1016F0001FB0BDE8F08F2DE9F04F1E0004464FF0FB
:10170000000783B015468B460FFA82F90FFA86F868
:10171000384618BF374908D000FB05F23BF81220C5
:1017200021F81020401C8642F6D8DFF8D4A015F02E
:10173000010FDAF8000090F84C10ADF8001090F8A6
:101740004D10ADF80210B0F84A10ADF80410B0F822
:101750004800ADF806001ED0711E01FB05F06A1CA2
:10176000514300230BEB400004EB4101002E11D943
:10177000B5F1010C06D430F81C2021F81C20BCF176
:10178000010CF8D5A1EB4501891E5B1CA0EB4500BF
:10179000B342EDD3A3460CF068FF60B105F0CBFB7C
:1017A000012808D14FEA48000FFA80F806204FEAD6
:1017B0006909ADF802000CF05DFF68460CF06EFFA1
:1017C000414648460CF06FFF594620460CF070FF2A
:1017D0000CF05FFF15F0010F21D0002321462246B7
:1017E000002E1CD90020002D11D932F810C009E0BC
:1017F00094010110B4440110744F0110D0FC00108A
:10180000DC01011021F810C0401C8542EDD802EB2C
:101810004500821C5B1C01EB4501B342E2D3002171
:10182000002E53D9FE4A01FB05F332F8110034F8BB
:101830001330C01A00B222F811000028B4BF42428F
:1018400002461744F74AD2F800C09CF94420002A07
:10185000C8BF4FF00108BCBF4FF00008524232D061
:101860000028B4BF43420346BCF846C063452AD9AA
:101870000004530090FBF3FC0120012A84BF01FB0C
:10188000052AA5EB02091ED9B8F1000F0CD009EB0F
:10189000000301FB05330CFB00FE34F813B00BEB27
:1018A0002E4B24F813B00BE0AAEB000304EB430328
:1018B0000CFB00FE33F802BC0BEB2E4B23F802BCF2
:1018C000401C9042E0D3491CB142ABD3D64847619B
:1018D00003B03846BDE8F08F2DE9F0410746D34804
:1018E000D14EDFF854830578D148B2690478D148E5
:1018F000A0FB02304308A3EB8300831805FB04F030
:10190000420003EB830008EB00200CF06FFDB06990
:10191000421CB261002F08BFBDE8F081032A38BF26
:10192000BDE8F0810CF0A6FE214628460CF0BBFE77
:1019300008F5206308F5A062BF4938460CF0BDFEEB
:10194000BDE8F0410CF0A5BEB749888070472DE98D
:10195000F041BA4E8AB00546B348CDE90056A6F12B
:1019600080080C46CDF80880B0F9041003913F2997
:10197000C8BF3F2005DC11F1400FB8BF6FF03F003A
:1019800000DA0390002004900CF074FEA848A74FE2
:10199000017838780CF087FE68460CF093FE0890CA
:1019A0000CF077FEC4E90068BDF814002081BDF892
:1019B00016006081BDF81800A081BDF81A00E08112
:1019C000BDF81C002082BDF81E006082BDF81C001E
:1019D000BDF81E103A7801FB020035F910000AB07C
:1019E000BDE8F0812DE9FF4F85B00CF070FE0128B5
:1019F00013D00CF071FE01281CBF069890F900105E
:101A00000BD00698007801280ABF01290020012088
:101A1000069A117009B0BDE8F08F0CF062FE8349A0
:101A200000254FF002090C788149CC460A78012143
:101A300000917C490968B1F91AA10395CAF1000126
:101A40000EB200EB8401901E022853DD0098A2EB39
:101A50000902201AC31ECDE90123A2F1010BA0F156
:101A600001080098804538DD01EB400731F910206E
:101A70007B88D31A1BB2B342B8BFAA452FDB02281A
:101A80000ED9DDF808E086450ADD37F904ECA2EB53
:101A90000E0E764504DDB7F90470D71BBE421EDC7E
:101AA000CC45C8BFE34513DD13F10A0F10DA0A2D48
:101AB0000EDD051B071931F8155031F81770AD1AF6
:101AC000D21B12B22DB212F10A0F01DA0A2D06DC76
:101AD000401C80B21D468045C6DC039808B1012138
:101AE0008FE70CF101001FFA80FC019801EB440123
:101AF0006045B6DC002184E74B48406A70474A489D
:101B0000C06970474848006A70474D4870472DE9E2
:101B1000FF4FADF6240D0027DDF860A87C1E9B4624
:101B20008DF81478BAF1000F1CBF9AF800008DF8F8
:101B300014083E48464D4FF4006290F800803C483F
:101B400005F5A06106783F48007802903E4800788D
:101B500000903E48007801903348D0F80890CDF8C6
:101B60001818DDF82418CDF81018406A0CF03EFC67
:101B70000CF0BCFDCDF80C08B8B1DDF82428029BB0
:101B80001046DDF80C180CF0B6FD3248007802283B
:101B900004BFDDF80C080CF0B3FD2E4800780928CE
:101BA00004BFDDF824080CF0ABFD0198012831D901
:101BB00028480078042804BFDDF824080CF0A0FDB4
:101BC0002846DDF824180DF017FDCDF8100821483F
:101BD0000078052804BFDDF810080CF091FD1248CC
:101BE000817851B9012181704FEA480000FB06F26B
:101BF0001948DDF810180CF0F9FB16480078142885
:101C000004BF15480CF07CFDDDF81008A84208BFA1
